:020000040000FA
:107800005469616E59696E673130300000000000C4
:1078100054593230302E303830303030625F747925
:10782000424154333247313339474B3634464200B4
:1078300043414E5F5354440000000000000000002C
:1078400043414E5F43485F300000000000000000ED
:1078500043414E5F3530304B6270730000000000D2
:10786000E8070000E0070000DF070000000000005C
:020000040000FA
:1080000050330020DD800000E5800000E7800000A4
:108010000000000000000000000000000000000060
:10802000000000000000000000000000EF800000E1
:108030000000000000000000F380000095C3010074
:108040009D120100E1120100111301004113010012
:1080500071130100A1130100D113010001140100EB
:10806000311401006114010095140100A9140100EC
:10807000B9140100ED140100FD1401000D150100FB
:108080004115010085150100CD15010015160100EF
:108090005D160100A5160100B5160100E9160100E4
:1080A0001D1701004D17010081170100B5170100D0
:1080B000C5170100D5170100091801003D1801007E
:1080C000EF3FE8FF0448854600F02CFA00480047DF
:1080D000E9070200C046C0465033002016488047DA
:1080E00016480047FEE7FEE7FEE7FEE7FEE7FEE78D
:1080F000FEE7FEE7FEE7FEE7FEE7FEE7FEE7FEE758
:10810000FEE7FEE7FEE7FEE7FEE7FEE7FEE7FEE747
:10811000FEE7FEE7FEE7FEE7FEE7FEE7FEE7FEE737
:10812000FEE7FEE7FEE7FEE7FEE7FEE7FEE7FEE727
:10813000FEE7FEE7FEE7000099C90100C5800000E8
:1081400030B50B46014600202022012409E00D46EF
:10815000D5409D4205D31D469540491B2546954077
:1081600040191546521E002DF1DC30BD70B50024BB
:108170002546002801DA01244042002901DA0125C0
:108180004942FFF7DDFFAC4200D04042002C00D056
:10819000494270BDF0B51FB40646002082B00546C6
:1081A0004024019100901BE0019922460F46304681
:1081B00000F066F9049A059B801A994110D3104685
:1081C0001946224600F04CF9361A8F410197224693
:1081D00001200021009F00F043F938184D41009024
:1081E0002046641E0028DFDC019B009829463246A9
:1081F00007B0F0BDF0B51FB486B00020009001902C
:1082000002900698069980B204900798090C02041F
:108210000014114307900027089D099806913E46D7
:108220003C4603900398A9B20204000C0390049802
:108230002D0C154348430021224600F011F9C719BF
:10824000714110340E46402CECDB3846029A00F0A7
:1082500007F9009A019B80180090594102980191FA
:10826000103002904028CCDB00980BB0F0BD0346E4
:108270000B439B0703D009E008C9121F08C0042A5A
:10828000FAD203E00B780370401C491C521EF9D24D
:108290007047D2B201E00270401C491EFBD2704709
:1082A0000022F6E710B513460A4604461946FFF7C2
:1082B000F0FF204610BD30B504460020034600E024
:1082C0005B1C934203D2E05CCD5C401BF8D030BD18
:1082D0000321001D401E037812021A43491EF9D5DE
:1082E00010467047034603220870000A491C521EBC
:1082F000FAD518467047024670B54A40D30FDB07DF
:1083000040002DD04A002AD0010E140E00021202A5
:108310000919400A520A8418E50104465443000A28
:10832000120A2E045043A4194219200CC543AA185E
:10833000120C0125AD03521C521912047F3924047A
:1083400000D0521C104301D44000491EC2B20C069A
:10835000C0092018401C4008802A02D003E00020F9
:1083600070BD40084000002900DA0020184370BDAD
:1083700070B502464A40D50F40004A00ED0740085C
:108380005208002814D0002A12D0C40DD30D410287
:108390000120C0055202490A520AE41A09181218AB
:1083A0007D34914201D3641C00E04900002C01DAC5
:1083B000002070BD0023914201D3891A0343400875
:1083C00049000028F7D100290AD0914202D10121A9
:1083D000C90705E0914201D2012101E00121C94311
:1083E000E005C018401900F05CF870BD10B500221F
:1083F0009623114600F05DF810BDC20FD207400071
:1084000040080BD0C10D0723DB01C9184002090544
:10841000400A1143C208400711437047002001463B
:108420007047000010B5002904DB0124E407404236
:108430008C412146002B04DB1C460123DB07524202
:10844000A341994200D1904210BD00000122D20701
:10845000002800DB101A002900DB511A88427047FF
:1084600010B5202A04DB0146203A9140002010BDBF
:10847000914020239C1A0346E3401943904010BDCD
:1084800010B5202A04DB0846203AD040002110BD58
:108490000B46D340D0402024A21A914008431946ED
:1084A00010BD002904DA401C490001D140084000F9
:1084B000704770B40024050C05D11024000402D1CB
:1084C000002921D01124050E01D100020834050F26
:1084D00001D10001241D850F01D18000A41C0028BA
:1084E00001DB4000641C002908D020252E1B0D460E
:1084F000F540A14000D001212943084301061B1B80
:10850000000ADB1D02D5002070BC7047DB0518187F
:1085100080180029F8DA401C4900F5D170BC4008E9
:1085200040007047064C0125064E05E0E36807CC85
:108530002B430C3C98471034B442F7D3FFF7C6FDE9
:10854000241C0200441C020070B58C180578401CE5
:108550006B075B0F01D10378401C2A1106D102780A
:10856000401C03E006780E70401C491C5B1EF9D1CC
:108570002B0705D40023521E0DD40B70491CFAE7BB
:108580000378401CCB1A921C03E01D780D70491C27
:108590005B1C521EF9D5A142D8D3002070BD70B526
:1085A00007F01AF80524204618F0D8F800252846C8
:1085B00007F006F8204618F0D1F80126304606F0FC
:1085C000DBFF204618F0CAF8284606F0D5FF204603
:1085D00018F0C4F8304606F0F3FF204618F0BEF855
:1085E00070BDB0B506F0F8FF0524204618F0B6F8C7
:1085F0000125284606F0E4FF204618F0AFF828468B
:1086000006F0BAFF204618F0A9F8002006F0B4FFE3
:10861000204618F0A3F8B0BDF0B581B006F0C8FF51
:10862000052018F09BF808270026012006F0A4FF7B
:108630000524204618F092F8204618F08FF806F02E
:10864000ADFF0546204618F089F8002006F094FF9B
:10865000204618F083F876002E437F1E3806E4D1BA
:10866000F0B201B0F0BD70B50446002006F084FF02
:1086700006F0B2FF052018F071F80826E0B2C00934
:1086800006F09EFF0525284618F068F8012006F040
:1086900073FF284618F062F8002006F06DFF2846A8
:1086A00018F05CF8284618F059F86400761E300679
:1086B000E4D1052018F052F8012070BDF0B583B068
:1086C000019314460E4607460120384302900325C5
:1086D00004E000F08EF86D1E280631D000F067F837
:1086E0003846FFF7C0FF00F0A7F80028F1D1304668
:1086F000FFF7B9FF00F0A0F80028EAD100F057F822
:108700000298FFF7B0FF00F097F80028E1D1019838
:1087100002280BD3451E0026FFF77EFF2070FFF7CF
:108720003EFF641C761CF0B28542F5DCFFF774FF57
:108730002070FFF756FF00F05CF8202003B0F0BD7A
:10874000102003B0F0BDF0B583B01C46009201913B
:108750000290032504E000F04CF86D1E280623D09B
:1087600000F025F80298FFF77EFF00F065F800287A
:10877000F1D10198FFF777FF00F05EF80028EAD109
:10878000002C0CD00026009F3878FFF76CFF00F01B
:1087900053F80028DFD1761C7F1CA642F4D300F0EA
:1087A00028F8082003B0F0BD102003B0F0BDB0B52C
:1087B00006F012FF0524204617F0D0FF01252846B9
:1087C00006F0DAFE204617F0C9FF284606F0F8FE4C
:1087D000204617F0C3FF0025284606F0F1FE20468C
:1087E00017F0BCFF284606F0C7FE642017F0B6FF5E
:1087F000B0BDB0B506F0F0FE0524204617F0AEFF80
:108800000025284606F0B8FE204617F0A7FF2846A8
:1088100006F0D6FE204617F0A1FF0125284606F0F7
:10882000ABFE204617F09AFF284606F0C9FE6420EA
:1088300017F094FFB0BD0000B0B506F0B9FE0524F6
:10884000204617F08BFF012006F096FE204617F019
:1088500085FF0B4D06F0A2FE044606F087FE002CB5
:1088600002D06D1E2804F5D10525284617F076FFA5
:10887000002006F081FE284617F070FF2046B0BDAC
:1088800033210000034801780B2901D8491C0170ED
:108890007047C0463F2F002070B584B00025039577
:1088A00002950195009506F061FE0F20C6430E4C1F
:1088B0001036F1B2A0206A461023FFF744FF20468D
:1088C00017F04CFF204617F049FF912EF0D3A0205F
:1088D000B0216A461023FFF736FF204617F03EFF0F
:1088E0000248058004B070BD581B0000322F0020E4
:1088F00070B5022902D2EB24E0B270BD891EEB25CF
:108900000022134605E0401C5B1CDDB2A94225464F
:108910000EDB04786C40154604E034466E1C072DCF
:108920003546F0D26608E407F7D09A246640F4E7AB
:10893000E0B270BDF0B591B00C91417810AA117001
:1089400083781B025918C37804792402E3181B04A6
:1089500059180B0ED3700C0C94700D0A55700B91B6
:1089600008956918099409190A93C9180278D2431D
:108970008918427983791B029A18C379047A2402F0
:10898000E3181B049A188918130A0693C918130CC4
:108990000593C9180792120E04928918827AC37A35
:1089A0001B029A18037B0F90447B2402E3181B04DC
:1089B00098180918020A02928918020C0192891863
:1089C0000D910390000E0E9000200346014606E034
:1089D00032409A40D2B211435B1C082B0ED00126C4
:1089E00035469D400746024602E07F1C042FEFD02B
:1089F00010ACE45D2542F8D0521CF6E70E9C0D98B1
:108A00000019C3B20F98827B934205D0427A9142FB
:108A100002D1002011B0F0BD1021FFF769FF0C99C1
:108A2000CC72019A8A72029A4A72039A0A72049A62
:108A3000CA71059A8A71069A4A71079A0A710A9A46
:108A4000CA70099A8A70089A4A700B9A0A7011B013
:108A5000F0BDF0B58DB055220270002747720B783B
:108A60004370CA79059202728A790492C2714A7976
:108A7000039282710A7902924271CA7A0892427311
:108A80008A7A019202734E7AC6720C7A84720CAAA8
:108A900013704D782D02EB188D78C97809024919A9
:108AA0000904CB18190E01711D0CC57009931B0A1E
:108AB0000B90837038460A91D17007959570069394
:108AC000537031020919089A1202019BD21812043C
:108AD0005118089103990902029A8918059A1202FD
:108AE000049BD2181204511805913D463A4605E000
:108AF0002640AE4032436D1C082D0ED00124214685
:108B0000A9400346064602E05B1C042BF0D00CAFE4
:108B1000FF5C3942F8D0761CF6E70B9B5A72099835
:108B200006994018079940180A994018059A801824
:108B3000110A4018110C4018110E4018089A80189C
:108B4000110A4018110C4018110E4018563898732D
:108B500010211846FFF7CCFE0DB0F0BDF0B58FB078
:108B60000446FF20E070A07060700F20C0430290A8
:108B70000F302070704817F0F1FD704908686328C5
:108B800001D8642008606E4F002038806D4E01903F
:108B9000308008E00B99814222D338881030388029
:108BA00080B2A1286DD206F0E1FC3978A02003AA9A
:108BB0001023FFF783FD30802028EED103AD0BA9F1
:108BC0002846FFF7B7FEE97B8842E6D1287855288A
:108BD000E3D15D48017800290298DBD10846D9E746
:108BE0003888A0284DD8C0B20021019105E006F0D8
:108BF000BDFC3988C8B2A12943D2C1B2A02003AAC2
:108C00001023FFF75BFD3080398810313980202830
:108C100037D103AD07A92846FFF78CFEE97B8842D0
:108C2000E5D128785528E2D14748007800280299F4
:108C300000D1014607988842D9D240490A68962156
:108C400051430B9A824208D90818904219D30BA9B4
:108C50000E222046FFF70BFBC9E78918814210D38B
:108C600007A90E222046FFF702FB0BA80A99818173
:108C700007980B9008980C9009980D9038880190EF
:108C8000B5E72078617809020818A178E278120225
:108C9000511809040818401C24D100200190388084
:108CA000A020B02103AA1023FFF708FD3080202860
:108CB00018D103AD0BA92846FFF73CFEE97B88429B
:108CC00010D1287855280DD11F480078002800D1F0
:108CD00002900B980299884204D20BA90E222046DA
:108CE000FFF7C5FA2078617809020818A178E278C0
:108CF0001202511809040818401C0CD10020E0721F
:108D0000A07260722072E071A07160712071E070D9
:108D1000A070607020700198388020786178090216
:108D20000818A178E27812025118090408180749B6
:108D3000086030880FB0F0BD701101002C2F0020AA
:108D4000322F0020282F00202B2F0020382F00202A
:108D5000F0B581B000910646214800250570002A33
:108D60002ED01446C036631B71190F200840102204
:108D7000101A834200D303461A480278102A01D001
:108D8000042A1AD1C809FE2707405F2F13D80127EC
:108D9000B8436038C0B29E3282420CD3009A521956
:108DA000C9B2DFB23B46FFF789FC0F490880ED19D5
:108DB000A542D8D304E0082000E004200A49088036
:108DC000094801880020042902D0082900D0012088
:108DD00003490870411E8841400001B0F0BDC04603
:108DE0003E2F00202A2F00203C2F00200A4A01237A
:108DF00013700A4A10700A4A11600A4A0021116071
:108E0000042801D105218901102801D11D208101EB
:108E1000054801807047C0462B2F00202A2F0020D4
:108E20002C2F0020382F0020302F0020F0B587B0E5
:108E3000994D00262E80994B1B688B4224D1994C6A
:108E40002188202925D1029000920196964C002776
:108E50002760964D964E2878062809D806F086FB9E
:108E60002068401C2060B042F5D38D480421018069
:108E70002F70904C20880107029B31D08848202118
:108E80000180854D019E0BE001204002844908804D
:108E900006E003A8FFF762FE208081488021018060
:108EA0007F4800883F2807DD874988420BDC40283F
:108EB00012D0802810D010E004280DD008280AD045
:108EC000202809D009E001214A02904204D0C902B9
:108ED000884201D001E002262E80288807B0F0BD2C
:108EE000A128019E00D32780009A012A6A4D1ED135
:108EF000187B012856D1DF719F715F711F711F733D
:108F0000587B012804D1DF729F725F721F725F73FA
:108F100003AF38461946FFF79CFDF87320880028F8
:108F200046D01038C1B2A02003AA102344E0002A82
:108F3000B6D1614801780029B2D00270187859780A
:108F4000090208189978DA781202511809040818E9
:108F50005A490978002901D00F21C943884233D2E8
:108F6000274603AC20461946FFF773FDE0733978B6
:108F7000A02010232246FFF7E6FB029A484908800A
:108F800008288DD13888103038801078517809023F
:108F900008189178D2781202511809040818484923
:108FA00008607DE7597B012911D10128A3D0A7E7EB
:108FB000A02003AA10230146FFF7C5FB384908800B
:108FC0003D48009901706BE70120C0025EE73D4813
:108FD0000078012812D103AC20461946FFF739FD6D
:108FE000E073A020B02110232246FFF7ACFB2C49F0
:108FF00008800828E4D133480770E1E718785978E9
:10900000090208189978DA78120251180904081828
:109010002B490968214A12685118884203D2204816
:1090200040210180CCE725490978002901D00F2192
:10903000C94388422DD203AF384619461C46FFF774
:1090400008FDF8731B480178A02010233A46FFF76B
:109050007AFB134908800828B2D1164908881030D5
:1090600008802078617809020818A178E278120255
:109070005118090408181249086008490A6815219E
:109080005143FFF75DF800299AD101200D4908707E
:1090900096E70120C00291E7442F00202C2F0020EA
:1090A000422F0020282F0020482F00203F2F002093
:1090B000818D5B00322F0020342F00202B2F0020C9
:1090C000382F0020402F0020FF010000F0B585B0B0
:1090D0000646434C0027278004921018414A128804
:1090E000904241D201910397404F00200290386096
:1090F0003F4C404D2078052809D806F037FA3868EB
:10910000401C3860A842F5D33748042101800298FA
:1091100020703948018839480278102A01D0042A81
:1091200032D188190346C033049C651A0F240440C9
:109130001020001B854200DB0546DC09603C01264F
:109140003002E7B27F09052F12D3B443E6B29E3254
:10915000B242234C039F0DD301984218D9B2EBB20F
:109160003046FFF7F0FA05E01F482021018011E0AA
:109170001B4C039F1C49088008280BD1E8B21E4AEB
:1091800011880818108005E0012080021649088027
:10919000134C039F144800881F2809DD202813D092
:1091A00001210A0290420FD0890288420CD00CE0C3
:1091B000042809D0082808D10F480088049988425B
:1091C00001D3022700E001272780208802210143E4
:1091D000022902D1084900220A8005B0F0BDC0462C
:1091E000442F0020302F0020422F0020482F002045
:1091F0003F2F0020818D5B004C2F00202A2F002064
:10920000F0B585B0044600200190042C6FD20BF01D
:109210009FFF002801D10CF01BF80020009000BF38
:109220000098401C00900BF093FF039003980028D7
:1092300003D0484900988842F2D30398002856D1B9
:10924000042145480BF066FF444845490880210148
:10925000444A515C4900404A505A41490A88012118
:10926000090300F055F902900120049020013D49C6
:1092700040184078002801D100264BE020013949F0
:1092800040184078012802D13548068842E0200184
:1092900034494018407802282AD120014018057925
:1092A0002901304A515C49002B4A505A2C490A88FE
:1092B0000121090300F02CF9064628012A49431828
:1092C0002801284940180289280140180021C76850
:1092D0003046B84706462801224BC018C2882801EC
:1092E000C0188178304600F087F8064612E02DE07D
:1092F00020011C4940184078032804D02001401860
:109300004078132804D1200116494018868801E0CE
:10931000002004900498002818D020011249431816
:109320002001104940180289200140183146C768C1
:109330000298B847019020010A4BC018C28820014A
:10934000C0188178019800F057F80190019805B095
:10935000F0BD000050C3000006010020881300008B
:1093600000010020C012020000130200F8B50546FB
:109370000E4614460020009001211C4801751C482F
:10938000007888431A490870084680780821084305
:109390001749887000208871084600780121084329
:1093A0001349087008460572002717E01048007836
:1093B000802108430E49087000BF0E48007D002838
:1093C000FBD000200B4908750948C0892080A41CE7
:1093D0000748C1890098081800907F1CB742E5D360
:1093E00031460098FEF7ACFE80B2F8BD4061004007
:1093F000005004404060004010B50346012908D1E8
:10940000094CA41A9C4202D99C18A0B20BE0064851
:1094100009E0022906D1934202DD9C1AA0B202E0C3
:10942000002000E0184610BDFFFF000010B5044604
:109430000121202002F00AF80020324908700121A1
:1094400031480175002031490875152016F06EFE6F
:109450002C488078E17808432A498870084680784B
:1094600021780843274988702078802806D108464B
:109470000079E17949000843224908712148807840
:10948000E17A08431F498870A078002803D1084674
:10949000007908710FE0A078012806D119480079F9
:1094A000602108431749087105E0164800798021BA
:1094B00008431449087113488079217908431149F8
:1094C000887108468079617908430E498871207A4D
:1094D000C872607A88720846007838218843094942
:1094E0000870084600786178C9000843054908708B
:1094F000A07A0873084600780121084301490870E2
:1095000010BD000000500440406100404060004039
:10951000F8B504460E461746002E01D100250FE08F
:10952000A64201DC3D460BE00094009C20467843B7
:10953000009031460098FEF703FE0090009885B237
:109540002846F8BD0146042904D28A00024BD218ED
:10955000508800E0002070471C29002001460429A3
:1095600003D28A00024B985C00E0002070470000A4
:109570001C290020FFB587B004460898844203DA0E
:109580000A988068002802D12448019042E0089897
:10959000001B82B20292002625460A9880680021AC
:1095A0002F463A463346049605910690FEF722FE72
:1095B00005460E46002328463146029AFEF7EAFD8C
:1095C00005460E46304600210A46494050400143B8
:1095D00002D0124801901DE003950A98C068039DCF
:1095E000A84202D30020019014E00A98C1680398B1
:1095F000401A039009990398FEF7A2FD039003987F
:10960000000C0004002802D00448019002E00398F6
:1096100080B2019001980BB0F0BD0000FFFF000088
:1096200010B5084800788021884306490870012158
:1096300005480175002005490875152016F076FDCE
:1096400010BD0000005004404061004040600040F8
:10965000F8B505460E4614461F4621462846FEF735
:1096600085FD80B2F8BD0000FFB587B006460A98B8
:109670004068002801D1029035E00A9801684068EE
:1096800008180390002534460021274603980695C4
:109690000491059038462946049B059AFEF7AAFDD9
:1096A00004460D460A984068024600230190204671
:1096B0002946FEF76FFD04460D4600232046294645
:1096C000099AFEF767FD04460D46284607492140E2
:1096D000002359405840014303D00448C04302903E
:1096E00001E0A0B2029002980BB0F0BD0000FFFFB5
:1096F00010B5FE4800688079030016F0FDFC0705F0
:109700009ED8F5F4F3F2F100F848006840790300C0
:1097100016F0F2FC0805138A2A8A468A638A12F038
:1097200071FD0020F1490968C873F048006840796C
:10973000401CEE49096848717DE0ED494969EB4AF2
:109740001268D27A885C12F0D5FDE848006840794A
:10975000401CE64909684871E44800684079401CAB
:10976000E2490968487166E009F0D8FF002810D185
:1097700012F0C0FDDD4800684079401CDB490968F3
:109780004871DA4800684079401CD8490968487136
:1097900005E012F061FD0020D449096848714AE0F3
:1097A00009F0BCFF002811D1112012F0A3FDCF4811
:1097B00000684079401CCD4909684871CB48006871
:1097C0004079401CC9490968487105E012F044FD20
:1097D0000020C649096848712DE009F09FFF002864
:1097E0001BD1C2480068C07A401CC0490968C872D1
:1097F000BE480068C07ABE49097888420DDB002067
:10980000BA490968C872B94909684862B748006826
:109810008079401CB5490968887112F01DFD00204F
:10982000B2490968487106E012F016FD0020AF4900
:109830000968487100BF00BF32E3AC480068407C53
:10984000002817D0AA48C068002803D0A848C168DB
:10985000192088470020A54909684862A348006884
:109860008079401CA1490968887100209F490968D6
:1098700048711BE09D480068406A282807D29B4831
:109880000068406A401C9949096848620EE000205F
:10989000964909684862954800688079401C934958
:1098A000096888710020914909684871F8E28F4879
:1098B00000684079030016F01FFC080518A42FA4C7
:1098C0004CA480A412F09EFC002088490968C8734B
:1098D000864800684079401C84490968487197E0CF
:1098E000D4E2C7E230E25DE194E0814949697F4A10
:1098F0001268D27A885C12F0FDFC7C4800684079DE
:10990000401C7A4909684871784800684079401CD1
:109910007649096848717BE009F000FF002811D101
:10992000012012F0E7FC714800684079401C6F4943
:10993000096848716D4800684079401C6B490968A6
:10994000487105E012F088FC0020684909684871F8
:109950005EE009F0E3FE002828D164490968C97A6D
:1099600024225143634A12688918604A1268D27BE4
:10997000885C12F0BFFC5D480068C07B401C5B49FE
:109980000968C87359480068C07B242814D3574815
:1099900000684079401C554909684871534800687F
:1099A0004079401C51490968487105E012F054FCA7
:1099B00000204E49096848712AE009F0AFFE0028EE
:1099C00018D14A480068C07A401C48490968C872E2
:1099D00046480068C07A4649097888420ADB002078
:1099E00042490968C872414800688079401C3F4973
:1099F0000968887112F030FC00203C490968487100
:109A000006E012F029FC002038490968487100BFBF
:109A100000BF45E2354800684079030016F06CFB52
:109A20000A0614B92BB948B978B995B912F0EAFB0E
:109A300000202E490968C8732C4800684079401CF2
:109A40002A4909684871ABE029494969274A1268DF
:109A5000D27A885C12F04EFC244800684079401CA1
:109A6000224909684871214800684079401C1F4913
:109A70000968487194E009F051FE002811D14A208C
:109A800012F038FC194800684079401C17490968F1
:109A90004871164800684079401C144909684871AB
:109AA00005E012F0D9FB002010490968487177E001
:109AB00009F034FE002824D1FF2012F01BFC0B48D3
:109AC0000068C07B401C09490968C87307480068E2
:109AD000C07B24281BD3054800684079401C0349FB
:109AE0000968487101480068407905E0CC0700200A
:109AF000102F0020C8070020401CEA49096848715F
:109B000005E012F0A9FB0020E6490968487147E02A
:109B100009F004FE002811D1FF2012F0EBFBE14810
:109B200000684079401CDF4909684871DD480068D9
:109B30004079401CDB490968487105E012F08CFB54
:109B40000020D849096848712AE009F0E7FD00289B
:109B500018D1D4480068C07A401CD2490968C8723C
:109B6000D0480068C07AD049097888420ADB0020D2
:109B7000CC490968C872CB4800688079401CC94943
:109B80000968887112F068FB0020C64909684871AD
:109B900006E012F061FB0020C2490968487100BF6D
:109BA00000BF7DE1BF4800684079030016F0A4FAC9
:109BB0000C0715C32CC349C366C382C39FC312F0ED
:109BC00021FB0020B7490968C873B648006840798E
:109BD000401CB44909684871B4E0B3494969B14AC5
:109BE0001268D27A885C12F085FBAE480068407932
:109BF000401CAC4909684871AA4800684079401C7B
:109C0000A849096848719DE009F088FD002811D134
:109C1000772012F06FFBA34800684079401CA149EF
:109C2000096848719F4800684079401C9D4909684F
:109C3000487105E012F010FB00209A49096848714C
:109C400080E009F06BFD002811D10C2012F052FBCE
:109C5000944800684079401C9249096848719148CD
:109C600000684079401C8F490968487105E012F08E
:109C7000F3FA00208B490968487163E009F04EFD52
:109C8000002810D112F036FB864800684079401C4D
:109C9000844909684871834800684079401C8149BB
:109CA0000968487105E012F0D7FA00207D4909687B
:109CB000487147E009F032FD002811D1132012F05D
:109CC00019FB784800684079401C7649096848715A
:109CD000744800684079401C72490968487105E081
:109CE00012F0BAFA00206F49096848712AE009F0B9
:109CF00015FD002818D16B480068C07A401C6949DE
:109D00000968C87267480068C07A6749097888425C
:109D10000ADB002063490968C872624800688079DC
:109D2000401C60490968887112F096FA00205D496C
:109D30000968487106E012F08FFA00205949096855
:109D4000487100BF00BFABE056480068407903008F
:109D500016F0D2F9080513872A874787638712F020
:109D600051FA00204F490968C8734E48006840798D
:109D7000401C4C49096848717AE04B494969494A95
:109D80001268D27A885C12F0B5FA464800684079C9
:109D9000401C444909684871424800684079401CA9
:109DA00040490968487163E009F0B8FC002811D106
:109DB000492012F09FFA3B4800684079401C39491D
:109DC00009684871374800684079401C354909687E
:109DD000487105E012F040FA0020324909684871E4
:109DE00046E009F09BFC002810D112F083FA2D48C0
:109DF00000684079401C2B4909684871294800686F
:109E00004079401C27490968487105E012F024FA9E
:109E100000202449096848712AE009F07FFC0028E5
:109E200018D120480068C07A401C1E490968C872D1
:109E30001C480068C07A1C49097888420ADB002067
:109E400018490968C872174800688079401C15498C
:109E50000968887112F000FA0020124909684871F7
:109E600006E012F0F9F900200E490968487100BFB8
:109E700000BF15E000200B4909688871094909688D
:109E80004871062007490968C87009E012F0E4F932
:109E9000002004490968487102490968887100BFB7
:109EA00000BF10BDCC070020102F002010B56A485D
:109EB00000684079030016F01FF9090610C627C68E
:109EC00044C6608EC60012F09DF963480068407970
:109ED000401C614909684871BCE0604949695E4AB3
:109EE0001268D27A885C12F005FA5B480068407903
:109EF000401C594909684871574800684079401C1E
:109F0000554909684871A5E009F008FC002811D1FD
:109F10007F2012F0EFF9504800684079401C4E490C
:109F2000096848714C4800684079401C4A490968F2
:109F3000487105E012F090F900204749096848711E
:109F400088E009F0EBFB002810D112F0D3F9424869
:109F500000684079401C4049096848713E480068E3
:109F60004079401C3C490968487105E012F074F9D9
:109F700000203949096848716CE009F0CFFB0028DE
:109F800022D135480068C07A401C33490968C8723C
:109F900031480068C07A3149097888420FDB0020D7
:109FA0002D490968C8722C4800684079401C2A492C
:109FB00009684871002028490968486208E00020C3
:109FC00025490968487103E0002023490968487160
:109FD00012F042F93EE020480068407C002816D08C
:109FE0001E48C068002803D01C48C1681920884753
:109FF00000201949096848621749096848711649DB
:10A0000009688871052014490968C8701AE0124867
:10A010000068406A282807D20F480068406A401C40
:10A020000D49096848620DE000200B490968486243
:10A030000949096848710849096888710520064975
:10A040000968C87006E012F007F9002002490968A3
:10A05000487100BF00BF10BDCC070020102F0020AA
:10A0600010B50024F7480068807A01287ED1F548B1
:10A070000068C07900287AD0F2480068807900280A
:10A0800004D0012874D0022873D191E1ED48006812
:10A09000007B24286ED2EB480068C07901287AD171
:10A0A000002475E0E7480068C07A24214843E64967
:10A0B00009684018E3490968097B415CE148006888
:10A0C000C07A24225043E14A12688018DD4A12689F
:10A0D000127B805C814229D0DA480068C07A242152
:10A0E0004843DA4909684018D6490968097B415C48
:10A0F000D4480068C07A24225043D34A126880189A
:10A10000D04A1268127B8154CE480068407B2428D4
:10A1100005D3CC480068007BCA4909684873C94820
:10A120000068007BC7490968887308E0C548006873
:10A13000407B242803D20120C24909688871C148A4
:10A140000068007B401CBF4909680873BD4800686F
:10A15000007B242808D3BB480068407B242803D216
:10A160000120B84909688871B64805E0D3E1CDE11E
:10A1700069E0BAE138E00EE00068007B242804D2F0
:10A18000B04800688079012800D103E0601CC4B2A7
:10A19000242C87D356E0002413E0AA480068C07A34
:10A1A00024214843A94909684018015DA548006871
:10A1B000C07A24225043A44A126880180155601CBA
:10A1C000C4B2242CE9D300209E4909684873232097
:10A1D0009C490968887301209A490968887124207C
:10A1E0009849096808732DE00020964909680873AA
:10A1F00094480068C07A401C92490968C872914826
:10A200000068C07A92490978884217DB8D48006857
:10A21000007C012804D102208A490968887106E07F
:10A22000002088490968887186490968C87100203A
:10A2300084490968C8728349096808740020814903
:10A240000968487161E17F4800684079030015F0B2
:10A2500053FF080513A62AA651A68EA60120794908
:10A260000968087411F0CEFF764800684079401CF8
:10A2700074490968487199E075494969714A1268D9
:10A28000D27A885C12F036F86E4800684079401C3B
:10A290006C49096848716B4800684079401C6949FD
:10A2A0000968487182E009F039FA00281BD1654934
:10A2B0000968497B491CC8B212F01CF86148006863
:10A2C000407B60490968C8735E4800684079401C5B
:10A2D0005C49096848715B4800684079401C5949ED
:10A2E0000968487105E011F0B7FF00205549096879
:10A2F00048715BE009F012FA00282BD15149096836
:10A30000C97A24225143504A126889184D4A12686A
:10A31000D27B885C11F0EEFF4A480068C07B401C8D
:10A3200048490968C87347480068C07B45490968BF
:10A33000897B88421ADD434800684079401C4149C6
:10A34000096848713F4800684079401C3D490968E8
:10A3500048710BE011F080FF3A480068407B3949B2
:10A360000968C87300203749096848711EE009F080
:10A37000D5F900280CD13349096888712420314966
:10A380000968C8732F49096848732E49096888739A
:10A3900011F062FF00202B490968487106E011F0B6
:10A3A0005BFF002027490968487100BF00BFACE08F
:10A3B000244800684079030015F09EFE08050F8EC2
:10A3C000268E4C8E688E11F01DFF1E480068407965
:10A3D000401C1C490968487185E01D494969194AB2
:10A3E0001268D27A885C11F085FF164800684079BF
:10A3F000401C144909684871124800684079401CA3
:10A400001049096848716EE009F088F9002811D1F7
:10A41000492011F06FFF0B4800684079401C094942
:10A4200009684871074800684079401C0549096877
:10A43000487105E011F010FF0020024909684871D9
:10A4400051E00000CC070020C8070020C40700200E
:10A45000102F002009F062F9002810D111F04AFFF6
:10A460009C4800684079401C9A490968487199489D
:10A4700000684079401C97490968487105E011F06F
:10A48000EBFE00209349096848712CE009F046F979
:10A4900000281AD18F480068C07A401C8D4909688D
:10A4A000C8728C480068C07A8B49097888420CDBF6
:10A4B000002088490968C8728649096888718549F9
:10A4C0000968487183490968C87111F0C5FE002008
:10A4D00080490968487106E011F0BEFE00207D4900
:10A4E0000968487100BF00BF0FE011F0B5FE002001
:10A4F0007849096848717749096888717549096818
:10A50000087374490968C87200BFE2E0002071490D
:10A5100009688872DDE06F480068807A0228F4D10B
:10A520006C480068007A002879D06A480068407951
:10A53000030015F0E1FD0B0711BB25BB41545EBBC9
:10A540007590BB0011F05EFE624800684079401CC7
:10A55000604909684871B7E05F494969087811F0B6
:10A56000C9FE5C4800684079401C5A490968487136
:10A57000584800684079401C564909684871A3E072
:10A5800009F0CCF8002810D111F0B4FE5148006851
:10A590004079401C4F49096848714E48006840792D
:10A5A000401C4C490968487105E011F055FE002037
:10A5B00048490968487187E009F0B0F8002807D1D8
:10A5C000444800684079401C42490968487103E0EA
:10A5D000002040490968487111F03EFE74E011F016
:10A5E00011FE3C4800684079401C3A4909684871AE
:10A5F0006AE0394949690978491CC8B211F07AFE04
:10A60000344800684079401C324909684871314833
:10A6100000684079401C2F490968487154E054E0B3
:10A6200009F07CF800280FD111F0BEFD2949096816
:10A630008870012011F032FE264800684079401CE5
:10A6400024490968487105E011F006FE00202149FF
:10A650000968487138E01F480068807811280CD1DB
:10A6600000201C4909680872AA201A4909688870E4
:10A67000002018490968487011E0164800684078C1
:10A68000401C144909684870124800684078032843
:10A6900005D309F0E3F800200E490968487011F06D
:10A6A000DBFD00200B49096848710DE011F0D4FD75
:10A6B0000020084909684871064909684870AA20BD
:10A6C00004490968887000BF03E000200149096857
:10A6D000887210BDCC070020102F0020F0B5054671
:10A6E0000C4616461F462088482806DA3A46294670
:10A6F000304604F079FF012800D0F0BD2088C0006A
:10A700002E502088401C208000BFF6E710B502467E
:10A710009000074BC018405C002802D00320C043C3
:10A7200010BD01209300024C1B1958540020F7E77C
:10A73000902A002070B5002508E06D1C1B4885425A
:10A7400002D20AF0B1FD01E0002503E00AF000FDAD
:10A750000028F2D100BF022100200AF007FD0321EA
:10A7600000200AF003FD052100200AF0FFFC07216C
:10A7700000200AF0FBFC002408E00020A1000C4AA5
:10A780005054A10089184880601CC4B2042CF4D332
:10A7900001200849087000204870052088700020BA
:10A7A000C87005480549088070BD000050C300000E
:10A7B0001C29002002010020881300000001002055
:10A7C000F8B58D480078030015F096FC06040516D0
:10A7D0003D5EFDFC0EE10AF03BFD00208649C8709D
:10A7E000487008468078002802D10320087002E0F3
:10A7F000022081490870FDE07F488078002804D05D
:10A800007D488078401E7C4988700AF0A1FC0028B1
:10A810000BD10AF01DFD00207749C87008468078EA
:10A8200000280FD1032008700CE07348C078401C4A
:10A830007149C8700846C078052803D30520087000
:10A840000AF032FDD6E00AF083FC00280ED1042184
:10A850006A480AF05FFC00206749C8704870684881
:10A86000684908800420644908700CE06248C07898
:10A87000401C6149C8700846C078052803D30520EC
:10A8800008700AF011FDB5E05B49497809015E4A9C
:10A89000515C4900594A505A5A490A880121090312
:10A8A000FEF736FE009001255348407800015649D6
:10A8B00040184078002801D100243CE04E48407800
:10A8C0000001514940184078012802D14D480488C0
:10A8D00031E04948407800014B494018407802284F
:10A8E00012D1454949780901474A89180879FEF784
:10A8F00029FE0446404949780901434A89180879E4
:10A90000FEF72CFE054616E03B48407800013E4924
:10A9100040184078032806D0374840780001401896
:10A920004078132806D13448407800013649401851
:10A93000848800E00025002D2FD02F4840780001AA
:10A94000324943182C48407800012F4940180289A9
:10A9500029484078000140182146C7680098B84748
:10A960000646254840780001274BC018C288224877
:10A9700040780001C01881783046FEF73DFD06465C
:10A980001D484078800022494018468001201A491D
:10A99000497889001E4A50540AE000201649497837
:10A9A00089001B4A89184880134949788900505406
:10A9B00011484078401C10494870084640780428E7
:10A9C00009D301E013E007E00AF042FC00200A4945
:10A9D0004870032008700DE00AF0BAFB002803D18C
:10A9E00001200549087001E00AF05EFC02E0FFF773
:10A9F000A1FE00BF00BFF8BD02010020060100203B
:10AA00008813000000010020C012020000130200A1
:10AA10001C29002010B50AF065FB002405E0002089
:10AA2000A100074A5054601CC4B2042CF7D3002084
:10AA3000044908700520887003480449088010BD47
:10AA40001C290020020100208813000000010020C2
:10AA500070B50446002000F0AFF8002000F0DAF8EE
:10AA6000002000F09BF8002000F0C4F8002000F067
:10AA700087F8002000F0AEF800BF012000F08EF84B
:10AA8000012000F0B7F8002521E0002000F086F852
:10AA9000002000F0AFF880202040002806D00120E0
:10AAA00000F08AF8012000F0B5F805E0002000F081
:10AAB00083F8002000F0AEF800BF012000F06EF82F
:10AAC000012000F097F86006040E681CC5B2082D3E
:10AAD000DBDB012000F054F8012000F07BF870BDB2
:10AAE00070B504460D46012000F066F8012000F024
:10AAF00091F8002000F052F8002000F07BF80020D0
:10AB000000F03EF8002000F065F800BF012000F0E2
:10AB100045F8012000F06EF8002628E0002000F043
:10AB20003DF8002000F066F880202040002803D087
:10AB3000012000F041F802E0002000F03DF8802004
:10AB40002840002803D0012000F064F802E0002033
:10AB500000F060F800BF012000F020F8012000F0B4
:10AB600049F86006040E6806050E701CC6B2082E71
:10AB7000D4DB012000F004F8012000F02BF870BDB8
:10AB800010B50446002C04D0812103200AF01EFCDD
:10AB900003E0802103200AF019FC10BD10B5044623
:10ABA000002C04D0812104200AF010FC03E0802155
:10ABB00004200AF00BFC10BD10B50446002C04D094
:10ABC000812102200AF002FC03E0802102200AF029
:10ABD000FDFB10BD10B50446002C04D081210448B3
:10ABE0000AF0F4FB03E0802101480AF0EFFB10BDFE
:10ABF0000107000010B50446002C05D08121072074
:10AC000000020AF0E3FB04E08021072000020AF0C2
:10AC1000DDFB10BD10B50446002C04D08121044892
:10AC20000AF0D4FB03E0802101480AF0CFFB10BDFD
:10AC30000207000010B5F920FFF70AFF8820FFF790
:10AC400007FF9020FFF704FF9820FFF701FF08217E
:10AC50000846FFF745FFE820FFF7FAFE12210846F5
:10AC6000FFF73EFFA020FFF7F3FE70210846FFF735
:10AC700037FFA820FFF7ECFE70210846FFF730FFF2
:10AC8000B020FFF7E5FE70210846FFF729FFB82046
:10AC9000FFF7DEFE00210846FFF722FFC020FFF786
:10ACA000D7FE00210846FFF71BFFC820FFF7D0FEA4
:10ACB00000210846FFF714FFD020FFF7C9FE2F211F
:10ACC0000846FFF70DFFD820FFF7C2FE2F210846E8
:10ACD000FFF706FFE020FFF7BBFE2F210846FFF736
:10ACE000FFFE4020FFF7B4FE00210846FFF7F8FE04
:10ACF0000A20FFF7ADFE002405E000210846FFF71B
:10AD0000EFFE601CC4B25A2CF7DB00240AE00020DE
:10AD10000B4908550B4908550B4908550B4908556F
:10AD2000601CC4B25A2CF2DB8120FFF791FE002098
:10AD3000074908708870C8700871487010BD00001D
:10AD4000442600209E260020F826002052270020BE
:10AD5000D700002010B58020FFF77AFE10BD00005C
:10AD60000020044908700120034908700020487041
:10AD700070470000DC000020D700002010B54848D4
:10AD8000007800287AD046488078030015F0B4F99E
:10AD90000604434A535A687E414800794149085C99
:10ADA0003F490979404A515C884209D13C480079C1
:10ADB0003E49085C3A4909793D4A515C88421BD0BA
:10ADC000374800793749085C35490979364A505483
:10ADD000334800793549085C31490979344A50547F
:10ADE0002F48C078002803D004202D49887011E036
:10ADF00001202B4988700DE000202949C8700846C1
:10AE00000079401C0871084600795A2802DB0020AE
:10AE10000871087041E04020FFF71AFE0220204927
:10AE200088703AE01E4A11791079FFF759FE032025
:10AE30001B49887031E00A20FFF70AFE04201849F8
:10AE400088702AE0164A1279194B995C144A1279D3
:10AE5000154B985CFFF744FE0520114988701CE0F3
:10AE60000F480079401C0E490871084600795A289D
:10AE700005DB002008710870C87003E00EE00120B7
:10AE80000749C87000200649887006E00020044980
:10AE900008708870C870087100BF00BF10BD000046
:10AEA000D7000020442600209E260020F8260020FF
:10AEB0005227002010B511F0DDFD012837D1072001
:10AEC00009F0F0F9002810D01C480078052805DAB0
:10AED0001A480078401C1949087016E005201749E7
:10AEE00008700020164908700FE015480078052802
:10AEF00005DA13480078401C1149087005E0052068
:10AF00000F49087000200D4908700C48007805288A
:10AF100006D14B22D2000021012013F0A7FA0BE04A
:10AF20007D22D2000021012013F0A0FA04E00022CB
:10AF30001146012013F09AFA10BD00001D000020F8
:10AF40001C00002000200349087248708870486087
:10AF500070470000540A002058221152704710B563
:10AF600004460121022000F071FA0021022000F0C5
:10AF70006DFA10BD014600205322525C10231A4086
:10AF8000002A08D05322525C0C231A409210032A44
:10AF900018D1032016E05422525A0123DB031A4031
:10AFA000002A0ED05322525C0C231A409210032A1E
:10AFB00005D05322525C9207920F032A01D102203E
:10AFC00000E0012070470246002058239B5A0B40A6
:10AFD000002B01D0012000E0002070470146002234
:10AFE0006020405AFF231B0218400005020F100189
:10AFF000014BC018704700000055044010B5002AEE
:10B000000AD056231B5A0C0223435624235256239C
:10B010001B5A8B43235209E056231B5A0C02A343AD
:10B020005624235256231B5A0B43235210BD0000B3
:10B03000F8B504460D46012700263448844203D162
:10B040000121022000F002FA2878401EA07020881A
:10B05000FF210131084320802088400840002080E3
:10B06000A878401EC1B25A20015568790007000C2B
:10B07000E97909020843A97908435C210853288922
:10B0800081B240200153A868C000C10C4220015386
:10B09000A88981B244200153E868C000C10C462051
:10B0A0000153288A81B2482001532869C000C10C8D
:10B0B0004A200153A88A81B24C2001536869C0001C
:10B0C000C10C4E2001535020005B2979090208432E
:10B0D000502108535020005B2979884350210853A0
:10B0E00000E0761C5020005B4007400F2979884221
:10B0F00002D007488642F4D15020005B4007400F41
:10B100002979884200D000273846F8BD0054044011
:10B11000FFFF000030B5034600201C898C4209DD8A
:10B12000082A05D218244C431D682C19A05C02E0A3
:10B13000002000E0002030BD10B5024613898B428C
:10B1400005DD18234B431468E318987C00E00020C9
:10B1500010BD0146FF22C889C007C00F00280AD0D1
:10B160000120C88100E0521EC889C007C00F002816
:10B1700001D0002AF7D1C889C007C00F00280FD11D
:10B180000220C8810420C881487A400840004872E3
:10B19000487A38239843487200204872012070474B
:10B1A0000020FCE70246507A012318435072507A7F
:10B1B0000B78DB0018435072087A012808D1888880
:10B1C00050814868000C0123DB031843908108E09C
:10B1D000087A002805D15081486880001A4B184031
:10B1E0009081487A012804D1507A40231843507244
:10B1F00006E0487A002803D1507A402398435072E1
:10B200000878002811D1C87A1072087B1070487B2A
:10B210005070887B9070CB7BD370087C10714B7C16
:10B220005371887C9071CB7CD371887A002803D0CD
:10B230000120C002D08101E00820D081FF20013030
:10B24000D081012070470000FC1F0000002904D0BD
:10B25000427A80231A43427203E0427A80239A435F
:10B260004272704730B5024600200F4B5024A45A5A
:10B270000D022C435025AC525024A45A8C43AC529E
:10B2800000E05B1E5024A45A6407640F8C4201D076
:10B29000002BF6D15024A45A6407640F002C01D06F
:10B2A000002000E0012030BDFFFF0000827A8023F3
:10B2B0001A40802A00D081727047000070B50446A1
:10B2C00000250023002D02D0012660200653042013
:10B2D000C88188890126F6033040002808D0012063
:10B2E00010728889C004C0084E893043506006E05F
:10B2F0000020107288890F4E304080105060087A0C
:10B30000D072002304E0CE5C10460C30C6545B1CA7
:10B31000D07A9842F7DCC88904263040002804D14E
:10B32000C889F6023040002801D0002070BDD07AD4
:10B33000FCE70000FC1F0000027C80231A40802AEA
:10B3400000D00174704710B50246FF23D089C007B2
:10B35000C00F00280AD00120D08100E05B1ED089F8
:10B36000C007C00F002801D0002BF7D1D089C0073B
:10B37000C00F002801D0002010BD507A01242043C6
:10B380005072507A3824A0435072C87A1072487AAA
:10B3900000280FD1087B1070487B5070887B90701C
:10B3A000CC7BD470087C10714C7C5471887C90717B
:10B3B000CC7CD471FF200130D0814000D081107A44
:10B3C000DAE70000F8B504460D460020002C00D155
:10B3D00000BF002A00D100BF012C01D1412630431B
:10B3E000012A01D112263043022C01D1C02630435C
:10B3F000022A01D130263043134E307076788027F0
:10B40000BE43114F7E70012C08D1FF2100BF0E4EAC
:10B41000B3781E460E4033468B42F8D10A4E7678FA
:10B420004027BE43084F7E70012A0BD100260096AC
:10B4300003E000BF009E761C0096FF276937009E40
:10B44000BE42F6D9F8BD000000040240002905D034
:10B45000054A12780243044B1A7004E0024A12783B
:10B460008243014B1A70704720040240002905D026
:10B47000054A927E0243044B9A7604E0024A927E89
:10B480008243014B9A76704700080240012006492A
:10B49000087000BF04480078802108400028F9D0D7
:10B4A0000120024908707047000C02409C010020F6
:10B4B00070B5034614460020002B01D1C0B202E053
:10B4C00005468035E8B2012902D1051DE8B206E043
:10B4D000022903D105460835E8B200E0C0B2012CCC
:10B4E00002D1851CE8B200E0C0B2084DA870AD786A
:10B4F00001263543054EB570002201E000BF521C05
:10B500007D252D01AA42F9D970BD0000000C024032
:10B5100070B500242448007920210840002801D07B
:10B52000224D3FE000F046F8054621480078802192
:10B530000840002836D01E4880780840002801D0F6
:10B540001A4D02E000F036F80546194880780007E9
:10B55000840F022C01DBAD0804E0012C01D16D0841
:10B5600000E000BF124880788007C00F002801D09B
:10B570002D0101E00C2045430D4800784007840F61
:10B58000002C02D1601CC4B207E0032C03D1601C64
:10B590004006040E01E06006040E21462846FCF732
:10B5A000CFFD0546284670BD0004024000127A0017
:10B5B000000C024000B5C0229178F82211401C4ACC
:10B5C00012781143EA2923D00ADC0A46E03A130034
:10B5D00014F092FD0A181C20242A2A2A2A161A2A54
:10B5E000ED291FD004DCEB2916D0EC291CD117E083
:10B5F000F02903D0F82917D10E4817E00E4815E0BE
:10B600000E4813E00E4811E00E480FE00E480DE022
:10B610000E480BE00E4809E00E4807E00E4805E032
:10B620000E4803E00E4801E00D4800BF00BF00BD1A
:10B63000201C02400090D003006CDC020048E801AE
:10B6400000366E010024F400001BB70000127A00DF
:10B65000808D5B0000093D00C0C62D0080841E0067
:10B6600040420F0010B50446204600F097FD002030
:10B6700010BD000010B5A8211348FCF711FE1248B8
:10B68000124908601248486007200881002088722B
:10B6900007220F490D4800F065FA00210B48FFF71B
:10B6A00005FEA0210B48FCF7FBFD0A480A4948604B
:10B6B0000A4B05220A49084800F0E0FB55210648DC
:10B6C000FFF73AFE10BD00006C0800204C08002077
:10B6D000F80E0200140900205808002065B600008A
:10B6E0006C0E02000C4A127812060B4B5B781B049E
:10B6F0001A43094B9B781B021A43074BDB781A430A
:10B70000104642084240D20083085A401146034A7C
:10B710005140034A116070471307002001020000E6
:10B7200018070020F8B504460F46A07A4006400EE0
:10B73000002874D10025ACE018206843216808185F
:10B74000407C01283CD10121182068432268101850
:10B75000017400260CE0182068432168081808309E
:10B76000815D18206843226810188155701CC6B28C
:10B77000082EF0D3002118206843226810180174A5
:10B780001820684322681018417418206843226802
:10B7900010184161182068432268101881742C2009
:10B7A000684361680818406A002809D018236B4371
:10B7B0002268D0182C236B436268D218516A8847DC
:10B7C00018206843216808184069FF21C94388424E
:10B7D0005DD818206843216808184069C1191820ED
:10B7E00068432268101841611820684321680818CE
:10B7F00041692C206843626810188069814246D3F1
:10B800001820684321680818807C55283FD05521AE
:10B8100018206843226810188174002624E03CE058
:10B820001820684321680818805D2C2169436268EC
:10B8300051181031895D0840182169432268511858
:10B8400088551820684321680818805D2C216943B9
:10B85000626851180831895D0843182169432268DC
:10B8600051188855701CC6B2082ED9D32C206843B5
:10B8700061680818806A002809D018236B43226881
:10B88000D0182C236B436268D218916A8847681CD1
:10B8900085B22089A84200DD4EE7F8BD10B5044608
:10B8A000002014F08DFF022841D1214800780028A3
:10B8B00002D101201E4908701D48007801281FD1BF
:10B8C0001B484078401C1A49487021465A20FCF712
:10B8D00037FC17494978884229D800201449487014
:10B8E00008468078401C8870084680780A2803D370
:10B8F0000020887002200870002014F091FF16E0EC
:10B900000B480078022812D109484078401C0849A9
:10B91000487021467D20C000FCF712FC044949789C
:10B92000884204D800200249487014F079FF10BD05
:10B930007600002000B587B000216846017104211F
:10B9400041710C480290411003910B4904910591FB
:10B950000A480690FFF78EFE01A814F0C5FF00F01C
:10B9600043FB00F00FF80021054809F09BFD07B0EC
:10B9700000BD0000FFFF1F00FFFFFF1FEDBB000029
:10B980000205000010B5FF20023072494860002017
:10B9900008720120087000204872012088726E48E9
:10B9A000FFF7D7FB6B496C48FFF7FCFB01216A48A6
:10B9B000FFF74CFC69486749486000200872012085
:10B9C0000870002048720120887263481030FFF729
:10B9D000C0FB604960481030FFF7E4FB01215E487E
:10B9E0001030FFF733FC5D48401E5A494860002084
:10B9F00008720120087000204872012088725648A1
:10BA00005030FFF7A6FB534953485030FFF7CAFBAD
:10BA1000012151485030FFF719FC5048C1384D49B9
:10BA20004860002008720120087000204872012040
:10BA3000887249484030FFF78CFB46494648403001
:10BA4000FFF7B0FB012144484030FFF7FFFBFF2028
:10BA50001230404948600020087201200870002020
:10BA60004872012088723C486030FFF772FB394908
:10BA700039486030FFF796FB012137486030FFF707
:10BA8000E5FBFF2021303349486000200872012087
:10BA9000087000204872012088722F48A030FFF7FC
:10BAA00058FB2C492C48A030FFF77CFB01212A4889
:10BAB000A030FFF7CBFB29488F382649486000208B
:10BAC0000872012008700020487201208872224804
:10BAD000E030FFF73EFB1F491F48E030FFF762FBF5
:10BAE00001211D48E030FFF7B1FB3F20400119491B
:10BAF0004860002008720120087000204872012070
:10BB0000887215482030FFF724FB12491248203074
:10BB1000FFF748FB012110482030FFF797FB104842
:10BB20000C4948600020087201200870002048720B
:10BB30000120887208483030FFF70BFB05490648A2
:10BB40003030FFF72FFB012103483030FFF77EFB39
:10BB500010BD0000542A00201055044002040000CB
:10BB6000DF070000F0B50B46144643600481002156
:10BB700036E0002216E02C254D4346687519AD5C71
:10BB800018274F430668F619B5542C254D434668CF
:10BB90007519AD5C18274F430668F6190836B55479
:10BBA000551CEAB2082AE6D3002518274F43066839
:10BBB000F619357418274F430668F6197574182757
:10BBC0004F430668F619B57418274F430668F619EF
:10BBD000F57418274F430668F61975614D1CA9B214
:10BBE00005898D42C5DC00258572F0BD70B504461F
:10BBF000606800F055FE0546E27A23460C3329467C
:10BC0000094800F015FE09496068884203D0491CC4
:10BC10006068884206D1E17AA28890B222460C324E
:10BC200003F022F870BD00004C080020DF07000080
:10BC3000F8B5054600262C46002C11D000BF03E0C5
:10BC40000020A055701CC6B2082EF9D304F03CFFAA
:10BC5000C000082108400746206888433843206018
:10BC6000F8BD0000F8B5054600262C46002C49D04A
:10BC700000BF03E00020A055701CC6B2082EF9D307
:10BC80002148007B002809D12088000A000220807A
:10BC90002088FF2109028843208012E005F022F865
:10BCA00007122088000A00023843208005F01AF8A5
:10BCB0000002FF21090208400746208888433843D4
:10BCC00020801148407B002809D16088000A0002CA
:10BCD00060806088FF2109028843608012E005F0DF
:10BCE000F1F807126088000A00023843608005F00E
:10BCF000E9F80002FF2109020840074660888843EE
:10BD000038436080F8BD00003428002070B5054637
:10BD100000262C46002C2CD000BF03E00020A055AC
:10BD2000701CC6B2082EF9D305F0E8F801280AD134
:10BD300031202070012060705920A0700820E07030
:10BD40000020207115E005F0D9F802280AD1312031
:10BD50002070012060705920A0700820E070012040
:10BD6000207106E0002020706070A070E07002205A
:10BD7000207170BDFEB5054600260020019001F03F
:10BD80002FFD0A210090FCF7DBF9074604F0CCFEFA
:10BD90000A210090FCF7EAF980B201902C46002CB1
:10BDA0003AD000BF03E00020A055701CC6B2082E98
:10BDB000F9D3FF21090260688843390C0902FF2288
:10BDC0001202114008436060110260688843390A1A
:10BDD0000904120211400843606060680002000A12
:10BDE0003906090E09060843606004F091FFFF2838
:10BDF00006DDFF21090420688843401820600BE01D
:10BE000004F086FF0004FF21090408400090206828
:10BE10008843009908432060FEBDFEB50546002614
:10BE200000200190002704F057FC64210090FCF7EB
:10BE30009DF980B20190002001F0F4FC87B22C46FD
:10BE4000002C1AD000BF03E00020A055701CC6B221
:10BE5000082EF9D3FF210904206888433912090408
:10BE6000FF22120411400843206020680002000AEB
:10BE70003906090E090608432060FEBDFFB581B0F2
:10BE800004460F46002500260020009027600398F6
:10BE900020810498E0600020207400BF9DE01C20F9
:10BEA0006843216808586A01616888501C2068430B
:10BEB0002168081880686A016168891848601C2038
:10BEC00068432168081840686A01616889188860B9
:10BED0001C20684321680818C0686A0161688918D5
:10BEE000C8601C20684321680818007C6A016168EA
:10BEF000891808741C20684321680818407C6A016E
:10BF00006168891848741C20684321680818807C7F
:10BF10006A016168891888831C20684321680818B1
:10BF2000C07C6A0161688918887400206A016168B0
:10BF30008918C8741C2068432168081840680028C4
:10BF400013D01C20684321680818C07C002805D144
:10BF5000401E6A0161688918C8831AE00020C04346
:10BF60006A0161688918C88313E01C20684321684E
:10BF70000818C07C002805D000206A016168891873
:10BF8000C88306E000206A0161688918C88301201F
:10BF90000090002607E000216A01606880181430D4
:10BFA0008155701CC6B2690160684018808BB04230
:10BFB000F1DC1C20684321680818406900280AD079
:10BFC0006B016268D218104614301C236B43226840
:10BFD000D21851698847681CC5B22089A84200DD83
:10BFE0005DE7009805B0F0BD00B58BB068480790DC
:10BFF000002108A801706846017608A84170002059
:10C0000064498872082108A8C170002004E0002259
:10C0100009A90A54411CC8B208A9C9788142F6DCB2
:10C020005D48FFF796F806A95B48FFF7BBF858484C
:10C03000401C0790002108A801706846017608A8F6
:10C040004170002053498872082108A8C17000205F
:10C0500004E0002209A90A54411CC8B208A9C97801
:10C060008142F6DC4C484030FFF773F806A94A4895
:10C070004030FFF797F8452000010790002108A8FD
:10C0800001706846017608A8417000204149887215
:10C09000082108A8C170002004E0002209A90A5460
:10C0A000411CC8B208A9C9788142F6DC3A48503030
:10C0B000FFF74FF806A938485030FFF773F8112002
:10C0C00040010790002108A801706846017608A881
:10C0D000417000202F498872082108A8C1700020F3
:10C0E00004E0002209A90A54411CC8B208A9C97871
:10C0F0008142F6DC28482030FFF72BF806A92648B5
:10C100002030FFF74FF80B20C0010790002108A84E
:10C1100001706846017608A8417000201D498872A8
:10C12000082108A8C170002004E0002209A90A54CF
:10C13000411CC8B208A9C9788142F6DC16486030B3
:10C14000FFF707F806A914486030FFF72BF8FD2029
:10C15000C000029000216846017301714173817330
:10C160000821C173002004E0002204A90A54411CE4
:10C17000C8B26946C97B8142F6DC07481030FEF739
:10C18000E8FF01A904481030FFF70CF80BB000BD20
:10C19000EE060000542A00208055044030B585B0DA
:10C1A0000446002520680190A1796846C172617932
:10C1B000417200210172017000BF05E02046083085
:10C1C000415D03A841556D1C6846C07AA842F5D868
:10C1D0000B22D2010199881A914226D007DC184817
:10C1E000081A1CD023210901401A24D111E0FF387C
:10C1F0006F38002802D001281DD104E0694611489B
:10C20000FFF7A1F818E069460E484030FFF79BF8A9
:10C2100012E069460B485030FFF795F80CE069468C
:10C2200008482030FFF78FF806E06946054860307F
:10C23000FFF789F800E000BF00BF05B030BD000087
:10C240002002000080550440F0B585B004460F463A
:10C2500000250026207C4006400E55287ED100BFD8
:10C2600076E1690160684018807C002877D1690117
:10C270006068401840686A01616889188968884266
:10C2800009D26901606840184068C0196A01616894
:10C29000891848605AE1690160684018C068AF4970
:10C2A000884208D8690160684018C068401C6A016B
:10C2B00061688918C860690160684018C07C0028FE
:10C2C00021D1002607E000216A016068801814303F
:10C2D0008155701CC6B2690160684018808BB042FD
:10C2E000F1DC1C20684321680818406900280AD046
:10C2F0006B016268D218104614301C236B4322680D
:10C30000D2185169884769016068405800906901F6
:10C3100060684018017C6846017100214171690123
:10C3200060684018017F6846817169016068401843
:10C33000417C6846C171002608E0690160684018C8
:10C340001430815D02A88155701CC6B26901606815
:10C350004018808BB042F0DCE06801E0FCE01DE0BA
:10C36000002806D06846E16888476A016168891834
:10C37000C874690160684018C07C002804D16A0153
:10C38000616889184860E1E06901606840184068A8
:10C39000C01B6A01616889184860D7E0690160685C
:10C3A000401880680028EED0690160684018C08B92
:10C3B0000028E8D0690160684018C08B6A01616894
:10C3C0008918C968884207D1690160684018C08B24
:10C3D0006249C94388427DD169016068401840685C
:10C3E0006A01616889188968884209D269016068B0
:10C3F00040184068C0196A01616889184860A5E062
:10C4000000206A0161688918486069016068401805
:10C41000C0685249884208D8690160684018C068FD
:10C42000401C6A0161688918C860002607E0002185
:10C430006A016068801814308155701CC6B26901A9
:10C4400060684018808BB042F1DC1C206843216892
:10C450000818406900280AD06B016268D21810469B
:10C4600014301C236B432268D21851698847690134
:10C47000606840580090690160684018017C684617
:10C48000017100214171690160684018017F6846AF
:10C490008171690160684018417C6846C17100265D
:10C4A00008E06901606840181430815D02A8815578
:10C4B000701CC6B2690160684018808BB042F0DC25
:10C4C000E068002808D06846E16888476A0161682A
:10C4D000891800E015E0C874690160684018C07CE4
:10C4E000002804D16A016168891848602EE069015A
:10C4F000606840184068C01B6A016168891848601C
:10C5000024E01C20684321680818406800280FD0E8
:10C510000020C0436A0161688918C8831C206843F1
:10C520002168081840686A0161688918886008E015
:10C5300000206A0161688918C8836A0161688918E6
:10C54000886000206A0161688918C860681CC5B2EB
:10C550002089A84200DD84E605B0F0BD0000FFFFA1
:10C560007CB500BF19212C480078FBF7E9FD044693
:10C570002A4860432A4A8118002201200CF0E2FF79
:10C5800020460A2250436430001981B20022012063
:10C590000FF030F801200A2262431219D1B20A22A8
:10C5A000624312190090D0B201231A4609F08EFAA4
:10C5B000FF220721002006F049FF01200090019092
:10C5C0000B20604382B20B20604381B20023012024
:10C5D0000EF036FD6F20604381B201200FF0B0FAFB
:10C5E000104860430246032101200BF029FD00257D
:10C5F00005E0012128460BF05DFC681CC5B20F2D3B
:10C60000F7DB21460B2251436431C8B20FF0FCFC2A
:10C610000FF0E4FC7CBD000073000020672B0000DD
:10C62000A0860100FCB10100002005490870054901
:10C630000870054908700549087005490870704779
:10C64000740000207500002073000020720000209C
:10C6500071000020F0B589B000BF00BF00BF00BF6F
:10C6600000BF00BF00BF00BF00BF00BF5D48007833
:10C670003C2805DA5B480078401C5A49087002E003
:10C680003C2058490870574800781D2805DC56485A
:10C690000078401C544908700BE05348007800288B
:10C6A00002D15149087004E04F480078401E4E49BD
:10C6B000087003214C480078FBF758FD4B4948436C
:10C6C0000390052148480078FBF73AFD0446032112
:10C6D00045480078FBF74AFD0B214843643080B29F
:10C6E0000690414909788A0088180621FBF73EFD2B
:10C6F000FF21F531484380B2079003213A48007882
:10C70000FBF734FD0B214843643080B208900321CD
:10C7100035480078FBF72AFD35494843354940182C
:10C720000490032130480078FBF720FD0B210646DA
:10C730004E4303212C480078FBF718FD0B210746D8
:10C740004F43032128480078FBF710FD6F21484331
:10C7500080B2059003210120039A0BF071FCE1B235
:10C7600001200BF035FAE1B201231846069A09F0D0
:10C7700087FCFF21F5310798FBF7F8FCC0B20146B2
:10C78000029001200AF060F90022012008990EF0C1
:10C7900031FF0022012004990CF0D4FE01200599FC
:10C7A0000FF0CEF90120F9B20090F0B201231A4641
:10C7B000029009F08BF9FF220721002006F046FEC7
:10C7C000032109480078FBF7D1FC0B21484385B2CF
:10C7D0000120009000232A46294601900EF030FCEB
:10C7E00009B0F0BD7500002074000020FCB101000C
:10C7F000672B0000A0860100002000BF06E000219A
:10C80000044A1154044A1154411CC8B25A28F6DB98
:10C810007047000044260020F82600200348007AD4
:10C82000002801D10149487070470000540A0020D7
:10C83000FFB581B004460F463D462089A8422DDD54
:10C840001820684321680818007C002826D100269B
:10C8500009E00498815D18206843226810180830A8
:10C860008155701CC6B2082EF3D3012118206843ED
:10C870002268101841742C20684361680818006A07
:10C8800000280BD018236B432268D21810460830BA
:10C890002C236B436268D218116A884705B0F0BD3B
:10C8A00001460720124BCA1A994211D008DCCA1F50
:10C8B000FA3A002A14D0102A0CD01F2A14D10DE005
:10C8C000322A0FD0C02A07D0C12A0DD100200DE096
:10C8D00001200BE0022009E0032007E0042005E02E
:10C8E000052003E0062001E0072000BF00BF7047DD
:10C8F0004103000010B504467D21C900614308468C
:10C90000322103F08BFE10BDFF200B490870002080
:10C91000C0430A4908800A490880FF200949087075
:10C920000949087009490870002009490860094947
:10C930000860094908607047580000205A0000202C
:10C940005C0000205E0000205F00002060000020EE
:10C950004C000020500000205400002001480068D6
:10C960007047000050000020014800687047000038
:10C970004C00002010B5054909886522514308463E
:10C980006421FBF7F3FB80B210BD00005A000020C9
:10C9900001480078704700005F00002001480078DF
:10C9A000704700005800002010B510F063F801280F
:10C9B0002CD100F063F8012000F066F803F092FE3D
:10C9C000044600F043F804F08DF8044600F04AF8FD
:10C9D00004F0B6FA012805D100F03EF8012000F07D
:10C9E00047F805E0002000F037F8002000F040F89C
:10C9F00000201349086013480068134988421ED27A
:10CA000010480068801C0F49086018E000200D499C
:10CA100008600B4800680C49884204D20848006846
:10CA2000801C07490860002000F028F8012000F071
:10CA30002BF8002000F00AF8002000F013F810BDD9
:10CA4000500000204C000020FFFFFF7F01490880BC
:10CA5000704700005A00002001490870704700002C
:10CA60005F00002001490880704700005C00002042
:10CA700001490870704700006000002001490870FB
:10CA800070470000580000200149087070470000FE
:10CA90005E0000200021014A1171704700600040D3
:10CAA000002201494A757047006000400022014998
:10CAB0004A767047006000400021014A11727047B9
:10CAC000006000400021014A11737047006000407F
:10CAD0000021014A11747047006000400021014AA2
:10CAE00011757047006000400021014A11767047BF
:10CAF00000600040002201494A7370470060004016
:10CB0000002201494A7470470060004010B51C4C77
:10CB10001C49206888421ED106221B49201DFBF7B4
:10CB2000CAFB002817D11122184920460A30FBF70A
:10CB3000C2FB00280FD10622154920461B30FBF707
:10CB4000BAFB002807D10622124920462130FBF704
:10CB5000B2FB00280DD000F089FE0A480E4908609B
:10CB6000074813F08EFF0C4A2821054813F0B4FF44
:10CB700004E0282221460848FBF779FB10BD00009D
:10CB8000000250007AA7A55A290700202F0700208D
:10CB9000230700201D070020602E002000200849E8
:10CBA00008700849087001200749087000200749EB
:10CBB0000870074807490860002007490870704757
:10CBC0000B0700200A0700200D0700201207002095
:10CBD00025060000400700201C07002070B5044611
:10CBE00000BF9120604305460A212846FBF7A8FABA
:10CBF0000546284670BD000070B5A8B00546002463
:10CC00000026A0216846FBF74BFB00F09FFC1E4965
:10CC10000A6814216943505000211B4802681420FF
:10CC200068431018416018480268142068431018BF
:10CC3000816015484068002824D000BF17E06006D6
:10CC4000060E282E00D316E00F480168142060431A
:10CC50000858B1006A4650500B48016814206043E0
:10CC600008184168701C80001150601CC4B206484E
:10CC7000007AA042E3DC00BF6200034869464368D3
:10CC80000220984728B070BDD82E002030B5A9B03A
:10CC900000240025A02101A8FBF702FB00BF25E02E
:10CCA0006006050E00F052FC1F490A68142161431A
:10CCB000505000211C480268142060431018416045
:10CCC000194802681420604310188160282D0BD287
:10CCD00015480168142060430858A90001AA505063
:10CCE0000021681C80001150601CC4B20E48007AFC
:10CCF000A042D5DC0C484068002813D00A48007ACE
:10CD00004000282806D30848282201A943680220A9
:10CD1000984707E00448007A4200034801A94368A5
:10CD20000220984729B030BDD82E002010B50FF052
:10CD3000A1FE01287ED1FFF717FE5549884216D281
:10CD40000F2054494871887108468078002801D125
:10CD5000052048704F488078052802D100204D49B1
:10CD6000487000204B4908724872087035E0FA207C
:10CD70004849487188714849088803F0DBFD4648F6
:10CD8000807800280CD14349087008464079C87063
:10CD900008468079087100208870487048721CE04D
:10CDA00001203C4908700846407A022805D101203C
:10CDB00048720020C87008710FE03648407A002899
:10CDC0000BD10220334948720846407888700846E3
:10CDD0004079C8700846807908712E4880782D49BE
:10CDE0004978884213DD00202A49C8700846007936
:10CDF000401C0871084600798979884222DB0020AE
:10CE00002449087108468078401E88701AE021483D
:10CE1000807820494978884214DA00201D49087139
:10CE20000846C078401CC8700846C07849798842D6
:10CE300008DB00E01EE000201649C8700846807834
:10CE4000401C887014488078002803D101201149C3
:10CE500008721BE010480088732803DB02200D498C
:10CE6000087213E00C48008870280FDC0020094984
:10CE700008720BE000200749087008464079C87026
:10CE800008468079087100200872487210BD0000C1
:10CE9000B80B0000B40900207C00002000200449E9
:10CEA00088704870C8700871087248727047000036
:10CEB000B409002000200649088088700549887060
:10CEC0004870FA20C87008710020087248727047D4
:10CED0007C000020B409002070B503F033FC044648
:10CEE00003F042FC05460FF0C5FD01282ED10521B7
:10CEF0001A48FEF721F9552804D1002018498870F6
:10CF0000088027E0012D04D1002015498870088091
:10CF100020E00120124988701248844202DB201A66
:10CF200084B200E000240A212046FBF71FF90529FE
:10CF300001DB601D84B20C48844200DD04460A21F6
:10CF40002046FBF713F90649088003E00020044956
:10CF500088700880FFF7EAFE70BD00004C080020D2
:10CF60007C000020AA0A0000C60700001CB50020B3
:10CF70000090019000F0EAFA0B49086000200B498C
:10CF8000096808600A48006800280CD00749096849
:10CF900008680A21FBF7D4F80090012269460520B1
:10CFA000034B1B6898471CBDDC070020D0070020FE
:10CFB000D80700200020084948800849088008490F
:10CFC0000880084908700849887208490880488024
:10CFD0000120087170470000300000202000002070
:10CFE000220000202400002030080020280000201B
:10CFF000F8B503F089FB074603F098FB0090FFF7B4
:10D00000CDFC012860D10521C548FEF795F85528CB
:10D0100002D00098012807D10020C2490870C249F7
:10D020000880C249887256E0BE480078002810D1B6
:10D030000120BC4908703D462846E917890F0918A8
:10D0400089030D0CBA48854200DD0546B6480580C7
:10D0500041E0B648807A4000B4490F520846867ACB
:10D060000EE07000B1490D5A701E4000085A710060
:10D07000AE4A5052701E400011460D52701EC6B28C
:10D08000002E08DD7000A949095A701E4000A74A09
:10D09000105A8142E5DBA548807A401CA34988727A
:10D0A0000846807A052816DB002088720846C58865
:10D0B0002846E917890F09188D109D48854200DD23
:10D0C00005469948058006E0002096490870964973
:10D0D0000880964988729448058896480088A84236
:10D0E00057DA94480088281A84B2924800790128B7
:10D0F00027D190484088A0420BDA8E4840880A30F9
:10D100008C49488008464088A04204DD0846448097
:10D1100001E0884844808748448803212046FBF783
:10D1200025F884B2192C00DA1924824800880019E5
:10D130008049088008460088A84201DD084605802D
:10D14000CDE07C484088142805DD7A4840881438B2
:10D150007849488002E00020764948807548448834
:10D1600003212046FBF702F884B2192C03DA0120D0
:10D1700070490871B3E06F480088A04205DD6D4832
:10D180000088001B6B490880A9E0002069490880DD
:10D19000A5E068480088A84259DD66480088401B21
:10D1A00084B264480079012827D162484088142855
:10D1B00005DD6048408814385E49488002E0002060
:10D1C0005C4948805B48448803212046FAF7CEFF3B
:10D1D00084B2192C03DA0220564908717FE05548C1
:10D1E0000088001953490880084600885049884241
:10D1F00075DD08464F49088071E04E484088A042DE
:10D200000BDA4C4840880A304A4948800846408832
:10D21000A04204DD0846448001E046484480454879
:10D22000448803212046FAF7A1FF84B2192C00DAC2
:10D230001924404800882919884202DA3D480580AF
:10D240004DE03C480088001B3A49088047E03948D7
:10D25000448803212046FAF789FF84B2192C3EDD69
:10D2600034484088142805DD324840881438314954
:10D27000488002E000202F4948802E48448803213E
:10D280002046FAF773FF84B22A480079012813D1A7
:10D29000192C03DA02202749087120E0254800886C
:10D2A000001924490880084600882149884216DD73
:10D2B00008462049088012E0192C03DA01201D4994
:10D2C00008710CE01B480088A04205DD1948008861
:10D2D000001B1849088002E0002016490880164803
:10D2E0000088502804DC134800881349088016E0A1
:10D2F0001048008810490988884204DD0D480088DC
:10D300000D4908800BE00B4800880B490988081A72
:10D3100084B2502C03DB0748008807490880F8BD19
:10D320004C080020240000202000002030080020AD
:10D33000E02E0000280000202200002010B5044646
:10D3400064204443A1212046FAF7FAFE0446204611
:10D3500010BD00007CB5002400200190009000F07A
:10D360003FFA05460A21FAF7EBFE04460122694618
:10D37000042000F067FE0098401C002814D17D2096
:10D38000C000201811490860084600680190012279
:10D3900001A9032000F0A2FE0120009001226946AD
:10D3A000042000F09BFE0FE0009801280CD17D20A6
:10D3B0000001201805490860084600680190012214
:10D3C00001A9032000F08AFE7CBD0000240100209A
:10D3D00010B501200F49087000200F490968086046
:10D3E0000D49096848600C490968886000F07EF9B9
:10D3F000FFF7BCFDFFF74AFC08480068002807D08B
:10D4000001220548016808310020044B1B68984739
:10D4100010BD0000A9070020A4070020A0070020DD
:10D4200010B5184800681849884229D11748006883
:10D43000002804D015480068804715490870154831
:10D440000068002804D0134800688047124908701B
:10D4500012480068002804D010480068804710492E
:10D46000088010480068002805D00E4800688047F2
:10D470000D49088002E00D480B49088000F078F85B
:10D4800010BD0000B4070020785634129007002029
:10D49000A807002094070020AA0700209807002072
:10D4A000AC0700209C070020AE07002010270000DA
:10D4B00010B50023174C2360174C2370174C2370B2
:10D4C000174C2370174C2380174C2380174C237064
:10D4D000174C13682360174C53682360164C9368ED
:10D4E0002360164CD3682360154C13692360002811
:10D4F0000CD0144B1860134C0B682468A3600023F5
:10D50000104C246823600F4C246863600E4B014C60
:10D51000236010BDB4070020B0070020A80700203A
:10D52000AA070020AC070020AE070020A9070020B2
:10D530009007002094070020980700209C070020F7
:10D54000A0070020A4070020785634120548006880
:10D550000549884203D1054800688068704700206B
:10D56000C043FBE7B407002078563412A40700201C
:10D5700070B50024002500263048007801285CD1D1
:10D580002F480078002858D12E480078012854D11F
:10D590002D4805882D490988694308462C49FAF722
:10D5A000CFFD85B2E1200001854207D819216943EA
:10D5B00008460921FAF7C4FD044600E0244C25483A
:10D5C000006800680019234909680860214800685C
:10D5D0000068204909684968884207D31D480068E7
:10D5E00000681C4909684968461A0AE01948006839
:10D5F00040680021C943081A16490968096840189B
:10D60000461C1548864218D3344601462046FAF790
:10D6100097FD04460F48006841680F4860430818AA
:10D620000C490968486001200C49087009480068E5
:10D630008068001907490968886070BDA807002044
:10D64000A9070020AA070020AC070020AE07002091
:10D6500010270000A4070020A0860100B0070020CA
:10D6600000220C4B1A600C4B0A681A600B4B4A687C
:10D670001A600B4B8A681A600A4BCA681A600A4B18
:10D680000A691A60002801D0084A1060084A014B54
:10D690001A607047B407002090070020940700200C
:10D6A000980700209C070020A0070020A407002066
:10D6B0007856341210B50A48006800280ED0094880
:10D6C000007801280AD10020064908700122064886
:10D6D000016808310020024B1B68984710BD00000C
:10D6E000A0070020B0070020A40700201CB50020E0
:10D6F000009001900024FFF729FF04460E480068BF
:10D70000046000200C49096848600B49096888607A
:10D710000A48006800280DD007480068006800909B
:10D720000548006840680190022269460120034BC9
:10D730001B6898471CBD0000B8070020BC070020EC
:10D74000F8B505460C4616460027002D17D00E48A2
:10D750000560FFF7FBFE07462068B84203D90A4878
:10D760000068076003E00849206809680860064906
:10D770006068096848600449A0680968C86003488F
:10D78000066000F005F8F8BDB8070020BC070020CF
:10D7900070B500240025FFF7D9FE04460F48006845
:10D7A0000068A04200D903E00C4800680068251A10
:10D7B0000A480068406840190849096888600748B5
:10D7C0000068806805490968C968884205D9034826
:10D7D0000068C06801490968886070BDB80700200A
:10D7E0000148006880687047B8070020002801D011
:10D7F000024A1060024A116070470000B80700201A
:10D80000BC0700200549002005E00A1D135C044AFE
:10D810001354421CD0B22028F7DB7047000650009A
:10D820008C2E00200146104802681420484310182E
:10D8300082680D480368142048431818C068824263
:10D840000BD909480268142048431018C2680648DA
:10D8500003681420484318188260034802681420A3
:10D860004843101880687047D82E002000210020FF
:10D8700005E01A4A135C1A4A1354421CD0B2062817
:10D88000F7DB1121002006E0164A135C144A921DB2
:10D890001354421CD0B28842F6DB002006E0124A44
:10D8A000135C0F4A17321354421CD0B20628F6DB21
:10D8B000002006E00D4A135C094A1D321354421C35
:10D8C000D0B20628F6DB002005E00023044A23320C
:10D8D0001354421CD0B20128F7DB704729070020FF
:10D8E000642E00202F070020230700201D070020A2
:10D8F00038B50446002000900094012269460520B6
:10D9000000F0ECFB38BD000008B5002000900122BB
:10D910006946062000F096FB684600780C490873BB
:10D920006846407848730846007B0A4948730848AF
:10D93000407B88730648807BC8730548C07B0874A9
:10D94000002008730448054908600549086008BDBF
:10D9500034280020C009002071170000800000203A
:10D960008400002008B500200090012269460620AE
:10D9700000F068FB684600780F49087368464078F5
:10D98000487300200D490860486008724872887228
:10D990000948007B48730848407B88730648807BB1
:10D9A000C8730548C07B0874002008730448054903
:10D9B00008600549086008BD34280020C00900201F
:10D9C00071170000800000208400002038B500247A
:10D9D0000025002000900121FC48FDF7ADFB5528F3
:10D9E0000AD002F005FFFA49487302F015FFF84922
:10D9F00088730120087308E0F648007BF4494873F7
:10DA0000F448407B887300200873F148407B00286D
:10DA100004D1EF494873F049086053E0EC48407B7B
:10DA2000012829D1EC480068EC49884208D8EA4826
:10DA30000068401CE84908600120E549487341E05E
:10DA4000E448007B022812D0E248007B03280ED075
:10DA50000121DE48FDF770FB552803D00320DC4987
:10DA600048732FE0DB48007BD94948732AE0D94846
:10DA7000007BD749487325E0D548407B02280FD169
:10DA80000020D549086002F0DDFE00281AD002F01F
:10DA9000D9FE401C002815D00220CD49487311E062
:10DAA000CB48407B032806D10020CB4908600320E7
:10DAB000C749487306E00020C7490860C548007B95
:10DAC000C3494873C248807B002804D1C449086018
:10DAD000BF4988735CE0BE48807B012832D1C048D2
:10DAE0000068BE49884208D8BD480068401CBC494F
:10DAF00008600120B64988734AE0B548807C002858
:10DB000001D1B74908600120B1498874B148407B10
:10DB1000022812D0AF48407B03280ED00121AB4829
:10DB2000FDF70AFB552803D00320A94988732FE08D
:10DB3000A848407BA64988732AE0A648407BA449B0
:10DB4000887325E0A248807B02280FD10020A449D9
:10DB5000086002F095FE00281AD002F091FE401CE9
:10DB6000002815D002209A49887311E09848807BDC
:10DB7000032806D100209A4908600320944988733D
:10DB800006E00020964908609248007B904988731F
:10DB90008F48407B8F49097B884205D18C48807B28
:10DBA0008C49497B884246D08948407B8949097B1A
:10DBB000884202D001208649C8738548807B854908
:10DBC000497B884202D00120814908748048407B0B
:10DBD000022803D07E48407B032803D17C48407B49
:10DBE0007C4908737A48807B022803D07848807B80
:10DBF000032803D17648807B764948737448407B7C
:10DC000002280BD07248407B032807D07048807BE5
:10DC1000022803D06E48807B03280CD16D48017B1D
:10DC2000684601706B48417B684641700122694635
:10DC3000062000F053FA02F0E5FD044602F0F8FD7C
:10DC40000546FEF7ABFE012872D101215F48FDF7C2
:10DC500073FA552807D100205D49087248720860A0
:10DC600048608872CBE0FF2C01D0FF2D6AD1FF2CD9
:10DC70002ED1FF2D2CD0002055490872012048726A
:10DC80005848086058486843486048686621FAF771
:10DC900057FA4F494860084640685449884202D9BB
:10DCA00008464B4948604A484068323050498842EB
:10DCB00006D34748406832304B49FA39884203D985
:10DCC0000120434988729AE000204149887296E019
:10DCD000FF2C2ED0FF2D2CD101203D4908720020B1
:10DCE00048724048486040486043086008686621C0
:10DCF000FAF726FA36490860084600683B49884228
:10DD000002D9084632490860314800683230384943
:10DD1000884205D32E48006832303649884203D9FC
:10DD200001202B4988726AE000202949887266E048
:10DD3000A0E02E48264908604860002088720872DA
:10DD400048725CE00120224908724872264860430C
:10DD5000086008686621FAF7F3F91D49086008466B
:10DD600000682249884202D90846194908601E48BD
:10DD700068431749486048686621FAF7E1F9144991
:10DD80004860084640681949884202D90846104947
:10DD900048600F48006832301549884212D30C4859
:10DDA00000683230134988420CD809484068323044
:10DDB0000F49884206D30648406832300D49C831C1
:10DDC000884219D901200249887218E04C080020C5
:10DDD000C0090020342800208000002070170000B7
:10DDE00084000020DE030000BE0A0000AC26000014
:10DDF000A4060000FC080000002022498872214887
:10DE0000407B002802D11F49C87315E01D48407BA4
:10DE1000012802D11B49C8730EE01A48407B022832
:10DE200002D11849C87307E01648407B032803D184
:10DE30001449C873144808601248807B002802D136
:10DE4000104908741DE00F48807B012802D10D495C
:10DE5000087416E00B48807B022802D10949087437
:10DE60000FE00848807B03280BD106490874064858
:10DE7000486006E000200349087248720860486064
:10DE8000887238BDC0090020AC260000FFB583B001
:10DE900006460D46174600240020029000BF1420BD
:10DEA000784380190190002E57D00198002854D053
:10DEB0002B4806602A49069848600846077200BF4A
:10DEC00045E0FFF743FB0290200129580298814268
:10DED00004D820012858401C002806D12049029867
:10DEE0000A6814216143505006E0200129581C485B
:10DEF0000268142060431150200140194068401C02
:10DF0000002807D100211648026814206043101829
:10DF1000416008E02001401941681148026814205E
:10DF20006043101841602001401981680C48026864
:10DF3000142060431018C16020014019017B08487B
:10DF400002681420604310180161601CC4B20448C8
:10DF5000007AA042B5DC00F005F807B0F0BD000083
:10DF6000D82E002070B5002400250026FFF7EEFA19
:10DF7000054600BF4EE02A48016814206043085857
:10DF8000A84239D8264801681420604308582E1A40
:10DF9000234801681420604308184068811920480C
:10DFA000026814206043101881601D480168142025
:10DFB0006043081881681A480268142060431018EA
:10DFC000C068814224D916480168142060430818AB
:10DFD0000069002803D02046FEF70EFE18E0104826
:10DFE0000168142060430818C1680D4802681420B5
:10DFF0006043101881600BE00948016814206043F9
:10E000000818406806490A6814216143511888605D
:10E01000601CC4B20248007AA042ACDC70BD0000B3
:10E02000D82E002010B500BF14244C43231800281C
:10E0300005D0002B03D0024C20606260217210BD1D
:10E04000D82E0020F8B505460E4614462B0012F0D7
:10E0500053F80705131A21282F363D001D48FAF7FB
:10E060007DFD1D4908701B48FAF732F90746642107
:10E07000FAF766F830602AE0A004020C3146162058
:10E08000FAF766FE23E0A004020C31464820FAF7B6
:10E090005FFE1CE0A004020C31468020FAF758FE17
:10E0A00015E0A004020C3146A020FAF751FE0EE064
:10E0B000A004020C3146B020FAF74AFE07E06004E3
:10E0C000020C3146C020FAF743FE00E000BF00BF5B
:10E0D0000020F8BD26280020E100002070B505468C
:10E0E0000E4614462B0012F007F807051D242B32AC
:10E0F000393F46003068002802D1FAF7CDFB10E026
:10E1000064223168514308461C49FAF7EBF80020B5
:10E110001B490870012264211848FAF787FE184944
:10E12000087029E0A004020C31461620FAF7CEFF51
:10E1300022E0A004020C31464820FAF7C7FF1BE09A
:10E14000A004020C31468020FAF7C0FF14E0A004BE
:10E15000020C3146A020FAF7B9FF0DE0A2B2314619
:10E16000B020FAF7B3FF07E06004020C3146C0208C
:10E17000FAF7ACFF00E000BF00BF70BD1828002018
:10E18000E000002000B5AFB050211BA8FAF788F8D6
:10E1900000201A90142115A8FAF782F80020129096
:10E1A000139014901190402101A8FAF779F80020FB
:10E1B00000905149086001221BA9FFF743FF1B98FB
:10E1C000401C002801D11A9001E01B981A904B487E
:10E1D00015904B4816904B481790002018904A48CD
:10E1E000199015AA1AA94948FFF762F902221CA939
:10E1F0000120FFF727FF1C98401C002801D1129036
:10E2000001E01C9812901C98401C002801D113902A
:10E2100001E01D9813903E48149012A93D48199AA8
:10E22000FFF78EFA08221EA90220FFF70BFF1E98A7
:10E23000401C002801D1019001E01E9801901F9818
:10E24000029035480390012069460874801E0590AD
:10E2500032490791012101A80177881E09902F49B1
:10E260000B91012109A80173881E0D902B490F9174
:10E2700001210DA80173042201A92948199BFFF768
:10E2800005FE01221BA90320FFF7DCFE25491B9890
:10E2900008601B98401C002806D1FF20F53008605C
:10E2A00001220320FFF71AFF01221BA90520FFF717
:10E2B000C9FE1B98401C002807D101201A4988601C
:10E2C000012208310520FFF709FF01221BA90620C2
:10E2D000FFF7B8FE1B98401C002808D100216846B3
:10E2E00001704170012269460620FFF7F7FE0F48D2
:10E2F000014908602FB000BDE40000209DC9000066
:10E3000091C9000075C90000DDE00000AC270020C5
:10E3100076841E00B82700200F2700009F8601008A
:10E32000C82700202401002034280020A33AA55A41
:10E3300000B585B014216846F9F7B2FF00200F49F7
:10E3400008600F4800900F4801900F48029000208D
:10E3500003900E48049069460D48FFF781F90D4877
:10E360000499FFF743FA04210B48049AFFF75AFE79
:10E370000A480249086005B000BD0000E400002022
:10E380009DC9000091C9000075C90000DDE00000D2
:10E39000AC270020B8270020C8270020A33AA55AA0
:10E3A00000200C4908800C4908800C490880012095
:10E3B0000B49087000200B4908730B4908804880FE
:10E3C000012008710020074948800880074908603B
:10E3D00070470000380000203A0000204000002074
:10E3E000420000203C080020440000203C000020A7
:10E3F000F8B502F0C3F9064602F0CAF90746FEF77F
:10E40000CDFA012865D10521AB48FCF795FE5528CA
:10E4100007D10020A9490870A9490880A949888026
:10E420005FE0012F07D10020A4490870A4490880AB
:10E43000A449888055E0A1480078002808D101202F
:10E440009E49087035460A2068439D49088048E087
:10E450009C48007B42009B48801D8652801F047BA5
:10E4600011E061009748801D455A601E41009548A3
:10E47000801D415A62008152601E41009148801DFA
:10E480004552601EC4B2002C0ADD61008D48801D1B
:10E49000415A601E42008B48801D805A8142E0DB59
:10E4A0008848007B401C874908730846007B032886
:10E4B00007DB00200873084605890A206843804965
:10E4C00008807F4800887F49888001207B49087048
:10E4D00007E0002079490870794908807949087374
:10E4E0008880774800887849086074480078002858
:10E4F00015D0084600686C214843734908606421C0
:10E5000071480068F9F71CFE6F490860084600680A
:10E510006E49884206D908466B49086002E000202F
:10E52000694908606848006869490988884203D2D7
:10E53000654800680F2804D2634800886449088051
:10E540000AE06348008860490968401A0F2803D32D
:10E550005D4800885E4908805A480088401C594937
:10E560000880084600880A282CDB002008805948CB
:10E57000008857490988884203DA01205649087102
:10E5800008E05448008852490988884202DD022088
:10E590005149087150480079012840D14C48008801
:10E5A0004C49098888420DDB494801884948008860
:10E5B000FF309130814206DD46480088FF307330DD
:10E5C0004449088077E042480188424800889630F4
:10E5D000814205DD3F48008878303E4908806AE086
:10E5E0003B4801883B4800883230814205DD39488C
:10E5F00000881E30374908805DE03548018835487D
:10E6000000880A30814205DD324800880A303149ED
:10E61000088050E02E4800882E4908804BE02E48A4
:10E620000079022847D12A4800882A490988884267
:10E6300039DA27480088FF30913026490988884216
:10E6400006DA24480088FF387338224908802AE017
:10E650001F48008896301F490988884205DA1D48FE
:10E66000008878381B4908801DE01948008832303E
:10E6700018490988884205DA164800881E38154965
:10E68000088010E0124800880A3012490988884240
:10E6900005DA104800880A380E49088003E00C4863
:10E6A00000880C4908800B4800880849884202DB32
:10E6B000084608490880F8BD4C08002042000020A8
:10E6C000380000203C0800203C000020C607000065
:10E6D000400000203A0000204400002000200849AB
:10E6E000088008490880084908804880012008718E
:10E6F00000200649488008800549086070470000EE
:10E700003A00002040000020440000203C08002087
:10E710003C000020002004490870044908700021D2
:10E72000034801767047000088000020890000201F
:10E73000340A002070B500250024FEF72FF90128C7
:10E7400063D103213448FCF7F7FC552808D1002099
:10E75000324908703249087000213248017659E088
:10E760002F480078002807D102F0A8F82B4908703C
:10E7700001202B4908704DE001202949087002F062
:10E780009DF82849097E8900264A603A505025485C
:10E79000047E10E0A000234960390D5C601E8000FB
:10E7A0000858A1001F4A603A5050601E8000114670
:10E7B0000D50601EC4B2002C0ADDA000194960395A
:10E7C0000958601E8000174A603A10588142E1D310
:10E7D0001448007E401CC1B212480176007E1E28FB
:10E7E00018DB00210F48017601466039896B02462B
:10E7F000603AD26B89180246603A126C881803217D
:10E80000F9F79EFC0549087004E0002003490870F0
:10E810000349087070BD00004C08002088000020EB
:10E8200089000020340A0020F0B5A9B004460E4645
:10E830000025002700202890A0216846F9F730FD28
:10E84000FEF784FE26490A6814216143505024488B
:10E850000168142060430818C068B0420CD22048F8
:10E860000168142060430818C1681D48026814201C
:10E8700060431018416005E01948016814206043A6
:10E880000818466016484068002826D0002517E082
:10E890006806070E282F00D316E0114801681420DF
:10E8A00068430858B9006A4650500D480168142062
:10E8B000684308184168781C80001150681CC5B274
:10E8C0000748007AA842E3DC00BF6A0004486946B2
:10E8D00043680220984701202890289829B0F0BD6D
:10E8E000D82E002010B500F0F5FD00F0D7F810F09C
:10E8F0001DFB00F00DFB00F001F810BD70B54148A4
:10E900000078912800D070BD00F0BEF8012876D1C3
:10E910003D4800883D49088008468078F0218843BA
:10E9200020303A498870084680780009000135494E
:10E93000097A0907090F0843344988703148807AF9
:10E94000401E3049887208460089401C08810846EC
:10E950000089C988884216DA08202C498872002468
:10E960000EE0284841882848001D415C2748C01C0B
:10E97000015524484088401C22494880601CC4B28C
:10E98000072CEEDB2DE01F4800891E49C98888420C
:10E990001CD11C4800791B498978401AC5B2681CF3
:10E9A0001A49887200240EE0164841881648001D56
:10E9B000415C1648C01C015512484088401C114952
:10E9C0004880601CC4B2AC42EEDB0AE000F00EFDF1
:10E9D00000200C4908700C490888092100F0B8F99A
:10E9E00091E7012000F0C4FC084A917A1088921C3B
:10E9F00000F070F905490888002100F0C1F800BF57
:10EA000081E70000142C0020B02B0020402B0020B8
:10EA10001B49097E002932D01949897E0C225143B5
:10EA2000174A515A174A118000200CE01449897E78
:10EA30000C225143124A8918891C0A5C1149891C0D
:10EA40000A54411CC8B20828F0DB0D49897E0C220B
:10EA500051430B4A8918897A0A4A91720121D1726D
:10EA60000749097E491E064A11761146897E491CCE
:10EA700091761146897E022901DB0021917670474B
:10EA80000C2B0020342B00200349487B012802D1A5
:10EA90000021014A51737047242C002010B53348DF
:10EAA0004068002861D13148007B030011F024FB4D
:10EAB00007590512212E3D4A59002D48007800289B
:10EAC00007D000202A4908702A490888012100F04F
:10EAD0003FF947E026480078002809D00020244963
:10EAE000087025494A8808880123091D00F040F96B
:10EAF00038E01F480078002807D000201C49087023
:10EB00001C490888022100F023F92BE018480078FE
:10EB1000002809D000201649087017494A8808883B
:10EB20000923091D00F024F91CE011480078002891
:10EB300007D000200E4908700E490888092100F00E
:10EB400007F90FE00A480078002809D0002008499A
:10EB5000087009494A8808880323091D00F008F94C
:10EB600000E000BF00BF00F041FC10BD242C0020DD
:10EB7000142C0020B02B00204C2B002070470000EC
:10EB800070B504460D4634480088A04263D1002D7C
:10EB900061D13248007822284ED004DC20283DD0B4
:10EBA000212856D141E0902802D0912851D115E07A
:10EBB0002A48C08801280AD100202849087000F09E
:10EBC00015FC27490888002100F0C2F805E0032061
:10EBD00000F0CEFBA020214908703BE01F480089CF
:10EBE0001E49C98888420AD100201C49087000F0DB
:10EBF000FDFB1B490888002100F0AAF80DE017482A
:10EC0000807A002806D000F0F1FB1449087B00F060
:10EC100091FB02E0032000F0ABFB1BE0062000F0BC
:10EC2000A7FB11200D49087014E0062000F0A0FB9E
:10EC300011200A4908700DE000200849087000F012
:10EC4000D5FB08494A8808880923091D00F090F877
:10EC500000E000BF00BF70BD282B0020142C002056
:10EC6000B02B00204C2B002070B50346184C247E9E
:10EC7000022C00DB70BD164C647E0C256C43144DD9
:10EC80002B5300200AE0155C114C647E0C26744363
:10EC90000F4EA419A41C2554441CE0B28842F2D3A0
:10ECA0000B4C647E0C267443094EA419A1723446A1
:10ECB000247E641C35462C762C46647E641C6C765F
:10ECC0002C46647E022C01DB00246C7600BFD1E769
:10ECD0000C2B0020F0B585B007460D4616461A48A5
:10ECE0000780002406E031781748801C0155761C07
:10ECF000601CC4B2AC42F6DB2C4605E0AA211248E7
:10ED0000801C0155601CC4B2082CF7DB0E4800883B
:10ED1000019008216846C1720021417201720170A0
:10ED2000002406E00848801C015D03A80155601C12
:10ED3000C4B2082CF6DB69460448FCF704FB01204A
:10ED40000149887205B0F0BD282B00209055044081
:10ED500070B504460D462946204610F009F870BDEE
:10ED600070B504460D462946204610F00FF870BDD8
:10ED7000F8B504460D4616461F463B463246294620
:10ED8000204610F004F8F8BDF8B507460E461546C3
:10ED90005C480078002804D009213846FFF7D8FFE6
:10EDA000F8BD002D01D0602D04DD09213846FFF7A4
:10EDB000CFFFF5E7544807804580002406E031780E
:10EDC0005148001D0155761C601CC4B2AC42F6DBF4
:10EDD00000204C49487008468580FF2088727F20BB
:10EDE00008730846808808282EDA0120C880084663
:10EDF0008088488001200881434800884349088072
:10EE000008468078F0218843404988700846807819
:10EE1000000900013B4909790907090F08433B49EB
:10EE2000887038480079401C8872002407E0364812
:10EE3000001D015D3548C01C0155601CC4B231483D
:10EE40008088A042F3DC4AE00721681CF9F78EF9BC
:10EE5000002907D0072128460830F9F787F9294902
:10EE6000C88005E00721681CF9F780F92549C880AA
:10EE7000062024494880012008812348008823492E
:10EE8000088008468078F021884310301F49887038
:10EE900008468078000900011A4989880905090F88
:10EEA00008431A49887008464088FF2109028843B0
:10EEB000144989880902FF221202114008431349AC
:10EEC000488008208872002407E00F48001D015D7B
:10EED0000E48001D0155601CC4B2062CF5DB012054
:10EEE00000F046FA094A917A1088921CFFF7F2FE68
:10EEF000902004490870054908880021FFF740FE6A
:10EF000000BF4DE7142C0020B02B0020402B002028
:10EF100010B5FFF77DFD1448C07A002822D01248B2
:10EF200080780009002806D0012807D002280AD0DE
:10EF3000032810D10CE000F0A5F90FE000F09EF8D6
:10EF400000F062FA0AE000F011F800F05DFA05E066
:10EF500000F000F902E0FFF711FE00BF00BF002043
:10EF60000149C87210BD0000342B002010B5404884
:10EF70000078112800D010BD3E4800883F2149018B
:10EF8000884200D0F7E73B4880780007000F3849F7
:10EF9000097A0907090F88420CD00020344908700B
:10EFA00000F024FA34494A8808880423091DFFF731
:10EFB000DFFEE0E72E480089401C2D490881084605
:10EFC000807A401E887208460089C98888421BDA08
:10EFD0002848807A082800D0CDE700240EE0254894
:10EFE000C01C015D224842882348001D81542048EE
:10EFF0004088401C1E494880601CC4B2072CEEDBD0
:10F00000062000F0B5F930E0194880881849498891
:10F01000401A1849897A884203DA1648807A082803
:10F0200000D0A8E700240EE01248C01C015D104883
:10F0300042881148001D8154601CC4B20C484088AD
:10F04000401C0B4948800A48408809498988884201
:10F05000EADB00200649087000F0C8F906494A8832
:10F0600008880023091DFFF783FE00BF83E7000027
:10F07000142C0020342B00204C2B002070B532487B
:10F08000007880210840802800D170BD2F4800887A
:10F090003F214901884200D0F7E72C48807A0828B0
:10F0A00000D0F2E72948807805072D0F2D02274868
:10F0B0004088000A0543082D00DAE6E700202249CF
:10F0C0004870062048800846858001200881082075
:10F0D00088720020C8728988481C0721F9F746F811
:10F0E000002909D018498988084608300721F9F70E
:10F0F0003DF81549C88007E013498988481C072155
:10F10000F9F734F81049C880104800881049088081
:10F1100008464580002407E00C48001D015D0C48AE
:10F12000001D0155601CC4B2062CF5DB042000F064
:10F130001FF9102004490870054A51881088FFF70C
:10F140000FFE00BFA1E70000142C0020342B00208C
:10F150004C2B002010B548480078A02808D046481D
:10F160000078912804D044480078A12800D010BD30
:10F17000424800883F21490188420AD04049088816
:10F180000921FFF7E5FD00F031F900203A49087048
:10F19000EDE73A48807A08280AD0394908880921D9
:10F1A000FFF7D6FD00F022F9002033490870DEE7B2
:10F1B000324880780007000F002804D001282DD0A5
:10F1C00002284BD136E02C484078002800D050E08F
:10F1D0002A48C078002803D101202749487003E05D
:10F1E0002648C078244988722348007891280BD09B
:10F1F00022480079002803D101201F49087303E049
:10F200001E4800791C49087391201B49087000F0C2
:10F21000EDF81949087B00F08DF82AE0164840788F
:10F22000002800D025E0A12013490870032000F039
:10F230009FF81EE010484078002800D019E00E48E2
:10F240000078A02809D10E4908880821FFF780FD21
:10F2500000F0CCF80020084908700AE00849088846
:10F260000521FFF775FD00F0C1F800200249087084
:10F2700000BF00BF00BF7AE7142C0020342B002011
:10F28000B02B002010B52848007880210840802845
:10F2900000D110BD24480078002806D023480088FB
:10F2A0003F214901884200D0F3E72048807A1F4976
:10F2B00089780907090F884203DD1C48807A0828ED
:10F2C00000D0E6E7194880780007000F002805D035
:10F2D000164880780007000F072800DDD9E713489B
:10F2E000008813490880114880780007000F488083
:10F2F000002407E00D48C01C015D0D48001D0155AC
:10F30000601CC4B20A484088A042F3DC00200649D1
:10F31000087000F06BF806494A8808880023091D28
:10F32000FFF726FD00BFB4E7142C0020342B00208B
:10F330004C2B00207F2805DC7D21C90041430A4A6F
:10F3400091600DE0F12808DBF92806DC0107090FC0
:10F3500064225143044A916002E00449024A9160E8
:10F360000221014A51737047242C002018F001003B
:10F3700000B5030010F0C0FE0729050B11171D236F
:10F3800029000121144A11731449516022E002211D
:10F39000114A1173114951601CE003210E4A117387
:10F3A0000F49516016E004210B4A11730D49516059
:10F3B00010E00521084A1173002151600AE006217E
:10F3C000054A11730849516004E00021024A117393
:10F3D000516000BF00BF00BD242C0020A8610000C8
:10F3E000F824010028230000F04902000020014910
:10F3F00008737047242C0020024909880918014A23
:10F4000011807047242C002010B52F480078102858
:10F4100018D12E48408860280ADD2D4880780009E0
:10F420000001801C2A49887022202749087025E0A5
:10F43000274880780009000125498870202022494A
:10F4400008701BE020480078112816D11E48807AE9
:10F45000002800D010BD1C484078002800D0F9E7F3
:10F460000820194988721A48807800090001184953
:10F47000887020201449087000E0EBE7FD20C000F0
:10F480001349088008468078F021884330301049BD
:10F4900088700846C0780020C8700846007914209B
:10F4A0000871032088720220FFF762FF084A917AF0
:10F4B0001088921CFFF70EFC054908880021FFF711
:10F4C0005FFB00BFC6E70000142C00204C2B00207F
:10F4D000402B0020244A118852888A4242D0224A76
:10F4E00052888A4204DA204A52888A1A90B207E087
:10F4F0001D4A52880023DB439A1A521C521890B2BC
:10F50000194A5180127B002A10D0174A5268002AEB
:10F510000CD0154A5268824205D9134A5268121A11
:10F52000114B5A6002E000220F4B5A600E4A527B88
:10F53000022A17D10C4A9268002A0CD00A4A926813
:10F54000824205D9084A9268121A074B9A6002E073
:10F550000022054B9A60044A9268002A02D10122D7
:10F56000014B5A7370470000242C002010B506F0A0
:10F5700073F810BD00BF704710B5044680202043CB
:10F5800001460320400205F021FF10BD10B51021F7
:10F590000320400205F01AFF10BD000010B5022440
:10F5A000024805F063FF0446204610BD0106000036
:10F5B00010B50021014805F009FF10BD010600004B
:10F5C00010B50446802020430146024805F0FEFEA7
:10F5D00010BD00000106000010B51021014805F023
:10F5E000F5FE10BD0106000030B503460C460021B3
:10F5F00001250D48834201D0002B01D1022030BDEE
:10F60000012A01D10120FAE7002108E0C8002058B2
:10F61000984202D100252846F1E7481C81B2914268
:10F62000F4DB2846EBE70000FFFF0000002000BFEE
:10F6300014E00021C200134B9950C200D2189180EF
:10F64000C200114B9950C200D2189180C2000F4BDA
:10F650009950C200D2189180411C88B24828E8DB3A
:10F660000B490C4A11600C495160002191600B4913
:10F6700011610B49D16000210A4A11800A4A1170B8
:10F6800070470000841F0020C421002004240020B3
:10F69000490B0100701F0020E50B01008F0C0100D9
:10F6A000810C0100D2000020D6000020F0B585B00A
:10F6B0000646674F3846039002900025002400203C
:10F6C0000190009063480068002803D061490868F1
:10F6D000804707465F484068002803D05D49486876
:10F6E000804703905B488068002803D059498868A8
:10F6F0008047029057480069002803D0554908699F
:10F70000804700905348C068002803D05149C8681A
:10F7100080470546482D00DD48250098002876D012
:10F72000002D74DD4C480088A8420BDA2B463A467F
:10F7300049494A48FAF7D2FF2B4647494748039AB6
:10F74000FAF7CCFF44480088002833DD424800889F
:10F75000A84202D1002040490880002415E0E000C2
:10F760003F490858E1003D4A515888420BD0E0001B
:10F7700011460858E1003A4A5050E0001146085836
:10F78000E100384A5050601C84B2AC42E7DB0120F3
:10F79000354908702C460BE00020E100314A5050FA
:10F7A000E1002F4A5050E1002C4A5050601C84B2B6
:10F7B000482CF1DB2B4800682549884246D029486F
:10F7C00080882A49884205DA264880888019254998
:10F7D00088803BE00020234988800846006801902B
:10F7E000012D33DD002408E0601CC0001D490858CD
:10F7F000E1001C4A5050601C84B2681EA042F3DC39
:10F80000691EC900174A019850501FE0FFE7002009
:10F8100015490870002414E00020E100114A5050FE
:10F82000E10089188880E1000C4A5050E1008918F5
:10F830008880E1000A4A5050E10089188880601CE5
:10F8400084B2482CE8DB00200349088005B0F0BDF5
:10F85000FFFF0000701F0020D2000020C421002004
:10F8600004240020841F0020D600002088130000FC
:10F870002E480078401C2D4908702D480078401C07
:10F880002B4908702B480078401C2A4908702A48E8
:10F890000068401C2849086008460068FF21913133
:10F8A000884202D900202449086020480078C828EE
:10F8B00002D900201D4908701D480078842802D90B
:10F8C00000201B4908701B480078502802D90020EE
:10F8D00018490870194818490968405C18490870A7
:10F8E000184812490978405C1749087017481049B0
:10F8F0000978405C1649087016480E490978405C42
:10F9000015490870154809490978405C1449087080
:10F91000144806490978405C1349087013480349A4
:10F920000978405C12490870704700004F070020BA
:10F930005007002051070020540700205B160200EA
:10F9400048070020EB17020049070020B318020007
:10F950004A070020FF1902004C0700203719020057
:10F960004B0700204F1A02004D070020171B020012
:10F970004E07002010B58200054BD218525C012AB8
:10F9800004D100228300024C1B195A5410BD000000
:10F99000902A002010B50446204600F04FFA204679
:10F9A00000F002F810BD000010B50446B24800781F
:10F9B00000287DD1B1480088B149884278DAB14841
:10F9C000007800284FD0B0480078002803D0AB481A
:10F9D0000088AE490880AE480078002818D1A748B2
:10F9E0000188AA4800880F30814206D30120A84927
:10F9F0000870A2480088A5490880A0480088A3494B
:10FA0000098888421CDA9D480088A049088017E0D0
:10FA10009E480188994800880F30814206D3002013
:10FA20009B49087095480088984908809348008849
:10FA300096490988884203DD9048008893490880E8
:10FA400093480078002857D192480078042803D0C2
:10FA50008D480078002807D088480088822803DA7B
:10FA600005208C490870A1E08A480078032803D05B
:10FA700085480078002809D080480088FF21193186
:10FA8000884203DA0420834908708FE081480078B7
:10FA9000022803D07C48007800280AD077480088E4
:10FAA000FF21AF31884204DA03207A4908707DE0F3
:10FAB000E0E078480078012803D0734800780028F7
:10FAC00008D06E4800887449884203DA02207149E0
:10FAD00008706BE06F480078002803D06A4800780F
:10FAE000002863D0654800886B49C83188425DDAD8
:10FAF00001206849087059E065480078012855D10F
:10FB000064480078012803D05F480078002809D0B5
:10FB10005A4800886049C831884203DB00205D49AB
:10FB2000087043E05B480078022803D0564800780C
:10FB3000002808D0514800885749884203DB01203B
:10FB40005449087032E053480078032803D04E48E7
:10FB50000078002809D049480088FF21AF31884249
:10FB600003DB02204B49087020E04A480078042853
:10FB700003D045480078002809D040480088FF217C
:10FB80001931884203DB0320424908700EE04148E6
:10FB90000078052803D03C480078002806D0374874
:10FBA0000088822802DB04203A490870FCF7DCFE5A
:10FBB0003349643988425DD33848006800193749B1
:10FBC000086031480078002808D000202E490870CD
:10FBD000324908602F4800783149087000F082FDF2
:10FBE00000281FD12D4800682E49884239D30020B3
:10FBF0002A4908602A48007826490978884205DAA7
:10FC000027480078401C264908702AE024480078DC
:10FC100020490978884224DD21480078401E204987
:10FC200008701EE01D4800681F49884219D3002053
:10FC30001A4908601A48007816490978884205DA96
:10FC400017480078401C164908700AE014480078EC
:10FC500010490978884204DD11480078401E104997
:10FC600008700F4800780B490978884202D10020BB
:10FC70000A49086010BD00000B00002002000020AF
:10FC80001C0C0000120000200800002004000020CE
:10FC90000A00002006000020C60200001800002014
:10FCA00007000020C05D0000407E050000200B49D9
:10FCB00008700B49087001200A4908700A49087049
:10FCC00000200A4908700A4908700A4908800A4950
:10FCD00008800A4908800A49087070470600002019
:10FCE0000700002008000020090000200A00002072
:10FCF0000B0000200C0000200E000020100000204F
:10FD00001200002000200B4908700B4908700120E8
:10FD10000A4908700A49087000200A4908700A490F
:10FD200008700A4908800A4908800A4908800A4977
:10FD3000087070470600002007000020080000201F
:10FD4000090000200A0000200B0000200C00002009
:10FD50000E0000201000002012000020F1B5002746
:10FD600030480078002809D00320F9F7F7FB002875
:10FD700004D00320F9F7E6FB2B4908802B480088C4
:10FD80000A2847D3002029490880294800782828D4
:10FD900029D20320F9F7D6FB0746002407E06000CC
:10FDA0002449085AB84200DD05E0601CC4B220486E
:10FDB00000788442F3DB00BF1D48057808E0681E28
:10FDC00040001C49085A69001A4A5052681EC5B2C0
:10FDD000A542F4DC600017490F5215480078401C1A
:10FDE0001349087016E000260F2405E06000114951
:10FDF000085A8619601CC4B2192CF7D30A21304660
:10FE0000F8F79EF908490880002009490870012088
:10FE100009490870054801880098081803490880B6
:10FE2000F8BD00000900002002000020160000209C
:10FE300000000020E0070020120000203A49098855
:10FE40001E2928DA0021394A1180394A118039499E
:10FE50000988394A914207DC38490978002914D0C9
:10FE600034490988914210DD0121354A1170002181
:10FE7000344A1170344A1170304A11700121334AEA
:10FE800011700021324A11704CE02A490988091882
:10FE9000284A118046E024490988274A6432914261
:10FEA0002BDB0021234A1180214A11801F49098838
:10FEB000AF221201914207DC20490978002916D0AF
:10FEC0001A490988914212DD02211D4A1170002150
:10FED0001C4A117005211C4A11700021174A11702B
:10FEE00001211A4A11700021194A11701AE00F49B4
:10FEF000098809180D4A118014E000210D4A11806B
:10FF00000A4A11800A4909880B4A914205DD0021FD
:10FF10000B4A1170094A117004E005490988091853
:10FF2000034A1180704700000200002010000020EA
:10FF30000C0000200E000020B80B0000090000207B
:10FF40000B00002006000020070000200800002011
:10FF50000A0000200148007870470000B409002022
:10FF60000148007A70470000B409002001488078F9
:10FF700070470000B4090020014800887047000065
:10FF80007C000020F8B50023002500950024002205
:10FF900000BF94E001259D40ACB20D88254000953E
:10FFA000009DA5426FD11A468D79012D0DD1464D88
:10FFB00003263602AD192D5C012696403543424E8C
:10FFC00003273F02F61935540CE03F4D0326360255
:10FFD000AD192D5C01269640B5433B4E03273F02E9
:10FFE000F6193554CD78002D4ED1374D60352D5C46
:10FFF000CE78002E01D1012600E000269640B543C0
:020000040001F9
:10000000314E603635548D78002D2ED12E4D192667
:100010007601AD192D5C8E78002E01D1012600E00D
:1000200000269640B543284E19277F01F61935540E
:100030000D79002D0ED1244D50352D5C0E79002EFA
:1000400001D1012600E000269640B5431E4E5036F1
:10005000355423E01C4D50352D5C0E7996403543C8
:10006000EEB2194D50352E5418E0174D1926760171
:10007000AD192D5C8E7896403543134E19277F01BC
:10008000F61935540AE018E00F4D60352D5CCE7836
:1000900096403543EEB20C4D60352E544D79012D0E
:1000A0000AD1094D30352D5C012696403543EEB21C
:1000B000054D30352E5400E000BF5D1CABB2082B5F
:1000C00000DA67E7F8BD000000000440FFB507460E
:1000D00015461E4600243846019900F01FF80028F6
:1000E00002D0012004B0F0BD00240CE00A206043DF
:1000F0000949085CB04204D12946204600F05EF868
:1001000007E0601C84B20A2060430349085C0028B1
:10011000ECD100BF0020E5E7A80100200246002A3C
:1001200003D1402901DD01207047032A03D10229B0
:1001300001DD0120F8E7042A03D1202901DD012097
:10014000F2E7052A03D1202901DD0120ECE70C2A82
:1001500003D1102901DD0120E6E70D2A05D101298F
:1001600003DD402901DA0120DEE70E2A03D1202930
:1001700001D10120D8E70020D6E7000010B5064ADB
:1001800003231B02D218125C8A43034B032424026C
:100190001B191A5410BD00000000044010B5064A97
:1001A00003231B02D218125C0A43034B03242402CC
:1001B0001B191A5410BD00000000044070B502461F
:1001C0000020B1E00A2353435A4C1B195B1C440026
:1001D00004191B199B788B427DD10A235343554C3C
:1001E0001B195B1C440004191B195B78082B33D1C5
:1001F0000A2353434F4C1B195B1C440004191B5723
:100200004D4C4E4D6419E35C012423430A245443AE
:10021000484D6419641C450045196457464D474EC6
:10022000AD192B550A235343424C1B195B1C440048
:1002300004191B57404C35466419E35C02242343E0
:100240000A2454433B4D6419641C45004519645706
:10025000394DAD192B5564E00A235343354C1B1916
:100260005B1C440004191B195B78092B34D10A2349
:100270005343304C1B195B1C440004191B572E4C74
:100280002E4D6419E35C402423430A245443294D32
:100290006419641C450045196457274D274EAD1954
:1002A0002B550A235343234C1B195B1C4400041990
:1002B0001B57214C35466419E35C8024A3430A2470
:1002C00054431C4D6419641C4500451964571A4D6C
:1002D000AD192B5525E025E00A235343154C1B1976
:1002E0005B1C440004191B57134C144D6419E35C48
:1002F0000A2454430F4D6419641C450045196419C0
:1003000065780124AC402343DCB20A235343094DF2
:100310005B195B1C450045195B57074D074EAD192E
:10032000EC5404E0431CD8B2032800DA4AE700BFCB
:1003300070BD0000A8010020000004407508000006
:10034000F8B50024FCF72AFB012861D100F082FBFC
:100350000446FF220721002003F078F8012C21D168
:1003600000F098FC00280ED000F0A8FB054600F035
:1003700099FB064601200346024629460090304676
:1003800005F0A4FB50E000F099FB054600F08AFB65
:10039000064601200023024629460090304605F01B
:1003A00095FB41E0022C21D100F074FC00280ED016
:1003B00000F084FB054600F075FB0646012003466D
:1003C000024629460090304605F080FB2CE000F004
:1003D00075FB054600F066FB0646002001231A4621
:1003E00029460090304605F071FB1DE000F052FCFC
:1003F000054600F063FB064600F054FB074601206B
:1004000003462A4631460090384605F05FFB0BE074
:100410000020034602460146009005F057FB0022EB
:100420000721104603F012F8F8BD0000FEB50024C5
:1004300071480078012824D1FCF7B0FA012812D1C4
:10044000FCF78EF800BF0BE0182C02D1601CC4B280
:1004500004E0FF222146002002F0F8FF601CC4B235
:10046000242CF1DBC6E0FCF7C7F9002406E00022EB
:100470002146104602F0EAFF601CC4B2242CF6DBD1
:10048000B8E0FCF78BFA012876D1FCF76DFA5B49EE
:1004900088426ED300F00CFB064600F023FB0746B3
:1004A0000A21F7F74DFE05463246294601200BF09A
:1004B000A1F800F029FD064600F0CEFC0A210290CA
:1004C000F7F73EFE054600F0F3FA074632462946A6
:1004D00009F038F8FFF734FF00F0AAFA054629467C
:1004E000012007F075FB00F0F7FA0646FF21F53111
:1004F000F7F73CFEC5B22946012006F0A5FAFFF742
:1005000029FD0546FFF738FD0646FFF72FFD074694
:100510002B4632463946012005F0B2FD00F0E8F8DE
:100520000546294601200BF00BFB00F0B5FC054603
:1005300000F0C2FB064600F0B5FC074600F0C2FB27
:1005400000233A46014600960195029001200AF0E8
:1005500077FD00F075FC054600F06CFC064600F0E7
:1005600075FC07462A46314607F06AFD42E003E083
:10057000FFE7FCF76FF83DE0FCF73EF9002223218E
:10058000104602F063FF00222221104602F05EFFB7
:1005900000220721104602F059FF002208211046D0
:1005A00002F054FF00220921104602F04FFF002202
:1005B0000A21104602F04AFF00221321104602F0E1
:1005C00045FF00221121104602F040FF00221221B7
:1005D000104602F03BFF00220E21104602F036FFCB
:1005E00000220F21104602F031FF00221021104698
:1005F00002F02CFFFEBD0000FD000020B80B000043
:1006000001490860704700007C070020024800682C
:10061000401C01490860704778070020F3B581B09D
:10062000064600200E49086000F01EF8044600F05F
:100630001BF805462F1B3046029903F0B3FE0090CD
:100640000AE000F011F805462F1B06480068002854
:1006500002D004480068804700988742F1D3FEBD6D
:10066000780700207C0700200148006870470000E0
:10067000780700200B490978012901D101200FE0FA
:1006800008490978022901D1022009E005490978C1
:10069000032901D1042003E00121024A1170012045
:1006A000704700000D07002010B5094B1B8899B258
:1006B0000A12C8B2D3433133064C2370C3432333E9
:1006C000637013465633A37003467133E37010BD55
:1006D00040070020130700200148008870470000F1
:1006E00020000020014800887047000038000020EA
:1006F0000148007870470000880000200148007819
:10070000704700008900002010B50022052106482E
:10071000FAF700FD0402012205210348FAF7FAFC6A
:10072000201880B210BD00004C08002010B5062231
:1007300005210348FAF7EEFCC006C00F10BD00000B
:100740004C08002010B5042205210648FAF7E2FC07
:100750000402052211460348FAF7DCFC201880B297
:1007600010BD00004C08002010B5062205210248EB
:10077000FAF7D0FCC01110BD4C08002010B50222C1
:1007800005210248FAF7C6FC10BD00004C08002005
:1007900010B5062205210348FAF7BCFC8006C00FFD
:1007A00010BD00004C08002010B5042202210348AF
:1007B000FAF7B0FCC007C00F10BD00004C080020C5
:1007C00010B5052202210348FAF7A4FCC007C00FA8
:1007D00010BD00004C08002010B500220421034881
:1007E000FAF798FC4006400F10BD00004C080020AE
:1007F00010B5042201210248FAF78CFC801110BDCB
:100800004C08002010B5002201210248FAF782FCB2
:1008100010BD00004C08002010B50522012103483E
:10082000FAF778FC8007800F10BD00004C0800200C
:1008300010B5012211460248FAF76CFC10BD000009
:100840004C08002010B5002206210C48FAF762FC83
:100850000402012206210948FAF75CFC2018040270
:10086000022206210548FAF755FC2018040203224B
:1008700006210248FAF74EFC201810BD4C08002053
:1008800010B5042206210C48FAF744FC04020522A4
:1008900006210948FAF73EFC2018040206221146F8
:1008A0000548FAF737FC20180402072206210248FF
:1008B000FAF730FC201810BD4C08002010B50222B9
:1008C00003210248FAF726FC10BD00004C08002066
:1008D00010B5032200210248FAF71CFC10BD0000ED
:1008E0004C08002010B5002211460248FAF712FC0D
:1008F00010BD00004C08002010B504220021024861
:10090000FAF708FC10BD00004C08002010B50122C9
:1009100000210248FAF7FEFB10BD00004C08002041
:1009200010B5052200210248FAF7F4FB10BD0000C3
:100930004C080020322815DA3C498978012903DD6A
:1009400001213A4A517070E038498978002905DD63
:100950002F286ADC0021354A517066E00021334AB5
:10096000517062E03E2817DA322815DB2F4989786A
:10097000022903DD02212D4A517056E02B49897866
:10098000012905DD3B2850DC0121284A51704CE04B
:100990000121264A517048E0502817DA3E2815DB1D
:1009A00022498978032903DD0321204A51703CE064
:1009B0001E498978022905DD4D2836DC02211B4AB3
:1009C000517032E00221194A51702EE0622817DA84
:1009D000502815DB15498978042903DD0421134AC1
:1009E000517022E011498978032905DD5F281CDC5C
:1009F00003210E4A517018E003210C4A517014E093
:100A000073280FDA62280DDB08498978042905DD8F
:100A100070280ADC0421054A517006E00421034ACB
:100A2000517002E00521014A51707047B40900205D
:100A30000148007870470000070000200148006866
:100A400070470000841F00200148007870470000B4
:100A5000F10000200148007870470000F0000020FD
:100A6000F8B5002600240025FCF7BAFE07460A2147
:100A7000F7F766FB054609480068854200D303E0A6
:100A800006480068461B34467D200001844200D39E
:100A90000446034804600068F8BD000024010020FB
:100AA000200100200148007870470000F500002078
:100AB0000148007970470000342800200148407840
:100AC00070470000F50000200148007A70470000E0
:100AD000342800200020704701480088704700003B
:100AE0002200002010B50024FFF7E2FF00280AD101
:100AF0000A4800880A49884202DB084607490880FC
:100B00000648048808E005480088FCF717FC84B212
:100B10000448844200DB0446204610BD3A00002011
:100B2000C6070000CE040000002005490988054AD8
:100B3000914202DB1146024A118001490888704740
:100B40003A000020C6070000F8B50027002500265F
:100B50000024FFF7C7FE0546FFF7D8FE0646F02043
:100B6000284000110A2805DBF02028400011C01C95
:100B7000044303E0F0202840001104432402280726
:100B8000000F0A2804DB2807000FC01C044302E002
:100B90002807000F04432402F020304000110A28E7
:100BA00005DBF02030400011C01C044303E0F020BE
:100BB00030400011044324023007000F0A2804DBF0
:100BC0003007000FC01C044302E03007000F04434D
:100BD000002C01D10248F8BD27463846FBE700004B
:100BE000FFFF0000F8B50027002500260024FFF7CE
:100BF00083FE0546FFF794FE0646F02028400011CC
:100C00000A2805DBF02028400011C01C044303E043
:100C1000F02028400011044324022807000F0A286E
:100C200004DB2807000FC01C044302E02807000F64
:100C300004432402F020304000110A2805DBF02094
:100C400030400011C01C044303E0F020304000118C
:100C5000044324023007000F0A2804DB3007000F8A
:100C6000C01C044302E03007000F0443002C01D1F4
:100C70000248F8BD27463846FBE70000FFFF0000AA
:100C800010B50024FFF724FE0446204610BD0120C5
:100C900070470000014800787047000049070020B5
:100CA00001480078704700004B0700200148C07BD6
:100CB00070470000C00900200148007A704700001A
:100CC000C009002010B5002405480088323084B2E5
:100CD00064212046F7F74AFA84B2204610BD00008E
:100CE000C009002070B5002407490868FBF776FFAB
:100CF00005466421F7F724FA84B20448844200DDF3
:100D00000446204670BD0000C0090020DE0300003C
:100D100010B5002400F016F8012801D103240CE0DE
:100D200000F010F8022802D1FF24373405E00A2130
:100D300003480088F7F71AFA84B2204610BD000075
:100D40000200002001480078704700000B000020DE
:100D500010B50024044804F089FB002801D00124C8
:100D600000E00024204610BD0307000010B5002459
:100D7000044804F07BFB002801D0012400E000249B
:100D8000204610BD0507000010B50024044804F0FB
:100D90006DFB002801D0012400E00024204610BD96
:100DA0000707000010B50024062004F05FFB0028B0
:100DB00001D0012400E00024204610BD10B500241D
:100DC000052004F053FB002801D0012400E000249A
:100DD000204610BD10B50024044804F047FB00284D
:100DE00001D0012400E00024204610BD06070000C9
:100DF00010B50024044804F039FB002801D0012478
:100E000000E00024204610BD0305000010B50024BA
:100E1000044804F02BFB002801D0012400E000244A
:100E2000204610BD040500000148807A704700008C
:100E3000C00900200148807870470000540A002053
:100E40000148406870470000540A0020014840787B
:100E500070470000540A002070B50024FFF728FEF8
:100E6000002803D1FCF7BCFC04460DE0FFF720FE90
:100E7000012806D1FCF7B4FC0546FCF75FFA0446EE
:100E800002E0FCF7ADFC0446204670BD0148007C42
:100E900070470000C00900200148407A70470000F8
:100EA000C009002010B5002405488088323084B283
:100EB00064212046F7F75AF984B2204610BD00009D
:100EC000C009002070B5002407494868FBF786FE7A
:100ED00005466421F7F734F984B20448844200DD02
:100EE0000446204670BD0000C0090020DE0300005B
:100EF0000148007B70470000C009002001480078CD
:100F000070470000F400002070B50024FFF7D0FD0A
:100F1000002803D1FCF786FC04460FE0FFF7C8FD6C
:100F2000012807D10020FCF77DFC0546FCF706FAF6
:100F3000044603E00020FCF775FC0446204670BD23
:100F400001480078704700004200002070B5054657
:100F50000024032D00D170BD002D01D0012D1BD127
:100F600081210320800204F031FA8021134804F02B
:100F70002DFA32211248FFF751FB002409E0A200AC
:100F8000104BD2189178A200985A04F01FFA601CF6
:100F9000C4B23B2CF3DB0FE0022D0DD1002409E09D
:100FA000A200094BD2189178A200985A04F00EFAC8
:100FB000601CC4B23B2CF3DB00BFCCE70206000090
:100FC000A0860100940C0200800D0200F8B50021FB
:100FD00000240023002200BF0AE001258D40ABB2AF
:100FE00005881D402C469C4200D10A464D1CA9B2E2
:100FF0001029F2DB0588FF2D1FDC284D6D7E068849
:10100000B543264E757635462D7E0688B543234E6C
:10101000357635466D7E8678F607F60F9640354371
:101020001E4E757635462D7E867802273E40760820
:1010300096403543194E357622E0184DED7E0688F0
:10104000B543164EF5763546AD7E0688B543134E4C
:10105000B5768578ED07ED0F1646083EB5400F4E84
:10106000F67E35430D4EF5768578022635406D08BF
:101070001646083EB540094EB67E3543074EB57656
:101080000025009505E000BF6D462D786D1CEEB281
:1010900000966D462D78012DF5D9F8BD206B0440E2
:1010A000C107C90F002905D00021394A117100225A
:1010B00038490A7102210140002905D00021344A33
:1010C0001172002233490A7204210140002905D01F
:1010D00000212F4A117300222E490A730821014072
:1010E000002905D000212A4A1174002229490A74D6
:1010F00010210140002905D00021254A1175002248
:1011000024490A7520210140002905D00021204AE8
:10111000117600221F490A7640210140002904D09F
:1011200000221B494A711B494A7180210140002954
:1011300004D0002216494A7216494A72FF21013131
:101140000140002904D0002211494A7311494A7311
:10115000012149020140002904D000220C494A74AF
:101160000C494A74012189020140002904D000225F
:1011700007494A7507494A750121C90201400029FA
:1011800004D0002202494A7602494A76704700009C
:101190000060004000610040C107C90F002905D070
:1011A00001223C490A7100213B4A11710221014090
:1011B000002905D0012237490A720021364A1172EE
:1011C00004210140002905D0012232490A7300217F
:1011D000314A117308210140002905D001222D490F
:1011E0000A7400212C4A117410210140002905D0F5
:1011F000012228490A750021274A11752021014042
:10120000002905D0012223490A760021224A1176BD
:1012100040210140002905D001221E494A710022C7
:101220001D494A7180210140002905D00122194938
:101230004A72002218494A72FF21013101400029F7
:1012400005D0012213494A73002213494A73012130
:1012500049020140002905D001220E494A740022AA
:101260000D494A74012189020140002905D001225B
:1012700008494A75002208494A750121C9020140FE
:10128000002905D0012203494A76002202494A7604
:1012900070470000006100400060004010B50C483D
:1012A0000078002803D00B4A5068916888470848A6
:1012B0004078002803D0084A50689168884704485D
:1012C0008078002803D0054A50689168884710BD8F
:1012D00000600040F802002078040020F80500209B
:1012E00010B508480079002803D0074A10695169F1
:1012F000884704484079002803D0044A5068916820
:10130000884710BD00600040F802002084040020DF
:1013100010B50848007A002803D0074AD069116A3E
:1013200088470448407A002803D0044A50689168EE
:10133000884710BD00600040F802002090040020A3
:1013400010B50848007B002803D0074A906AD16A8C
:1013500088470448407B002803D0044A50689168BD
:10136000884710BD00600040F80200209C04002067
:1013700010B50848007C002803D0074A506B916BD9
:1013800088470448407C002803D0044A506891688C
:10139000884710BD00600040F8020020A80400202B
:1013A00010B50848007D002803D0074A106C516C26
:1013B00088470448407D002803D0044A506891685B
:1013C000884710BD00600040F8020020B4040020EF
:1013D00010B50848007E002803D0074AD06C116D74
:1013E00088470448407E002803D0044A506891682A
:1013F000884710BD00600040F8020020C0040020B3
:1014000010B50848407F002803D0074A506891680B
:1014100088470448007F002803D0044A906DD16DAE
:10142000884710BD00600040CC040020F802002076
:1014300010B508484078002803D0074A50689168E2
:10144000884704480078002803D0044A506E916E03
:10145000884710BD20600040D8040020F80200201A
:1014600010B509480079002803D0084A106F516F61
:1014700088470548001D4078002803D0044A50687A
:101480009168884710BD000020600040F8020020ED
:10149000E404002010B5034AD06F78329168884781
:1014A00010BD0000F802002010B5024A5068916893
:1014B000884710BD7C03002010B50948007C002837
:1014C00003D0084A50689168884705481030407832
:1014D000002803D0044A50689168884710BD000076
:1014E00020600040880300200805002010B5024A53
:1014F00050689168884710BD9403002010B5024AD7
:1015000050689168884710BDA003002010B50948B5
:10151000007F002803D0084A506891688847054832
:101520001C304078002803D0044A506891688847EE
:1015300010BD000020600040AC0300202C050020FE
:1015400010B50C480078002803D00B4A5068916809
:10155000884708484078002803D0084A50689168B6
:10156000884704488078002803D0054A506891686D
:10157000884710BD40600040B803002038050020B7
:10158000B806002010B50D480079002803D00C4A99
:101590005068916888470948001D4078002803D0AA
:1015A000084A5068916888470448001D80780028E0
:1015B00003D0054A50689168884710BD40600040DC
:1015C000C403002044050020C406002010B50D48C7
:1015D000007A002803D00C4A50689168884709486F
:1015E00008304078002803D0084A5068916888473E
:1015F000044808308078002803D0054A5068916874
:10160000884710BD40600040D003002050050020F6
:10161000D006002010B50D48007B002803D00C4AEE
:1016200050689168884709480C304078002803D0FA
:10163000084A50689168884704480C308078002830
:1016400003D0054A50689168884710BD406000404B
:10165000DC0300205C050020DC06002010B50D48EE
:10166000007C002803D00C4A5068916888470948DC
:1016700010304078002803D0084A506891688847A5
:10168000044810308078002803D0054A50689168DB
:10169000884710BD40600040E80300206805002036
:1016A000E806002010B5024A50689168884710BDCE
:1016B000F403002010B50948007E002803D0084A32
:1016C000506891688847054818304078002803D052
:1016D000044A50689168884710BD0000406000408F
:1016E000000400208005002010B50948007F002874
:1016F00003D0084A50689168884705481C304078F4
:10170000002803D0044A50689168884710BD000043
:10171000406000400C0400208C05002010B50848F3
:101720000078002803D0074A506891688847044829
:101730004078002803D0044A50689168884710BD5B
:1017400060600040180400209805002010B509488A
:101750000079002803D0084A5068916888470548F6
:10176000001D4078002803D0044A506891688847DB
:1017700010BD00006060004024040020A40500208B
:1017800010B50948007A002803D0084A50689168CB
:101790008847054808304078002803D0044A50683C
:1017A0009168884710BD0000606000403004002050
:1017B000B005002010B5024A50689168884710BDF6
:1017C0003C04002010B5024A50689168884710BD5B
:1017D0004804002010B50948007D002803D0084ABD
:1017E000506891688847054814304078002803D035
:1017F000044A50689168884710BD0000606000404E
:1018000054040020D405002010B50948007E0028AB
:1018100003D0084A506891688847054818304078D6
:10182000002803D0044A50689168884710BD000022
:101830006060004060040020E005002010B5094809
:10184000007F002803D0084A5068916888470548FF
:101850001C304078002803D0044A506891688847BB
:1018600010BD0000606000406C040020EC0500200A
:1018700010B5FE4800688079002806D001286ED097
:1018800002286DD003286CD104E2F8480068407942
:1018900003000EF031FC0A0614BC2BBC47BC67BC2D
:1018A0009BBC0AF0AFFC0020F0490968C873EF4800
:1018B00000684079401CED4909684871AEE0EC4988
:1018C0000969EA4A1268D27A885C0AF013FDE7488F
:1018D00000684079401CE54909684871E3480068A0
:1018E0004079401CE1490968487197E001F016FF12
:1018F000002810D10AF0FEFCDC4800684079401C4A
:10190000DA4909684871D94800684079401CD749CC
:101910000968487105E00AF09FFC0020D349096876
:1019200048717BE001F0FAFE002811D101200AF095
:10193000E1FCCE4800684079401CCC4909684871F8
:10194000CA4800684079401CC8490968487105E0E8
:101950000AF082FC0020C549096848715EE05FE03A
:10196000FEE0A3E101F0DAFE002828D1BF490968B2
:10197000C97A24225143BF4A12688918BB4A1268A7
:10198000D27B885C0AF0B6FCB8480068C07B401C7B
:10199000B6490968C873B5480068C07B242814D3C9
:1019A000B24800684079401CB04909684871AF48A6
:1019B00000684079401CAD490968487105E00AF0AB
:1019C0004BFC0020A9490968487127E001F0A6FEF8
:1019D000002815D1A5480068C07A401CA3490968B1
:1019E000C872A2480068C07AA1490978884207DB1A
:1019F00000209E490968C87201209C4909688871C5
:101A00000AF02AFC002099490968487106E00AF0AA
:101A100023FC002095490968487100BF00BF4FE1D1
:101A200092480068407903000EF066FB08051391A8
:101A30002A91479170910AF0E5FB00208B490968D3
:101A4000C8738A4800684079401C88490968487111
:101A500084E087490969854A1268D27A885C0AF06D
:101A600049FC824800684079401C804909684871F7
:101A70007E4800684079401C7C49096848716DE0E7
:101A800001F04CFE002811D126200AF033FC7748E3
:101A900000684079401C75490968487173480068BE
:101AA0004079401C71490968487105E00AF0D4FB8F
:101AB00000206E490968487150E001F02FFE0028AF
:101AC0001DD101200AF016FC68480068C07B401C4C
:101AD00066490968C87365480068C07B242814D328
:101AE000624800684079401C6049096848715F4855
:101AF00000684079401C5D490968487105E00AF0BA
:101B0000ABFB002059490968487127E001F006FE47
:101B1000002815D155480068C07A401C534909680F
:101B2000C87252480068C07A51490978884207DB78
:101B300000204E490968C87202204C490968887122
:101B40000AF08AFB002049490968487106E00AF05A
:101B500083FB002045490968487100BF00BFAFE022
:101B600042480068407903000EF0C6FA0805138B5E
:101B70002A8B478B638B0AF045FB00203B490968A1
:101B8000C8733A4800684079401C38490968487170
:101B90007EE037490969354A1268D27A885C0AF0D2
:101BA000A9FB324800684079401C304909684871F7
:101BB0002E4800684079401C2C490968487167E04C
:101BC00001F0ACFD002811D125200AF093FB274835
:101BD00000684079401C254909684871234800681D
:101BE0004079401C21490968487105E00AF034FB3E
:101BF00000201E49096848714AE001F08FFD002865
:101C000010D10AF077FB194800684079401C174949
:101C100009684871154800684079401C13490968F3
:101C2000487105E00AF018FB002010490968487166
:101C30002EE001F073FD002815D10C480068C07A31
:101C4000401C0A490968C87208480068C07A0849F7
:101C50000978884207DB002004490968C87203201C
:101C60000249096888710AF0F7FA05E0CC070020FC
:101C7000102F0020C8070020002012490968487171
:101C800006E00AF0E9FA00200E490968487100BF31
:101C900000BF15E000200B490968887109490968EF
:101CA0004871062007490968C87009E00AF0D4FAAB
:101CB000002004490968487102490968887100BF19
:101CC00000BF10BDCC07002010B56A4800684079FD
:101CD00003000EF011FA090610C627C644C6608E2E
:101CE000C6000AF08FFA634800684079401C6149D9
:101CF00009684871BCE0604909695E4A1268D27A95
:101D0000885C0AF0F7FA5B4800684079401C594942
:101D100009684871574800684079401C554909686E
:101D20004871A5E001F0FAFC002811D14F200AF01B
:101D3000E1FA504800684079401C4E4909684871F2
:101D40004C4800684079401C4A490968487105E0E0
:101D50000AF082FA002047490968487188E001F0DA
:101D6000DDFC002810D10AF0C5FA4248006840792D
:101D7000401C4049096848713E4800684079401C51
:101D80003C490968487105E00AF066FA00203949C3
:101D9000096848716CE001F0C1FC002822D1354887
:101DA0000068C07A401C33490968C872314800682D
:101DB000C07A3149097888420FDB00202D49096833
:101DC000C8722C4800684079401C2A49096848714B
:101DD000002028490968486208E000202549096870
:101DE000487103E000202349096848710AF034FA79
:101DF0003EE020480068407C002816D01E48C0689D
:101E0000002803D01C48C1681920884700201949C0
:101E10000968486217490968487116490968887154
:101E2000052014490968C8701AE012480068406A21
:101E3000282807D20F480068406A401C0D490968ED
:101E400048620DE000200B490968486209490968A9
:101E50004871084909688871052006490968C870F1
:101E600006E00AF0F9F9002002490968487100BF4C
:101E700000BF10BDCC070020102F002010B500249B
:101E8000F7480068807A01287ED1F5480068C0795B
:101E900000287AD0F24800688079002804D0012810
:101EA00074D0022873D191E1ED480068007B2428AA
:101EB0006ED2EB480068C07901287AD1002475E021
:101EC000E7480068C07A24214843E6490968401879
:101ED000E3490968097B415CE1480068C07A242233
:101EE0005043E14A12688018DD4A1268127B805C18
:101EF000814229D0DA480068C07A24214843DA496F
:101F000009684018D6490968097B415CD4480068D3
:101F1000C07A24225043D34A12688018D04A1268EB
:101F2000127B8154CE480068407B242805D3CC48DE
:101F30000068007BCA4909684873C9480068007B8B
:101F4000C7490968887308E0C5480068407B2428B1
:101F500003D20120C24909688871C1480068007B2A
:101F6000401CBF4909680873BD480068007B2428ED
:101F700008D3BB480068407B242803D20120B8491D
:101F800009688871B64805E0D3E1CDE169E0BAE1BE
:101F900038E00EE00068007B242804D2B0480068D6
:101FA0008079012800D103E0601CC4B2242C87D3BF
:101FB00056E0002413E0AA480068C07A2421484370
:101FC000A94909684018015DA5480068C07A242223
:101FD0005043A44A126880180155601CC4B2242CD6
:101FE000E9D300209E490968487323209C49096869
:101FF000887301209A4909688871242098490968E2
:1020000008732DE000209649096808739448006819
:10201000C07A401C92490968C87291480068C07A29
:1020200092490978884217DB8D480068007C0128B6
:1020300004D102208A490968887106E00020884995
:102040000968887186490968C8710020844909684F
:10205000C872834909680874002081490968487179
:1020600061E17F480068407903000EF045F80805FB
:1020700013A62AA651A68EA60120794909680874DC
:102080000AF0C0F8764800684079401C7449096835
:10209000487199E075490969714A1268D27A885C79
:1020A0000AF028F96E4800684079401C6C490968BC
:1020B00048716B4800684079401C6949096848715B
:1020C00082E001F02BFB00281BD165490968497BA0
:1020D000491CC8B20AF00EF961480068407B6049AB
:1020E0000968C8735E4800684079401C5C4909680B
:1020F00048715B4800684079401C5949096848713B
:1021000005E00AF0A9F800205549096848715BE02C
:1021100001F004FB00282BD151490968C97A242217
:102120005143504A126889184D4A1268D27B885C24
:102130000AF0E0F84A480068C07B401C484909683A
:10214000C87347480068C07B45490968897B884255
:102150001ADD434800684079401C414909684871CC
:102160003F4800684079401C3D49096848710BE0D0
:102170000AF072F83A480068407B39490968C87328
:1021800000203749096848711EE001F0C7FA0028AD
:102190000CD1334909688871242031490968C87312
:1021A0002F49096848732E49096888730AF054F862
:1021B00000202B490968487106E00AF04DF800201C
:1021C00027490968487100BF00BFACE02448006897
:1021D000407903000DF090FF08050F8E268E4C8E7F
:1021E000688E0AF00FF81E4800684079401C1C49B0
:1021F0000968487185E01D490969194A1268D27A4F
:10220000885C0AF077F8164800684079401C144949
:1022100009684871124800684079401C10490968F3
:1022200048716EE001F07AFA002811D125200AF0F9
:1022300061F80B4800684079401C094909684871F9
:10224000074800684079401C05490968487105E065
:102250000AF002F8002002490968487151E00000C4
:10226000CC070020C8070020C4070020102F002042
:1022700001F054FA002810D10AF03CF864480068D4
:102280004079401C6249096848716148006840799A
:10229000401C5F490968487105E009F0DDFF002036
:1022A0005B49096848712CE001F038FA00281AD11E
:1022B00057480068C07A401C55490968C87254489C
:1022C0000068C07A5349097888420CDB00205049E5
:1022D0000968C8724E49096888714D490968487192
:1022E0004B490968C87109F0B7FF002048490968DF
:1022F000487106E009F0B0FF0020454909684871BF
:1023000000BF00BF0FE009F0A7FF002040490968A7
:1023100048713F49096888713D49096808733C491B
:102320000968C87200BF71E00020394909688872E5
:102330006CE037480068807A022867D1344800682A
:10234000007A00285ED0324800684079002804D026
:1023500001280CD0032846D11BE009F053FF2C487C
:1023600000684079401C2A490968487149E000200A
:1023700009F0C0FF264800684079401C24490968DC
:102380004871234800684079401C21490968487118
:1023900037E009F001FF002812D11D48006840789D
:1023A000401C1B4909684870194800684078032898
:1023B00012D301F053FA00201549096848700BE068
:1023C0000020134909680872AA2011490968887019
:1023D00000200F490968487009F03EFF00200C49B1
:1023E000096848710DE009F037FF002008490968C5
:1023F0004871074909684870AA200549096888702A
:1024000000BF03E0002002490968887210BD000087
:10241000CC070020102F0020F8B504460D460026FA
:102420000C2060431D49085C002801D00120F8BD44
:102430000C2060431949401885600C206043401807
:102440008068002801D10120F1E701210C206043C0
:10245000124A115400222046E317DB0E1B185B11B1
:102460005B01E31A9B000E4FDB19E717FF0E3F19C4
:102470007F11DA550DF072FE00222046E317DB0EC5
:102480001B185B115B01E31A9F00064BFB18E71753
:10249000FF0E3F197F11DA553046C8E7F8020020D9
:1024A000006000400061004000BFFEE7094800886E
:1024B000401C08490880084600880749884208DD12
:1024C00006480078002804D0084602490880012008
:1024D00088707047EC000020DC050000F000002050
:1024E00010B515488078012824D1144800780128B7
:1024F0000CD113480078012808D1002011498870B8
:10250000084602F081FD00200D4908700B48007854
:1025100002280CD10C480078012808D10020094974
:102520008870084602F070FD0020074908700020FE
:102530000249087010BD0000EC000020F0000020EF
:10254000F2000020F5000020F3000020704700009A
:1025500010B500F05DFE012803D10020014908807C
:10256000887010BDEC000020F0B505460E461746F9
:1025700000243A463146284600F058FE00BF42E0AB
:1025800000202101394A126850522101374A12684D
:102590008918488000212001344A126880188180FF
:1025A0002001324A12688018C18020012F4A126827
:1025B0008018017220012D4A126880184172200192
:1025C0002A4A1268801881722001284A12688018ED
:1025D000C17200202101254A126889180873002160
:1025E0002001224A126880184173002021011F4AED
:1025F000126889188873002120011C4A126880180B
:10260000C173601CC4B21A484078A042B8DC642090
:102610001849096808807D20C0001649096848806B
:1026200015481449096888807D200001114909680E
:10263000C88010490968088110480E490968488116
:102640000F480C490968888140000A490968C88117
:102650003220084909680882FF20F53005490968D9
:102660004882044909688882F0BD00008C07002078
:1026700080070020880700204C040000102700007D
:102680003075000038B5002404E0002013490855D7
:10269000601C84B2282CF8D3012168464170017077
:1026A0006A460F490D48FFF75FFF7D21C9003220C0
:1026B00000F0ACF90B490C4800F0C6F90948643049
:1026C00000F058F90748C83000F064F9074800F0F6
:1026D00077F9074800F08AF938BD00004428002047
:1026E0004C12020028230000B80B00005424000004
:1026F0001027000010B524480078002803D10120DD
:10270000214908703EE020480078012810D11F4878
:102710000078012808D100201D498870084602F081
:1027200073FC00201949087002201749087029E03D
:1027300015480078022810D116480078012808D1E1
:10274000002013498870084602F05EFC0020114901
:10275000087003200C49087014E00B480078032827
:1027600003D10520084908700CE0074800780528C7
:1027700003D005480078062804D1002002490870DB
:102780000549087010BD0000F0000020F200002094
:10279000F5000020F3000020F4000020F8B500242C
:1027A000002500263548007800281ED134480078DE
:1027B000002803D101203249087016E03048007823
:1027C000012803D102202E4908700EE02C48007821
:1027D000022803D103202A49087006E0284800781F
:1027E000032802D1002026490870244800780128D7
:1027F0000ED10124172500262248012332462946FE
:102800000090204601F020FE01201F49087034E0AE
:102810001A48007802280FD101243B2500261948C8
:10282000401C0123324629460090204601F00CFE50
:1028300001201649087020E01048007803280DD1C7
:10284000FEF736F9002803D101201149087102E092
:1028500000200F4908710DF021FC0EE007480078B8
:10286000052803D106200549087006E003480078D2
:10287000062802D1052001490870F8BDF0000020AB
:10288000F1000020F5000020F2000020F3000020FD
:102890003428002010B5044623000DF02DFC095B00
:1028A000060E16171819595A5E00FAF75DF82C49EA
:1028B000884201D3FFF772FF50E0FAF755F8284934
:1028C000884201D3FFF716FF48E047E046E045E0C5
:1028D000FAF74AF82249884239D301F071FD2148BC
:1028E0000078032814D120480078002810D1FEF782
:1028F000EBF8002806D101201C4988608868FAF7A7
:10290000F7FF05E00020194988608868FAF7F0FFB2
:1029100014480078012805D113480078002801D117
:10292000FAF7B4F910480078052803D101201049BE
:1029300008700AE00C480078062803D102200C49F0
:10294000087002E000200A4908700BF073F905E0F6
:1029500004E003E0FFF7AAFD00E000BF00BF10BDE8
:10296000B80B0000F1000020F00000203428002007
:10297000F400002001460020054A126852898A426C
:1029800001DC012002E0024A126811817047000058
:102990008807002001460020084A126812898A42EE
:1029A00001DB012009E0054A126892898A4201DCB4
:1029B000012002E0014A1268518170478807002017
:1029C00001460020084A126852898A4201DB012030
:1029D00009E0054A1268D2898A4201DC012002E03E
:1029E000014A126891817047880700200146002043
:1029F000054A126892898A4201DB012002E0024AFC
:102A00001268D1817047000088070020024600202C
:102A10000C4B1B681B8A934201DD012010E08A42A7
:102A200001DB01200CE0074B1B689B888B4201DC1B
:102A3000012005E0034B1B681A80024B1B6859807C
:102A40007047000088070020024600200C4B1B68DE
:102A50001B8A934201DD012010E08A4201DB012044
:102A60000CE0074B1B685B88934201DB012005E00B
:102A7000034B1B689A80024B1B68D980704700008B
:102A80008807002070B5044600250C206043FE49ED
:102A9000096840184068002807D00C216143FA4AB1
:102AA000126889184868804705460C206043F6493B
:102AB0000968085C002873D10C206043F24909685A
:102AC00040188068002874D02001F0490968401837
:102AD000C07A02280AD1032D08D10C206043EA4AAB
:102AE0001268801881680120884762E02001E74968
:102AF00009684018C07A02280AD1042D08D10C2098
:102B00006043E14A1268801881680220884750E0DB
:102B10002001DE4909684018C07A02280AD1052D33
:102B200008D10C206043D84A1268801881680320BD
:102B300088473EE02001D54909684018C07A02283C
:102B40000AD1062D08D10C206043CF4A12688018A4
:102B50008168042088472CE02001CC49096840188E
:102B6000C07A02280AD1072D08D10C206043C64A3A
:102B7000126880188168052088471AE02001C3493F
:102B800009684018C07A02280BD1082D09D10C2001
:102B90006043BD4A1268801881680620884708E0B3
:102BA0000DE00C206043B84A12688018816800204C
:102BB00088472001B54909684018C5720CE30C200C
:102BC0006043B1490968085C012873D10C20604357
:102BD000AD49096840188068002874D02001AB49CD
:102BE00009684018C07A03280AD1022D08D10C20A8
:102BF0006043A54A1268801881680120884762E016
:102C00002001A24909684018C07A04280AD1022D7F
:102C100008D10C2060439C4A126880188168022009
:102C2000884750E02001994909684018C07A052872
:102C30000AD1022D08D10C206043934A12688018F3
:102C40008168032088473EE02001904909684018C8
:102C5000C07A06280AD1022D08D10C2060438A4A86
:102C6000126880188168042088472CE02001874979
:102C700009684018C07A07280AD1022D08D10C2013
:102C80006043814A126880188168052088471AE0ED
:102C900020017E4909684018C07A08280BD1022D0E
:102CA00009D10C206043784A126880188168062098
:102CB000884708E00DE00C206043734A12688018D2
:102CC0008168002088472001704909684018C57252
:102CD00082E20C2060436C490968085C0228F7D145
:102CE000002D7DD1200169490968085A68490968A1
:102CF000098A884275DA200164490968085A0A304D
:102D000081B22001614A1268115220015F490968AD
:102D1000085A5F490968098A884231DB20015B490A
:102D20000968401840885A4909680988884227DBA1
:102D30002001564909684018408855490968498862
:102D400088421DDC00202101504A12688918488001
:102D500020014E4909684018807A0028B8D10C201B
:102D6000604349490968401880680028B0D00C20A9
:102D70006043454A126880188168012088472BE229
:102D8000200142490968085A41490968098A88426C
:102D90009EDB20013D490968401840883C4909688C
:102DA0008988884294DB20013849096840184088A6
:102DB00037490968C98888428ADC00202101334AE2
:102DC0001268891848802001304909684018807AC3
:102DD0000028D4D10C2060432B490968401801E039
:102DE00063E00BE080680028C9D00C206043264ACD
:102DF00012688018816802208847EDE100202101D7
:102E0000224A1268891848802101204A12688918CC
:102E1000C872002120011D4A12688018C18020015B
:102E20001A4A1268801841722001184A12688018E4
:102E30008172184801782001144A126880180172C2
:102E400000202101114A12688918888021010F4A47
:102E500012688918087321010C4A1268891848738E
:102E600021010A4A12688918887300212001074A43
:102E700012688018C1730C20604303490968401828
:102E800080680028B9D007E0840700208C07002064
:102E900088070020800700200C206043CF4A12687A
:102EA000801881680020884796E1012DA5D1200176
:102EB000CB4909684018C07AA84225D000212001DA
:102EC000C74A12688018418000202101C44A126854
:102ED0008918C8802001C24909684018C572C148D4
:102EE00000782101BE4A1268891848720020210129
:102EF000BB4A126889188880BA4801782001B84A0C
:102F000012688018017267E12001B549096840180C
:102F1000007AB4490978884220D0B248007821016B
:102F2000AF4A1268891808722001AD490968401833
:102F3000407AAC490978884209D02001A84909683B
:102F4000401880882101A64A12688918C88000218B
:102F50002001A34A12688018818012E02001A04954
:102F6000096840188088A04988420AD220019C49FB
:102F70000968401880880A302101994A1268891826
:102F800088802001964909684018408896498842FF
:102F90000AD2200192490968401840880A3021016C
:102FA0008F4A12688918488020018D4909684018A5
:102FB000407A8C490978884205D001202101884A4D
:102FC000126889188872200185490968401840886C
:102FD000864909680988884204DB00212001804A6B
:102FE0001268115220017E4909684018807A002831
:102FF0007ED10C2060437949096840188068002818
:1030000077D02001764909684018408877490968D7
:103010000989884214DB2001714909684018007B46
:1030200000280DD10C2060436C4A1268801881681A
:103030000320884701202101694A12688918087312
:10304000200167490968401840886849096849892A
:10305000884214DB2001624909684018407B00283F
:103060000DD10C2060435D4A1268801881680420ED
:103070008847012021015A4A1268891848732001A3
:103080005749096840184088584909688989884221
:1030900014DB2001524909684018807B00280DD1BB
:1030A0000C2060434D4A12688018816805208847CB
:1030B000012021014A4A1268891888732001484971
:1030C00009684018408849490968C989884210DB65
:1030D0002001434909684018C07B00287CD10C209E
:1030E00060433E4A1268801881680620884701E0E4
:1030F00007E03BE001202101394A12688918C873B2
:103100006AE02001364909684018407A01282ED12A
:103110003448007802282AD1200131490968401832
:10312000C08832490968498A884255DB20012C4908
:103130000968401880882D490968898A88424BDBD4
:103140000C2060432549096840188068002843D056
:103150000C206043214A1268801881680720884744
:10316000002021011E4A12688918487234E02001AB
:103170001B4909684018407A02282DD11948007867
:10318000012829D12001164909684018C08817492B
:103190000968898A88421FDB2001114909684018A3
:1031A000808812490968498A884215DB0C206043EF
:1031B0000A4909684018806800280DD00C20604337
:1031C000064A12688018816808208847002021017B
:1031D000034A12688918487270BD000084070020F5
:1031E0008C07002080070020F0FF000088070020E7
:1031F00010B5002400BF04E02046FFF743FC601C2C
:10320000C4B202484078A042F6DC10BD800700201E
:1032100010B50024044802F029F9002800D000E08D
:103220000124204610BD00000304000010B5074B28
:1032300014781C7054785C70054B1960054B18604D
:1032400003461833044C236010BD000080070020A3
:1032500084070020880700208C07002010B5044652
:10326000012C09D1FF220C21002000F0EFF80121F0
:10327000022004F01FFE08E000220C21104600F09E
:10328000E5F80021022004F015FE10BD10B5002461
:1032900004210848F7F750FF552801D1012407E021
:1032A000042000F0FFFF002801D0002400E00124EA
:1032B000204610BD4C08002010B50446012C09D151
:1032C000FF221C21002000F0C1F80121062004F09B
:1032D000F1FD08E000221C21104600F0B7F80021A3
:1032E000062004F0E7FD10BD10B50024062000F014
:1032F000D9FF002801D0012400E00024204610BDA1
:1033000010B50446012C09D1FF221721002000F03E
:103310009DF80121042004F0CDFD08E000221721D2
:10332000104600F093F80021042004F0C3FD10BD06
:1033300000200449097A002901D0012000E0002082
:1033400070470000540A002010B50446022C1CD11E
:1033500000220D21104600F079F8FDF79BFC0028B3
:1033600009D0FF220B21002000F070F801210D2070
:1033700004F0A0FD58E000220B21104600F066F892
:1033800000210D2004F096FD4EE0032C1CD10022FC
:103390000B21104600F05AF8FDF77CFC002809D0FC
:1033A000FF220D21002000F051F801210D2004F032
:1033B00081FD39E000220D21104600F047F8002180
:1033C0000D2004F077FD2FE0042C0ED1FF220D21FB
:1033D000002000F03BF800220B21104600F036F8E8
:1033E00001210D2004F066FD1EE0012C0ED100220B
:1033F0000D21104600F02AF8FF220B21002000F0DA
:1034000025F801210D2004F055FD0DE000220D21CD
:10341000104600F01BF800220B21104600F016F8B1
:1034200000210D2004F046FD10BD10B50024FCF76E
:1034300097FD022801D1022406E0FCF791FD012846
:1034400001D1032400E00424204610BD10B5064B32
:103450001B78834207DD242905D224234343034CF0
:1034600024681B195A5410BD102F0020C4070020D7
:1034700010B574480068407903000CF03DFE0B075E
:1034800011D325D35A6D77D38DA8D30008F0BAFE97
:103490006C4800684079401C6A4909684871CFE06F
:1034A00069494969087808F025FF6648006840794D
:1034B000401C644909684871624800684079401CB2
:1034C000604909684871BBE000F028F9002811D173
:1034D0007F2008F00FFF5B4800684079401C594985
:1034E00009684871574800684079401C5549096887
:1034F00048711DE0534800684078401C51490968F4
:10350000487050480068407803280BD300204D498C
:1035100009684870AA204B49096888700320494906
:103520000968C87008F098FE00204649096848718B
:1035300086E000F0F3F8002807D14248006840799F
:10354000401C40490968487103E000203D49096872
:10355000487108F081FE73E008F054FE39480068B5
:103560004079401C37490968487169E03649496922
:103570000978491CC8B208F0BDFE3248006840799D
:10358000401C3049096848712E4800684079401C49
:103590002C490968487153E000F0C0F800280FD1A9
:1035A00008F002FE274909688870012008F076FEBD
:1035B000244800684079401C22490968487105E0A8
:1035C00008F04AFE00201F490968487138E01D488C
:1035D0000068807818280CD102201A490968087000
:1035E0000020184909684870042016490968C87005
:1035F00011E0144800684078401C1249096848707E
:10360000104800684078032805D300F027F900200F
:103610000C490968487008F01FFE00200949096834
:1036200048710DE008F018FE00200649096848714D
:10363000044909684870AA2002490968887000BFD7
:1036400000BF10BDCC070020102F002010B531485E
:1036500000684079002804D001280CD0032848D104
:103660001DE008F0CFFD2B4800684079401C294937
:10367000096848714BE028490969087808F03AFE62
:10368000244800684079401C224909684871214853
:1036900000684079401C1F490968487137E000F014
:1036A0003DF800280CD101201A4909680870002053
:1036B000184909684870042016490968C87011E063
:1036C000144800684078401C124909684870114845
:1036D00000684078032805D300F0C0F800200D49A9
:1036E0000968487008F0B8FD00200A490968487167
:1036F0000DE008F0B1FD0020064909684871054950
:1037000009684870AA2003490968887000BF00BF93
:1037100010BD0000CC070020102F002010B508F0CD
:103720003BFD04461F4800680078002838D01D483B
:103730000068C078042833D3002C09D1002119482F
:103740000068C07A8200174800681430815027E072
:1037500014480068C07A810012480068143040584C
:103760001149884211D20F480068C07A81000D4883
:10377000006814304058401C0A490968C97A8A0018
:1037800008490968143188500AE000F067F8002100
:1037900004480068C07A82000248006814308150F2
:1037A000204610BDCC070020B80B000000B587B044
:1037B00001206946087108480290084803900848AB
:1037C0000490084805900848069001A9074800F0B1
:1037D0000FF807B000BD0000153B0100595601006D
:1037E00085020200B9120200B8120200AC280020C3
:1037F000F8B506460F46002400253946304600F04D
:10380000EFF900BF14E000250EE000212420604302
:103810000B4A12688018415524206043094A1268F7
:1038200080184155681CC5B2242DEED3601CC4B26B
:1038300005480078A042E6DC00F010F8F8BD000072
:10384000C4070020C8070020102F002001200249D3
:103850000968087170470000CC07002010B500F01F
:1038600073F9002003490968087002490968C870A3
:1038700010BD0000CC07002007480068C07806286B
:1038800008D105480068C079002803D10120024909
:103890000968C87170470000CC07002010B5554872
:1038A0000068C07803000CF027FC08671D1A171485
:1038B000110E056650484068002803D04E48416804
:1038C0000020884793E000F0E5F890E000F0C6F8AB
:1038D0008DE000F0D1F88AE0FFF7B8FE87E0FFF74F
:1038E000C7FD84E044484068002803D0424841684E
:1038F000012088473F480068407C00281AD03E4895
:10390000C068002803D03C48C168C8208847002010
:10391000384909684862374800680078002804D0B0
:10392000042034490968C87024E00220314909683C
:10393000C8701FE02F480068406A401C2D49096884
:1039400048622C480068406A7D21C900884211D332
:103950000020284909684862264800680078002845
:1039600004D0042023490968C87003E002202149DB
:103970000968C8703BE000BF1F484068002803D0BA
:103980001D484168002088471A480068407C00288C
:1039900013D01948C068002803D01748C168C82050
:1039A0008847002013490968486212480068C078B7
:1039B000401C10490968C87018E00E480068406A49
:1039C000401C0C49096848620A480068406A7D2129
:1039D000C90088420AD300200649096848620548A0
:1039E0000068C078401C03490968C87000BF00BF68
:1039F00010BD0000CC070020102F002010B5154886
:103A00000068C078072824D001201249096848744A
:103A100008E011488068002802D00F498868804774
:103A2000FFF73CFF0B480068C0780628F1D1094831
:103A30000068007A0028ECD106480068C0790028A8
:103A4000E7D104480068807A0028E2D1014909687A
:103A5000487410BDCC070020102F002010B5054879
:103A600000680078012802D1FDF702FF01E0F5F7B8
:103A70003FFE10BDCC07002010B505480068007857
:103A8000012802D1FEF720F901E0F6F70FFA10BD88
:103A9000CC07002010B51D480068807A002829D185
:103AA0001A480068007A002803D0022017490968E4
:103AB000887216480068C079002803D00120134995
:103AC00009688872114800680079012812D1002025
:103AD0000E49096808710D490968887207200B4969
:103AE0000968C8700A484068002803D0084841683F
:103AF00000208847054800680078012802D1FEF7B9
:103B0000BDF901E0F6F7ACFA10BD0000CC070020CB
:103B1000102F002010B504462146084801F0C2FCD1
:103B200007480078002805D1002C03D03221054831
:103B3000FCF774FD0248047010BD00000103000092
:103B4000FE00002050C3000000202449096848708E
:103B5000AA20224909688870002020490968486223
:103B60001E49096808711D49096848711B4909689F
:103B700088711A490968C871184909680872174993
:103B80000968887215490968C87214490968087378
:103B900024201249096848731049096888730F493D
:103BA0000968C87300200D49096808740B49096841
:103BB00048740A490968887408490968C87407493B
:103BC0000968486100210548006881610348006870
:103BD000C16102480068016270470000CC07002004
:103BE00010B50A780D4B1860034628330C4C23603F
:103BF00024235343044628341B190A4C23600A4CDF
:103C00004B6863608B68A360CB68E3604B6963615A
:103C10000B6923610B78237010BD0000CC070020D6
:103C2000C4070020C8070020102F002007480068A4
:103C3000C078062808D105480068007A002803D11A
:103C4000012002490968087270470000CC07002073
:103C500010B50446012C09D1FF2220210020FFF7D6
:103C6000F5FB0121084604F025F908E00022202197
:103C70001046FFF7EBFB0021012004F01BF910BDFB
:103C800010B50024032000F00DFB002801D0012412
:103C900000E00024204610BD10B50446032C0ED1D0
:103CA000FF2215210020FFF7D1FB0022142110462E
:103CB000FFF7CCFB01210E2004F0FCF839E0022CC8
:103CC0001CD1FCF7E7FF002809D0FF2214210020B7
:103CD000FFF7BCFB01210E2004F0ECF808E0002205
:103CE00014211046FFF7B2FB00210E2004F0E2F889
:103CF000002215211046FFF7A9FB1AE0012C0ED176
:103D0000FF2214210020FFF7A1FB01210E2004F067
:103D1000D1F8002215211046FFF798FB09E0002298
:103D200015211046FFF792FB002214211046FFF7E1
:103D30008DFB10BD10B50024F8F716FE0949884226
:103D40000DD3FCF7FFFF002807D1FCF771FE012817
:103D500001DD032404E0022402E0022400E0012447
:103D6000204610BDB80B000010B50446012C09D147
:103D7000FF221D210020FFF769FB0121002004F034
:103D800099F808E000221D211046FFF75FFB002193
:103D9000084604F08FF810BD10B50024022000F092
:103DA00081FA002801D0012400E00024204610BD43
:103DB00010B50446012C09D1FF221E210020FFF777
:103DC00045FB0121092004F075F808E000221E21BE
:103DD0001046FFF73BFB0021092004F06BF810BDF3
:103DE00070B5002400250026FCF7DEFC0546FCF734
:103DF000E7FC064602210848F7F79EF9552800D14E
:103E000008E0012E01D1002404E0012D01D101249C
:103E100000E00024204670BD4C08002010B5044688
:103E2000012C09D1FF221F210020FFF70FFB0121E8
:103E3000082004F03FF808E000221F211046FFF799
:103E400005FB0021082004F035F810BD70B50024F2
:103E50000025FCF733FD054603211A48F7F76CF9F6
:103E6000552806D1012018490880002017490880EC
:103E700023E016480088012811D114490880FCF776
:103E800037FC762803DA01200F49088015E0FCF79B
:103E90002FFC782811DB00200B4908800DE0012061
:103EA0000A490880FCF724FC762803DA0120064939
:103EB000088002E000200449088003480488204666
:103EC00070BD00004C0800201A0100201C010020D9
:103ED00010B50446012C09D1FF2221210020FFF753
:103EE000B5FA0121072003F0E5FF08E000222121B7
:103EF0001046FFF7ABFA0021072003F0DBFF10BDEF
:103F000010B50024FCF7ACFD002801D1012400E02D
:103F10000024204610BD10B50446012C09D1FF2213
:103F200016210020FFF792FA0121032003F0C2FFBF
:103F300008E0002216211046FFF788FA002103202E
:103F400003F0B8FF10BD10B50024052000F0AAF959
:103F5000002801D0012400E00024204610BD10B547
:103F60000446012C09D1FF2219210020FFF76EFA27
:103F70000121052003F09EFF3CE0022C17D1FCF745
:103F800089FE002809D0FF2219210020FFF75EFAE0
:103F90000121052003F08EFF2CE00022192110469C
:103FA000FFF754FA0021052003F084FF22E0032CE0
:103FB00017D1FCF775FE002809D0FF221921002037
:103FC000FFF744FA0121052003F074FF12E00022FC
:103FD00019211046FFF73AFA0021052003F06AFF85
:103FE00008E0002219211046FFF730FA00210520D1
:103FF00003F060FF10BD000010B50024FCF764FD65
:1040000001282FD104211948F7F796F8552801D136
:10401000012428E0FCF7E0FB01280BD0FCF7DCFBD7
:10402000022807D0FCF7D8FB032803D0FCF7D4FB09
:10403000052801D1012416E0FCF7CEFB042801D1AC
:10404000022410E0FCF7C8FB062801D103240AE093
:10405000FCF7C2FB002803D0FCF7BEFB072802D107
:10406000002400E00024204610BD00004C08002081
:1040700010B50446012C0ED1FF221B210020FFF7B2
:10408000E5F900221A211046FFF7E0F901210A2084
:1040900003F010FF1EE0022C0ED1FF221A21002097
:1040A000FFF7D4F900221B211046FFF7CFF90121B9
:1040B0000A2003F0FFFE0DE000221A211046FFF750
:1040C000C5F900221B211046FFF7C0F900210A2084
:1040D00003F0F0FE10BD10B50024FCF7E7FD022848
:1040E00003D0FCF7D3FE022807D1FCF79DFE012880
:1040F00001D1012402E0022400E00224204610BD88
:1041000010B5F8F74BFC0446204610BD10B5034B24
:1041100008220349034800F013F910BD01410100D2
:10412000581202006C28002070B506465C48806872
:10413000002804D05A4988688047054600E00025D9
:104140000024A6E0564841680C20604308184088C7
:10415000A84207D0524841680C20604308184088A4
:1041600002287DD14E4841680C20604308188068C1
:1041700000280CD04A494A680C21614351188868CC
:10418000804747490968E2008918487009E04448B7
:1041900041680C206043095C41480068E2008018D7
:1041A00041703F480068E100401840783C49096888
:1041B000E200895C88420FD039480068E10040186D
:1041C000417837480068E20081540020344909688A
:1041D000E200891848605AE031480068E100401860
:1041E00041782F4842680C20604310184078814283
:1041F0001FD12B480068E1004018416828484268F8
:104200000C2060431018808881420BD82448006835
:10421000E10040184068801921490968E2008918C6
:10422000486034E001201E490968E200891848808E
:104230002DE01B480068E1004018416818484268BA
:104240000C2060431018C08881420DD814480068C3
:10425000E10040184068811911480068E20000E060
:1042600009E08018416012E000200D490968E20071
:10427000891848800BE0002009490968E200891884
:104280004880002106480068E20080184160601CF8
:1042900084B203488089A04200DD53E770BD00006E
:1042A000C82E00200146064A92898A4205DD044A4A
:1042B0001268CB00D218508800E000207047000040
:1042C000C82E0020002000BF14E00D494A680C21D0
:1042D00041435118498801290AD10021084A12682E
:1042E000C300D2185180064A1268C300D218516028
:1042F000411C88B2024989898142E6DC704700008E
:10430000C82E0020002000BF13E00C494A680C2191
:10431000414351184988002909D1084A1268C3004D
:10432000D2185180054A1268C300D2185160411C4E
:1043300088B2024989898142E7DC7047C82E002093
:10434000F0B504460020164DAB6069602C60AA8170
:1043500000BF1FE0124D6E680C254543755D104E81
:104360003668C700F61975700D4D6E680C2545430B
:10437000755D0B4E3668C700F5550025084E36684A
:10438000C700F6197580064E3668C700F6197560C5
:10439000451CA8B2024DAD898542DBDCF0BD0000B2
:1043A000C82E002070B505460E46002E05D03146B9
:1043B0002846F3F7C5FE044600E02C46204670BDB3
:1043C00010B5FCF74DFB00280DD1074800780128F7
:1043D00009D005480078032805D004480078002853
:1043E00001D1F8F7B7FF10BDF1000020F000002068
:1043F00008B500200090012269460520F9F722FE49
:104400000549009888600020044908700449087034
:104410000449087008BD000034280020F000002086
:10442000F2000020F300002008B5002000900122D7
:1044300069460520F9F706FE002002490871009838
:10444000886008BD3428002070B5049C257891420E
:1044500016DD01280AD18D4206DAFF26F61AAE4291
:104460000ED3EE18F5B20BE0154609E0022807D18D
:10447000954204DD9D4203DBEE1AF5B200E00D46E5
:10448000257070BD0D4A4168516081699161C168B4
:10449000D160416A5162016A11620168116041692B
:1044A000516181689160C169D16101691161816A5D
:1044B00091620021024A117070470000E42E002032
:1044C000C007002010B5FFF7FDFEF8F7ADF800219A
:1044D0000148F6F731FF10BD5808002010B5F8F775
:1044E000A3F8FFF70FFF09F0E7FD09F083FEFBF7E4
:1044F000DDFBFAF70FF9FFF77BFFF8F7CFFCF6F7D4
:1045000021FDF9F701FA55210448F6F715FFF8F7F0
:10451000FDFAF9F777F9FBF789F810BD5808002084
:104520001CB500203149087007F01CFE0020FCF784
:104530000DFD0CF009F9F7F7FDF955212C48F6F7B8
:10454000FBFEF8F7E3FAF9F75DF9F6F7F3F8F6F79B
:1045500071FBE12040020BF039FD00F069FAF6F73B
:10456000F1FC07F0DFFFF8F75FF8F9F719FFF8F74C
:1045700021FDF8F79FFCFFF7C9FDFEF783F8FFF771
:1045800015F9FFF73BFAF9F7FDFDFBF7BBFBFAF76F
:10459000C1F8184AFF219131012009F0F1FE0022F3
:1045A0001146012009F030FE09F06CFD09F022FEF1
:1045B000FFF73AFFF9F7D6F900200F4988714871E3
:1045C000087101208870487014200870072268461E
:1045D000F3F74DFE0199009800F0B4FF022101208D
:1045E00000F08CFEFBF722F81CBD0000FD0000204F
:1045F000580800200090D0030E01002070470000F2
:1046000010B50446552C03D105494869804702E09E
:1046100003490868804700200249087010BD000067
:10462000E42E0020C007002010B5464800780300A3
:104630000BF062FD0A06111B26303B465051738178
:1046400041484068002802D03F494868804701201F
:104650003C49087000BF3C488068002804D03A49B3
:10466000886880473749087069E03748C068002883
:1046700002D03549C868804703203249087000BF1E
:1046800031480069002804D02F49086980472D4926
:10469000087054E02C484069002802D02A49486933
:1046A000804700202749087049E027488069002892
:1046B00002D025498869804706202249087000BF3A
:1046C0002148C069002804D01F49C86980471D4996
:1046D000087034E000BF1B48007807280AD11A4848
:1046E000006A002802D01849086A80470920154945
:1046F000087011E01348007808280AD11248406A6F
:10470000002802D01049486A804709200D490870E6
:1047100002E000200B49087000BF0A48007800281A
:1047200008D00948806A002804D00749886A804771
:104730000449087003E000200249087000BF00BF70
:1047400010BD0000C0070020E42E002070470000CC
:1047500010B500200CF0B4F808F0BEFD08F012FE11
:1047600008F028FE00F0BEFCF6F7F4FA0220FCF791
:10477000EDFB002007490870FFF740F9FFF766F8E6
:10478000FFF78CF8F6F746F910200AF00FFA00F060
:10479000A9FD10BD9401002010B5012408F06AF9AC
:1047A000012801D1052407E0F8F7D8F80349884229
:1047B00001D2012400E00224204610BD204E00005A
:1047C00010B5062408F056F9002800D1002408F09E
:1047D00057F9012803D008F053F9072800D9092414
:1047E000204610BD10B5F6F7B5FA0022114601209B
:1047F00009F03CFE00213B48F6F79EFD002400BF77
:1048000000F02AFF32217D200001FBF707FF002086
:10481000354908700AE00022334801781046FEF757
:1048200015FE31480078401C2F4908702E4800784A
:104830002428F0DB00202D49087009E000212B48D6
:10484000007809F027FA29480078401C27490870A9
:10485000264800780D28F1DBFFF720F8F5F7B0FFC8
:1048600008F05AF822480078401C21490870084690
:104870000078052812D300200870FEF7FDFF1D48C0
:1048800000780A2805D300201A490870FFF7CEF9EE
:1048900004E018480078401C1649087008F0F0F849
:1048A0000128ADD908F0ECF80728A9D200200F495B
:1048B000087008E00D48007809F006FA0B48007807
:1048C000401C0A490870094800780D28F2DBF6F709
:1048D000B1F955210348F6F72FFDF8F715F82046F2
:1048E00010BD00005808002017010020150100200D
:1048F000160100201801002010B5032408E000F084
:10490000ABFE012000F0B2FD002801D0042400E03D
:10491000F5E700BF204610BD10B50020284908600B
:1049200007F020FC0120FCF711FBF7F703F85521F5
:104930002448F6F701FDF8F7E9F8F8F763FF0BF004
:1049400003FFF5F7F7FEF9F7F3FCF6F773F907F055
:10495000F3FFF9F725FDF9F7C1FEF8F72BFBFFF799
:10496000D5FBFDF78FFEFFF7CDFCFFF741FDFEF70E
:104970001DFFFFF743F800F05BF8E12040020BF069
:1049800025FBF6F7DFFAFBF7BDF9F9F7C3FE0E4A90
:10499000FF219131012009F0F3FC00221146012092
:1049A00009F032FC09F06EFB09F024FCF8F7ACFFCB
:1049B0000221012000F0A2FCFAF738FE10BD000031
:1049C00050000020580800200090D00370B5064623
:1049D0000D4614460E4806600E4805600E492068D4
:1049E00008600E49606808600D49A06808600D49BC
:1049F000206908600C49E06808600C49606908603B
:104A000005480068002802D003480068804770BD50
:104A1000C4000020CC000020AC000020B00000202A
:104A2000B4000020B8000020BC000020C00000201E
:104A300000B587B00C4801900C4802900C480390D8
:104A40000020049005900B48069000200A49086059
:104A500048600A490860486001AA0121C902084863
:104A6000FFF7B4FF07B000BD854A0100294E0100E1
:104A7000B14D0100DD4C010068120020600A0020E9
:104A80007017002001207047F3B5C3B00446449E60
:104A90000020009057E002E0641C761E00BF022E4A
:104AA00005D32078EB28F7D160789028F4D1072E31
:104AB00000D24AE0A778FD1CB54200D945E0A81E07
:104AC000205C0002691E615C08434290042D38D9C5
:104AD000291FA01C0BF052FE4299884226D11D4886
:104AE0000068002804D0B91EE01C1A4A12689047DA
:104AF00019480068002824D0E178684601712079BF
:104B000081116846417120798106890E684681715C
:104B1000381FC1B26846C171C279611D02A8F3F79E
:104B2000A6FB01A80C49096888470AE0002000900C
:104B300002E00098401C00900098A842F9D30020A1
:104B400000906419761B072EA5D200BF4498801BE5
:104B500045B0F0BDB8000020C0000020F7B5C0B0DF
:104B6000154600260027E81DFF210131884202DD9D
:104B7000002043B0F0BDEB216846017090214170E8
:104B8000281DC1B2684681700021C1704098C1B231
:104B9000684601710524002605E04198805D69465C
:104BA0000855641C761CAE42F7DBA11E00A802303B
:104BB0000BF0E4FD0746381269460855641C0F5592
:104BC000641C06480068002805D021466846034A50
:104BD00012689047CDE70020CBE70000B00000202E
:104BE00070B50024002500261B4840681A49096852
:104BF000884200D170BD184840681749096888424A
:104C000005D91548406814490968451A07E0124853
:104C1000006811494968401A012189020D1AFF2DC7
:104C200001D9FF2600E02E4600240DE00A48016865
:104C30000830405C0949085507480088401C800539
:104C4000800D05490860641CB442EFD3B1B203483B
:104C50000BF018FA00BFCDE7681200207016002094
:104C600070B500251A480068002830D0194A12880B
:104C7000FF230133991A184A1268164B1B88D01863
:104C8000134A126890470546002D20D0114800882D
:104C9000401910490880084601880F480068FFF74E
:104CA000F3FE0446002C0DDD0A480088844209DA30
:104CB00008480088021B0848006801190648006877
:104CC000F3F7D5FA03480088001B0249088070BD3D
:104CD000B4000020C8000020C400002038B50446FD
:104CE00000200090A07810280CD120792D49087060
:104CF00008460078012853D1002211462020FFF7F2
:104D00002DFF4DE0A078122803D1207925490872A3
:104D100046E0A078052803D12079224988723FE037
:104D2000A07802281DD120791E4948720846407A91
:104D3000012806D10090012269460420FFF70EFFEA
:104D40002EE01848407A02282AD100BFBFF34F8FC7
:104D500015481649C860BFF34F8F00BF00BF00BFA2
:104D6000FDE7A07801281BD12079332803D1012049
:104D70000C49487005E02079352802D10020094906
:104D80004870607907498870607A0006217A0904C2
:104D90000843E17909020843A179084301494860C1
:104DA00038BD0000540A00200400FA0500ED00E0C0
:104DB00070B503460022002400251A484068194EA9
:104DC0003668B04201D1002070BD16484068154ECB
:104DD0003668B04205D913484068124E3668841BC5
:104DE00007E0104800680F4E7668801B0126F60227
:104DF000341AA14201D9254600E00D4600220CE0FC
:104E0000084806680830805D985406480088401CB1
:104E10004005400D034E3060521CAA42F0D3284694
:104E2000D2E70000600A002070B50346002200248B
:104E300015484068144D2D68A84208D312484068B0
:104E4000114D2D68401B0125AD022C1A04E00E48BF
:104E500000680D4D6D68441BA14201D9012070BD51
:104E600000220CE09D5C08484668083085550838EB
:104E70008088401C8005800D034D6860521C8A426A
:104E8000F0D30020EBE700006812002010B50248C4
:104E9000FFF7F8FA10BD0000401302000021014A9C
:104EA0001175704740600040014600BFF020084087
:104EB00000110A23584302460807000F8018C0B2A9
:104EC00070470146002204E0501CC2B208460A386E
:104ED000C1B20A29F8DA1007000E08437047000033
:104EE00010B5044601218020F6F7B0FA607A012857
:104EF00005D14248C078102108434049C870607A03
:104F0000A22805D13E48007F802108433C4908770C
:104F1000607A3B49087700203A4948770846407F45
:104F20002178084337494877E07B002805D00846B8
:104F3000407F20210843334948773248407FC008EA
:104F4000C000A17A08432F4948770846807FF7219F
:104F500008402C498877E078FFF7B3FF2949887427
:104F6000A078FFF7AEFF2749C8746078FFF7A9FF64
:104F7000244908752078002805D10846007D21794C
:104F8000084320490875E079FFF79BFF1D498875A4
:104F90006079FFF796FF1B494875A079FFF791FFED
:104FA0001849C875207AFFF78CFF1649087608461D
:104FB000807F4006400E8877E07A002806D00846B9
:104FC000807F402108430F49887703E00D48807FA8
:104FD0000C498877A07BFFF774FF0A498876607BCD
:104FE000FFF76FFF0749C876207B08770846807F68
:104FF000102188430349887710BD00002004024037
:1050000060040440404F044010B504461B48807FB4
:1050100001210843194988772078FFF752FF174983
:1050200008756078FFF74DFF1449C874A078FFF742
:1050300048FF1249887420780C2806DD0846407F16
:10504000082108430D49487709E00C48407F0B4987
:1050500048770846007DE178084308490875074805
:10506000807F400840000549887700BF0348807F63
:10507000022108400028F9D110BD0000404F044033
:1050800010B500201449087616200BF05BF80021BB
:10509000124801761248407F802108431049487722
:1050A0000846807F012108430D49887700BF0C48DE
:1050B000807F022108400028F9D00948807F4008FD
:1050C00040000749887700BF0548807F02210840DB
:1050D0000028F9D110BD0000406000404061004050
:1050E000404F044010B500200749087000212020DF
:1050F000F6F7ACF90121054801750020044908754F
:1051000015200BF007F810BD00500440406100402E
:105110004060004070B504460D46002C14D0002DB0
:1051200012D0042D10D800F013F800280CD100265E
:1051300008E00649885D22460121F4F717F9A41C0E
:10514000701CC6B2AE42F4DB70BD0000BC1202009F
:1051500000200549897DC907C90F002901D0012018
:1051600000E00020704700000050044030B585B0DA
:1051700005460C4600200390049000900190029098
:10518000072C0BDC0120A04081B2684681810121FF
:10519000C17303A90220FAF7F5FE3EE0082C01D006
:1051A000092C0BD10120A04081B2684681810121E8
:1051B000C17303A90120FAF7E5FE2EE00A2C03D003
:1051C0000B2C01D00D2C0BD10120A04081B26846E0
:1051D00081810121C17303A90020FAF7D3FE1CE0ED
:1051E0000C2C01D00F2C0BD10120A04081B26846BD
:1051F00081810121C17303A90E20FAF7C3FE0CE0DF
:105200000E2C0AD10120A04081B268468181012183
:10521000C17303A90C20FAF7B5FE0021684601709E
:10522000C17041700121817000210171C1720D2195
:105230008172FF21017200214172F4F7F7F80349EE
:105240001520FDF7E9F805B030BD00009D4E0100C6
:1052500010B500201049087515200AF05BFF0021E9
:105260000E4801751520002809DB00BF00BFC206EB
:10527000D20E012191400A4A116000BF00BF00BF59
:10528000084880798011032805D0064800788021DD
:1052900008430449087010BD406000404061004070
:1052A00000E100E00050044010B5F4F7B9F910BD7A
:1052B00010B501231A4600211846F6F783F801229B
:1052C00011461046F6F7F4F8F6F7E0F803480BF04D
:1052D0002DFA02480249086010BD00000090D0037A
:1052E0004407002000BF0448006904210843024924
:1052F000086130BF00BF704700ED00E0F3B585B036
:105300000546002400270026002003900490EEB2FA
:105310002804070E0F2F54DA082E52DA002009E075
:105320000C214143284A515AA94201D1044603E0C5
:10533000411CC8B21728F3D300BF0120B04086B289
:105340000C20604320494018C3780C20604340186B
:105350008278F8B231460190FAF7B8FE6846868145
:10536000012181730021C17302214174F8B203A9A4
:10537000FAF708FE0C216143134A8918C888FBF725
:105380000BFF0C20604310494018C188684601811A
:1053900069460698887202A8FBF718FE0C22624341
:1053A000094BD21891680C226243D218042010567F
:1053B000FDF732F80C216143034A8918C888FBF7CE
:1053C0006FFE07B0F0BD0000D8140200FEB5054620
:1053D0000C460020C0430290EFB22804060E0F2EA8
:1053E00042DA082F40DA0120B84069460880802060
:1053F0002040002816D101208870A007800F0228C5
:1054000001D1487109E0A007800F012802D1694647
:10541000487102E0002069464871F0B26946FAF727
:10542000B1FD1FE00020694688700E202040002852
:1054300000D000BF10202040002802D1694608712A
:1054400002E0012069460871E007C00F002802D180
:105450006946887102E0012069468871F0B26946A8
:10546000FAF790FD002002900298FEBD30B501468B
:10547000CAB20C04230E00200F2B0FDA082A0DDA13
:1054800001249440A2B2064C03252D026419E45C69
:105490001440002C01D0012000E0002030BD0000AD
:1054A00000000440F8B504460F460020C0430090B9
:1054B000E6B22004050E0F2D11DA082E0FDA0120B6
:1054C000B04086B2002F04D1E8B23146FAF756FE5A
:1054D00003E0E8B23146FAF761FE00200090009840
:1054E000F8BD00001649897F01221143144A9177C3
:1054F00000BF1349897F022211400029F9D01049C9
:10550000897C81700E49C97C41700D49097D01700B
:105510000B498A7D8271497D01710949CA7D4271B9
:105520000A7EC271897F49084900054A917700BF08
:105530000349897F022211400029F9D170470000F8
:10554000404F044003B585B00020019002900390C5
:105550000490002168464173817E01A8C1706846AD
:10556000417E01A881706846017E4171002101A839
:105570000171082168460171817D01A8C1716846E9
:10558000C17D4172417D01A881716846017D01A8FC
:105590000172002168468173C17301A881730C21D7
:1055A00041734121684601740021C17401A8FFF7CD
:1055B00097FC1A200449888204491620FCF72CFF26
:1055C00000F006F807B000BD204F04407908020043
:1055D00010B5FFF755FD10BD70B504460D46601EB1
:1055E0000D49884200D90124002C00D1012440201B
:1055F0000A49087008460078604309494861032158
:10560000081F0AF0B7FD00200549886107200861DE
:105610000448056070BD0000FFFFFF00700100201E
:1056200000E000E06C0100200020C043002809DBFE
:10563000C206D20E01219140054A1160BFF34F8F7F
:10564000BFF36F8F00BF0020024908618861704777
:1056500080E100E000E000E010B50AF031FD10BD8F
:105660001A20084908722B2048723C2088724D206D
:10567000C8727F20044909680860AC20034948705B
:105680007047000000040240740100200010024036
:1056900010B51C480078012812D11B4800786428F6
:1056A00009DB022019494871087100201649087069
:1056B0001449087004E014480078401C124908702E
:1056C0001348007801281CD112480078012804D121
:1056D000002010490870104908700F4800783228DF
:1056E0000ADBF7F75BFA00210C48F5F7DFFD5521DF
:1056F0000B48F5F721FE04E007480078401C0649F6
:10570000087010BD110700201007002000070020BE
:105710000A0700200C0700200B0700204C0800207F
:1057200058080020F8B504460D46002700200090D8
:1057300003200003204000130090102C04D0122CF2
:1057400002D01148844217D122202840222806D1B5
:1057500027073F0F39460098F4F7D8FF0646122076
:10576000284012280ED12007000F471C3946009808
:10577000F4F7CCFF064605E02107090F0098F4F77F
:10578000C5FF06463046F8BD10100000F8B50446C7
:105790000D46002600270120000320400713102C8F
:1057A00004D0122C02D00F48844215D12220284068
:1057B000222805D12607360F31463846FAF7DAF89F
:1057C0001220284012280CD12007000F461C314619
:1057D0003846FAF7CFF804E02107090F3846FAF700
:1057E000C9F8F8BD10100000FFB58BB01C460020B2
:1057F0000790069005903848049010210B980840B7
:10580000002801D0022707E040210B98084000281B
:1058100001D0012700E00027002C04D01498047068
:105820000120089001E010200890002548E0002C9D
:1058300008D025466000294A115A0C98F2F780FCDE
:10584000079006E06800254A115A0C98F2F778FC98
:1058500007903E4630E0711C0798F2F771FC400853
:1058600006900D98F2F7C2FD03900D9A0699881ADA
:10587000F2F7BCFD18490190F2F73DFD0290039943
:10588000F2F776FD05900598F2F7B7FD4900490853
:10589000039102900498F2F7B0FD49004908019184
:1058A0000090039B029AF2F7BDFD03D20A95099678
:1058B00005980490701CC6B27F2ECCDD681CC5B262
:1058C00008988542B3DB14990A98087014990998CE
:1058D000487004980FB0F0BD0000C842EC150200FB
:1058E0000246412A2ED010DC212A2AD006DC102ABA
:1058F00045D0122A4BD0202A59D11CE0222A26D08A
:10590000232A2AD0402A52D116E081235B01D01AE3
:105910009A4228D008DC422A1AD0432A1ED02548B1
:105920001018002843D13AE0012822D020281BD0AB
:1059300021283CD11EE000BF1F4803890B4303818F
:1059400036E000BF1C4843890B43438130E000BF71
:10595000194883890B4383812AE000BF1648C38915
:105960000B43C38124E000BF144883880B4383802A
:105970001EE000BF1148C3880B43C38018E00E48E7
:1059800043890B43438103890B43038110E00A4899
:10599000C3890B43C38183890B43838108E0074894
:1059A000C3880B43C38083880B43838000E000BF20
:1059B00000BF7047F0EFFFFF0011044000140440E7
:1059C000F0B505460E46412D30D010DC212D2CD0EF
:1059D00006DC102D51D0122D56D0202D62D11CE0A6
:1059E000222D2AD0232D30D0402D5BD116E08121ED
:1059F0004901681A8D4230D008DC422D1ED0432D5B
:105A000024D02A48281800284CD144E001282CD062
:105A1000202823D0212845D128E000BF244F3888F2
:105A2000314600F049F804463DE000BF204F788839
:105A3000314600F041F8044635E000BF1C4FB888FD
:105A4000314600F039F804462DE000BF184FF888C1
:105A5000314600F031F8044625E000BF154F388884
:105A6000314600F029F804461DE000BF114F788848
:105A7000314600F021F8044615E00D4F7888314694
:105A800000F01AF804460EE0094FF888314600F09D
:105A900013F8044607E0074F7888314600F00CF809
:105AA000044600E000BF00BF2046F0BDF0EFFFFF5E
:105AB00000110440001404400246002013460B402D
:105AC000002B01D0012000E000207047FFB581B01D
:105AD0000E461746012F07D1F748407D0009000107
:105AE000C01DF549487505E0F348407D00090001F7
:105AF000F1494875049801287ED10A210198F2F7EE
:105B00001FFB0546ED48445DE007C00F002807D0A5
:105B1000E948007C00090001C01DE749087405E060
:105B2000E548007C00090001E34908740220204098
:105B3000002807D0E048C07BF02188437030DE4960
:105B4000C87305E0DC48C07BF0218843DA49C8739C
:105B500004202040002807D0D748807C000900019D
:105B6000C01DD549887405E0D348807C0009000138
:105B7000D149887408202040002807D0CE48407CB6
:105B8000F02188437030CC49487405E0CA48407C15
:105B9000F0218843C849487410202040002807D0CD
:105BA000C548407C00090001C01DC349487405E098
:105BB000C148407C00090001BF49487420202040B2
:105BC000002807D0BC48007CF02188437030BA49D7
:105BD000087405E0B848007CF0218843B649087491
:105BE00040202040002808D0B348807CF021884322
:105BF0007030B149887406E08BE0AF48807CF021BA
:105C00008843AD4988740A210198F2F799FA0D4644
:105C1000AA48445DE007C00F002807D0A648807B53
:105C2000F02188437030A449887305E0A248807B46
:105C3000F0218843A049887302202040002807D023
:105C40009D48807B00090001C01D9B49887305E0C9
:105C50009948807B000900019749887304202040FF
:105C6000002807D09448007DF02188437030924985
:105C7000087505E09048007DF02188438E4908753D
:105C800008202040002807D08B48007D0009000133
:105C9000C01D8949087505E08748007D000900019D
:105CA0008549087510202040002807D08248C07C14
:105CB000F021884370308049C87405E07E48C07C7C
:105CC000F02188437C49C87420202040002807D058
:105CD0007948C07B00090001C01D7749C87305E001
:105CE0007548C07B000900017349C87340202040FB
:105CF000002807D07048C07C00090001C01D6E4913
:105D0000C87454E06C48C07C000900016A49C8743A
:105D10004DE06948007C00090001674908740846A5
:105D2000C07BF02188436449C8730846807C000921
:105D3000000188740846407CF02188435E4948741D
:105D40000846407C0009000148740846007CF021A8
:105D50008843594908740846807CF0218843564995
:105D600088740846807BF02188435349887308462D
:105D7000807B0009000188730846007DF02188437C
:105D80004D4908750846007D000900010875084660
:105D9000C07CF02188434849C8740846C07B00098C
:105DA0000001C8730846C07C00090001C8740A9845
:105DB00001287DD10A213046F2F7C2F905463F4855
:105DC000445DE007C00F002807D03B48407B000936
:105DD0000001C01D3849487305E03748407B000981
:105DE00000013549487302202040002807D032487E
:105DF000007BF021884370302F49087305E02E485E
:105E0000007BF02188432C4908730420204000289F
:105E100007D02948807DF021884370302649887555
:105E200005E02548807DF0218843234988750820B6
:105E30002040002807D02048807D00090001C01DB7
:105E40001D49887505E01C48807D000900011A493C
:105E5000887510202040002807D01748407DF02189
:105E6000884370301449487505E01348407DF0219F
:105E700088431149487520202040002807D00E484B
:105E8000407BF021884370300B49487305E00A4895
:105E9000407BF02188430849487340202040002877
:105EA0000ED00548C07D00090001C01D024900E078
:105EB00092E0C8750AE00000442600202C10020081
:105EC0006D48C07D000900016B49C8750A21304644
:105ED000F2F736F90D466948445DE007C00F002827
:105EE00007D06548C07AF021884370306249C87293
:105EF00005E06148C07AF02188435F49C8720220FA
:105F00002040002807D05C48C07A00090001C01D6D
:105F10005949C87205E05848C07A0009000156493D
:105F2000C87204202040002807D05348407E000952
:105F30000001C01D5049487605E04F48407E0009E9
:105F400000014D49487608202040002807D04A48E3
:105F5000007EF021884370304749087605E04648C6
:105F6000007EF02188434449087610202040002814
:105F700007D04148007E00090001C01D3E49087657
:105F800005E03D48007E000900013B4908762020DD
:105F90002040002807D03848007B00090001C01DC0
:105FA0003549087305E03448007B00090001324997
:105FB000087340202040002807D02F48C07DF021E2
:105FC000884370302C49C87554E02B48C07DF021BF
:105FD00088432949C8754DE02748407B00090001E6
:105FE000254948730846007BF021884322490873FD
:105FF0000846807DF02188431F4988750846807DCA
:106000000009000188750846407DF02188431A493F
:1060100048750846407BF021884317494873084675
:10602000C07D00090001C8750846C07AF021884388
:106030001149C8720846C07A00090001C8720846B2
:10604000407E0009000148760846007EF021884322
:10605000094908760846007E0009000108760846CE
:10606000007B0009000108730846C07DF0218843C9
:106070000149C87505B0F0BD442600202C1002006F
:10608000FFB581B00E461746019801287ED10498CD
:10609000002828D1FB480078012824D0F6F764FCBA
:1060A000F94988421FD3FAF7F5FD00280DD0F748CB
:1060B000807DF02188437030F44988750846C07CA3
:1060C00000090001C01DC8741AE0F048807DF0216D
:1060D00088431030ED4988750846C07C00090001EE
:1060E000401CC8740CE0E948807DF0218843703082
:1060F000E64988750846C07C00090001C01DC874C7
:10610000E248C07CF02188437030E049C8740846FA
:10611000007EF02188437030DC4908760846807D97
:1061200000090001401C88750846407DF021884325
:106130001030D64948750846407D00090001401CD2
:1061400048750846007DF02188431030CF49087516
:106150000846007D00090001401C0875330009F065
:10616000CBFF062E261E140C042FC848007D000904
:106170000001C01DC549087500BFC448007DF0215D
:1061800088437030C149087500BF00E0AFE1BF48E7
:10619000407D00090001C01DBC49487500BFBB48D7
:1061A000407DF02188437030B849487500BFB7483A
:1061B000807D00090001C01DB449887500BF00E062
:1061C00000BF00BF049800285ED1AE4800780128C7
:1061D0005AD0F6F7C9FBAC49884255D3AB48C07FCB
:1061E000F0218843A949C8770846807F000900014B
:1061F00088770846407FF0218843A44948770846BD
:10620000007FF0218843A14908770846C07DF0212E
:1062100088439E49C8750846C07F00090001C877B9
:106220000846807FF0218843984988770846407F58
:1062300000090001C01D48770846807EF021884390
:10624000924988760846807E0009000188760846D3
:10625000407E0009000148760846007E00090001E2
:1062600008760846007F0009000108770846C07ECE
:10627000F02188438549C8760846407EF02188434E
:10628000703082494876B8E164213846F1F758FF0A
:106290000546012D07D17D48C07FF021884370302D
:1062A0007A49C87705E07948C07FF021884377496B
:1062B000C8770A213846F1F743FF0A210090F1F729
:1062C0003FFF0D46642F02D37148445D01E07148E1
:1062D000445DE007C00F002807D06C48807F0009AC
:1062E0000001C01D6949887705E06848807F000982
:1062F00000016649887702202040002807D06348C3
:10630000407FF021884370306049487705E05F485E
:10631000407FF02188435D494877042020400028D1
:1063200007D05A48007FF0218843703057490877DA
:1063300005E05648007FF02188435449087708203B
:106340002040002807D05148C07DF021884370309C
:106350004E49C87505E04D48C07DF02188434B4942
:10636000C87510202040002807D04848C07F000989
:106370000001C01D4549C87705E04448C07F0009B9
:1063800000014249C87720202040002807D03F481C
:10639000807FF021884370303C49887705E03B4896
:1063A000807FF021884339498877402020400028A9
:1063B00007D03648407F00090001C01D33494877A7
:1063C00005E03248407F00090001304948770A2142
:1063D0003846F1F7B5FE0D462D48445DE007C00F85
:1063E000002807D02948807EF02188437030274953
:1063F000887605E02548807EF02188432349887609
:1064000002202040002807D02048807E000900019B
:10641000C01D1E49887605E01C48807E00090001E9
:106420001A49887604202040002807D01748407E6B
:1064300000090001C01D1549487605E01348407E5B
:10644000000900011149487608202040002807D0A3
:106450000E48007E00090001C01D0C49087605E0C9
:106460000A48007E000900010849087610202040F3
:10647000002811D00548007F00090001C01D034914
:1064800008770FE0FD000020B80B0000182700205F
:106490002C1002003F1002005948007F0009000143
:1064A0005749087720202040002807D05448C07E54
:1064B000F021884370305249C87605E05048C07ECC
:1064C000F02188434E49C87640202040002807D05C
:1064D0004B48407EF02188437030494948768CE033
:1064E0004748407EF02188434549487685E0444846
:1064F000807D00090001424988750846407DF021F1
:1065000088433F4948750846407D000900014875A9
:106510000846007DF0218843394908750846007D0A
:106520000009000108750846C07C00090001C87414
:106530000846807DF0218843314988750846C07C33
:10654000F02188432E49C8740846007EF021884314
:106550002B4908760846C07FF02188432849C87730
:106560000846807F0009000188770846407FF021B7
:106570008843234948770846007FF0218843204913
:1065800008770846C07DF02188431D49C875084634
:10659000C07F00090001C8770846807FF02188434A
:1065A000174988770846407F000900014877084668
:1065B000807EF0218843124988760846807E000953
:1065C000000188760846407E0009000148760846AA
:1065D000007E0009000108760846007F00090001DE
:1065E00008770846C07EF02188430549C8760846EA
:1065F000407EF02188430249487605B0F0BD000096
:106600001827002010B50146002200200A0EFE4B7C
:10661000985CC307DB0F002B07D0FC4BDB7FF0241B
:10662000A3437033F94CE37705E0F84BDB7FF024AC
:10663000A343F64CE37702230340002B07D0F34B30
:10664000DB7F1B091B01DB1DF04CE37705E0EF4B03
:10665000DB7F1B091B01ED4CE37704230340002B78
:1066600007D0EA4B9B7F1B091B01DB1DE74CA3777F
:1066700005E0E64B9B7F1B091B01E44CA377082335
:106680000340002B09D0E14B20335B781B091B0131
:10669000DB1DDE4C2034637007E0DC4B20335B787D
:1066A0001B091B01D94C2034637010230340002BBD
:1066B00009D0D64B20331B78F024A3437033D34C3E
:1066C0002034237007E0D14B20331B78F024A34300
:1066D000CE4C2034237020230340002B09D0CB4B19
:1066E00020331B781B091B01DB1DC84C2034237091
:1066F00007E0C64B20331B781B091B01C34C203419
:10670000237040230340002B07D0C04B9B7FF02415
:10671000A3437033BD4CA37705E0BC4B9B7FF024B3
:10672000A343BA4CA377FF231B040B401A0CB64BB0
:10673000985CC307DB0F002B07D0B44B1B7F1B09F2
:106740001B01DB1DB14C237705E0B04B1B7F1B0900
:106750001B01AE4C237702230340002B07D0AB4B29
:10676000DB7EF024A3437033A84CE37605E0A74B0F
:10677000DB7EF024A343A54CE37604230340002BE7
:1067800007D0A24B9B7EF024A34370339F4CA3768B
:1067900005E09E4B9B7EF024A3439C4CA3760823EC
:1067A0000340002B07D0994B5B7FF024A343703349
:1067B000964C637705E0954B5B7FF024A343934CA5
:1067C000637710230340002B07D0904B5B7F1B099E
:1067D0001B01DB1D8D4C637705E08C4B5B7F1B0938
:1067E0001B018A4C637720230340002B07D0874B83
:1067F0001B7FF024A3437033844C237705E0834B45
:106800001B7FF024A343814C237740230340002BBC
:1068100007D07E4BDB7E1B091B01DB1D7B4CE37627
:1068200005E07A4BDB7E1B091B01784CE376FF23E6
:106830001B020B401A0A744B985CC307DB0F002B3A
:1068400007D0724B1B7EF024A34370336F4C23762A
:1068500005E06E4B1B7EF024A3436C4C2376022391
:106860000340002B07D0694B1B7E1B091B01DB1D5E
:10687000664C237605E0654B1B7E1B091B01634CB0
:10688000237604230340002B07D0604BDB7D1B09DC
:106890001B01DB1D5D4CE37505E05C4BDB7D1B09DB
:1068A0001B015A4CE37508230340002B07D0574BBC
:1068B0009B7E1B091B01DB1D544CA37605E0534B4B
:1068C0009B7E1B091B01514CA37610230340002B18
:1068D00007D04E4B5B7EF024A34370334B4C637662
:1068E00005E04A4B5B7EF024A343484C63762023AB
:1068F0000340002B07D0454B5B7E1B091B01DB1DB2
:10690000424C637605E0414B5B7E1B091B013F4C0B
:10691000637640230340002B07D03C4BDB7DF02403
:10692000A3437033394CE37505E0384BDB7DF0242D
:10693000A343364CE375CAB2334B985CC307DB0FF5
:10694000002B07D0314B1B7DF024A34370332F4C19
:10695000237505E02D4B1B7DF024A3432B4C2375A1
:1069600002230340002B07D0284B1B7D1B091B0172
:10697000DB1D264C237505E0244B1B7D1B091B01E9
:10698000224C237504230340002B07D01F4BDB7CD4
:106990001B091B01DB1D1D4CE37405E01B4BDB7C5D
:1069A0001B091B01194CE37408230340002B07D07B
:1069B000164B9B7CF024A3437033144CA37405E066
:1069C000124B9B7CF024A343104CA3741023034070
:1069D000002B07D00D4B5B7DF024A34370330B4C91
:1069E000637505E0094B5B7DF024A343074C637599
:1069F00020230340002B0BD0044B5B7D1B091B01A4
:106A0000DB1D024C637509E02C100200F826002003
:106A10000C4B5B7D1B091B010A4C63754023034033
:106A2000002B07D0074BDB7CF024A3437033054CCD
:106A3000E37405E0034BDB7CF024A343014CE374D7
:106A400010BD0000F826002000B501287ED1FE4AC6
:106A5000D278F0239A437032FB4BDA701A461279DF
:106A600012091201D21D1A711A461279F0239A43A3
:106A70007032F54B1A711A46527912091201D21D61
:106A80005A711A465279F0239A437032EE4B5A717A
:106A90001A46D27912091201D21DDA711A46D27938
:106AA000F0239A437032E84BDA711A46527A12098F
:106AB0001201D21D5A721A46527AF0239A4370324A
:106AC000E14B5A721A46927AF0239A437032DE4BA7
:106AD0009A721A469278F0239A437032DA4B9A707F
:106AE0001A46D27A12091201D21DDA721A46527867
:106AF00012091201D21D5A701A46D27AF0239A4313
:106B00007032D14BDA721A46203AD27FF0239A4380
:106B10007032CD4B203BDA77CB4A127B120912013F
:106B2000D21D20331A731A46203A927F120912019D
:106B3000D21D203B9A77C44A127BF0239A437032CD
:106B4000C14B1A731A46203A127F00E0F2E1F0239B
:106B50009A437032BC4B203B1A77BB4A527B1209D6
:106B60001201D21D20335A731A46203AD27E1209DE
:106B70001201D21D203BDA76B44AD278F0239A4330
:106B80007032B24BDA701A46127B12091201D21D12
:106B90001A731A46127912091201D21D1A711A4675
:106BA000927AF0239A437032A84B9A721A4612795D
:106BB000F0239A437032A54B1A711A465279120982
:106BC0001201D21D5A711A46927912091201D21D70
:106BD0009A711A46127A12091201D21D1A721A46B5
:106BE000127AF0239A437032984B1A721A46527AEC
:106BF00012091201D21D5A72934A92791209120196
:106C0000521C914B9A711A469279F0239A43103292
:106C10008D4B9A711A46127A12091201521C1A727D
:106C20001A46127AF0239A431032874B1A721A4688
:106C3000927A12091201521C9A721A46D2781209DB
:106C40001201521CDA701A46927812091201521C73
:106C50009A701A465278F0239A4310327A4B5A703F
:106C60001A461278F0239A431032774B1A701A465C
:106C7000127812091201521C1A701A46203AD27F59
:106C800012091201521C203BDA771A46927FF02338
:106C90009A4310326C4B203B9A771A46527FF0236E
:106CA0009A431032684B203B5A771A46527F12099A
:106CB0001201521C5A771A46127F12091201521CF5
:106CC0001A771A46D27EF0239A4310325E4B203B4D
:106CD000DA761A46927EF0239A4310325A4B203BC2
:106CE0009A765A4A127BF0239A431032574B1A7302
:106CF0001A46D27AF0239A431032544BDA721A466B
:106D0000D27A12091201521CDA721A46927A1209C8
:106D10001201521C9A721A46527AF0239A43103288
:106D20004A4B5A721A465279F0239A431032474B13
:106D30005A711A46D279F0239A431032434BDA71D2
:106D40000B0009F0D9F919F3E9DFD5CBC1B7ADA331
:106D5000998F87786E645A50463E362E261E160E40
:106D6000F5003A4AD279F0239A437032374BDA7100
:106D700000BF364A5279F0239A437032334B5A712E
:106D800000BF324A527AF0239A4370322F4B5A7224
:106D900000BF2E4A927A12091201D21D2B4B9A7211
:106DA00000BF2A4AD27A12091201D21D274BDA7289
:106DB00000BF264AD27AF0239A437032234BDA720C
:106DC00000BF224A127BF0239A4370321F4B1A7382
:106DD00000BF1D4A203A927EF0239A4370321A4B2C
:106DE000203B9A7600BF184A203AD27EF0239A437D
:106DF0007032154B203BDA7600BF134A203A127FDF
:106E000012091201D21D104B203B1A7700BF0E4A07
:106E1000203A527F12091201D21D0B4B203B5A77A8
:106E200000BF094A203A527FF0239A437032064B42
:106E3000203B5A7700BF044A203A927FF0239A43BE
:106E40007032014B203B03E06426002038270020ED
:106E50009A7700BFDC4AD27F12091201D21DDA4BA9
:106E6000DA7700BFD84A2032127812091201D21DF7
:106E7000D54B20331A7000BFD34A20321278F0234A
:106E80009A437032D04B20331A7000BFCE4A203262
:106E90005278F0239A437032CB4B20335A7000BFA4
:106EA000C94A2032927812091201D21DC64B2033F2
:106EB0009A7000BFC44A2032D27812091201D21D42
:106EC000C14B2033DA7000BFBF4A2032927A1209D8
:106ED0001201D21DBC4B20339A7200BFBA4A203235
:106EE000127AF0239A437032B74B20331A7200BFE4
:106EF000B54A2032127A12091201D21DB24B203348
:106F00001A7200BFB04A20329279F0239A4370324D
:106F1000AD4B20339A7100BFAB4A203292791209EF
:106F20001201D21DA84B20339A7100BF01E0FFE788
:106F300000BF47E1A44A2032D278F0239A43A24B03
:106F40002033DA701A461279120912011A711A46A0
:106F50001279F0239A439C4B20331A711A465279C6
:106F6000120912015A711A465279F0239A43964B2C
:106F700020335A711A46D27912091201DA711A466F
:106F8000D279F0239A43904B2033DA711A46527A21
:106F9000120912015A721A46527AF0239A438A4B06
:106FA00020335A721A46927AF0239A43864B203342
:106FB0009A721A469278F0239A43834B20339A7040
:106FC0001A46D27A12091201DA721A465278120956
:106FD00012015A701A46D27AF0239A437A4B203320
:106FE000DA72794AD27FF0239A43774BDA771A46DE
:106FF0002032127B1209120120331A73724A927FD7
:1070000012091201203B9A771A462032127BF02394
:107010009A436D4B20331A736B4A127FF0239A43C5
:10702000694B1A771A462032527B1209120120331B
:107030005A73654AD27E12091201203BDA76634AFE
:10704000D278F0239A43614BDA701A46127B120908
:1070500012011A731A461279120912011A711A468C
:10706000927AF0239A43594B9A721A461279F02376
:107070009A43564B1A711A465279120912015A71E3
:107080001A469279120912019A711A46127A120955
:1070900012011A721A46127AF0239A434B4B1A7253
:1070A0001A46527A120912015A72474A20329279CC
:1070B00012091201444B20339A711A469279F02337
:1070C0009A43414B20339A711A46127A12091201DF
:1070D0001A721A46127AF0239A433B4B20331A72E3
:1070E0001A46927A120912019A721A46D278120935
:1070F0001201DA701A469278120912019A701A4631
:107100005278F0239A43304B20335A701A46127843
:10711000F0239A432C4B20331A701A461278120926
:1071200012011A70284AD27F12091201203BDA7725
:107130001A46927FF0239A43234B9A771A46527F3E
:10714000F0239A43204B5A771A46527F12091201B4
:107150005A771A46127F120912011A771A46D27EFE
:10716000F0239A43184BDA761A46927EF0239A431C
:10717000154B9A76154A127BF0239A43134B1A73D8
:107180001A46D27AF0239A43104BDA721A46D27A10
:1071900012091201DA721A46927A120912019A72CF
:1071A0001A46527AF0239A43084B5A721A46527979
:1071B000F0239A43054B5A711A46D279F0239A4329
:1071C000024BDA7100BD0000442600203827002061
:1071D000F7B582B006461746002500200190002E24
:1071E0007ED1F9F737FC05285FD1F9F753FD002868
:1071F0000DD0FA484079F02188437030F749487142
:107200000846807800090001C01D88700AE0F34834
:107210004079F0218843F149487108468078000997
:1072200000018870ED48C07900090001EB49C87180
:1072300008468079000900018871084640790009F4
:10724000000148710846007AF0218843E34908723A
:107250000846007A0009000108720846C079F0214A
:107260008843DE49C8710846C07800090001C8702B
:1072700008468078F0218843D849887008464078CD
:10728000F0218843D549487008464078000900013C
:107290004870084600790009000108710846C07866
:1072A000F0218843CD49C87029E2CC484079F021CB
:1072B00088437030C9494871084680780009000148
:1072C000C01D88700846C07900090001C8710846D1
:1072D000807900090001887108464079000900E0C2
:1072E00034E0000148710846007AF0218843BB4928
:1072F00008720846007A0009000108720846C07941
:10730000F0218843B549C8710846C07800090001DA
:10731000C87008468078F0218843B04988700846D4
:107320004078F0218843AD4948700846407800090C
:1073300000014870084600790009000108710846FC
:10734000C078F0218843A549C870ADE7012E5FD110
:10735000F9F7A0FC00280DD0A0484079F02188431F
:1073600070309E4948710846807800090001C01DB0
:1073700088700AE099484079F0218843974948711C
:10738000084680780009000188709448C079000997
:1073900000019249C871084680790009000188718E
:1073A000084640790009000148710846007AF0213A
:1073B00088438A4908720846007A00090001087269
:1073C0000846C079F02188438449C8710846C078CE
:1073D00000090001C87008468078F02188437F4981
:1073E000887008464078F02188437C4948700846F8
:1073F0004078000900014870084600790009000142
:1074000008710846C078F02188437449C870DAE3EF
:10741000022E7DD1F9F71EFB05287AD1F9F73AFC47
:10742000002877D0012F76D10A210398F0F788FE43
:107430000546F9F74FFB002802D16948445D01E099
:107440006848445DE007C00F002807D06348C07952
:1074500000090001C01D6149C87105E05F48C0799D
:10746000000900015D49C87102202040002807D0B2
:107470005A48807900090001C01D5849887105E00B
:107480005648807900090001544988710420204041
:10749000002807D05148407900090001C01D4F491C
:1074A000487105E04D484079000900014B49487199
:1074B00008202040002807D04848007AF02188435F
:1074C00070304649087205E04448007AF02188434C
:1074D0004249087210202040002807D03F48007A17
:1074E00000090001C01D3D49087205E03B48007AD3
:1074F00000090001394908722020204000280BD0E3
:107500003648C079F021884370303449C87109E0A9
:10751000AEE242E1F4E0A4E03048C079F0218843D3
:107520002E49C87140202040002807D02B484079C0
:10753000F021884370302949487105E02748407997
:10754000F0218843254948710A210398F0F7F8FD96
:107550000D462348445DE007C00F002807D01F48B0
:10756000C07800090001C01D1C49C87005E01B4817
:10757000C078000900011949C87002202040002885
:1075800007D016488078F0218843703013498870FE
:1075900005E012488078F021884310498870042063
:1075A0002040002807D00D484078F02188437030F3
:1075B0000A49487005E009484078F02188430749A6
:1075C00048700820204000280ED004484078000968
:1075D0000001C01D014948700CE000008426002015
:1075E0002C1002003F100200FE4840780009000104
:1075F000FC49487010202040002807D0F948007945
:1076000000090001C01DF749087105E0F54800793F
:1076100000090001F349087120202040002807D00C
:10762000F048C078F02188437030EE49C87005E01A
:10763000EC48C078F0218843EA49C87040202040D7
:10764000002807D0E748807800090001C01DE549FF
:107650008870B8E2E348807800090001E149887049
:10766000B1E2E0484079F02188437030DD4948714B
:107670000846807800090001C01D88700846C0795E
:1076800000090001C871084680790009000188716D
:10769000084640790009000148710846007AF02147
:1076A0008843D04908720846007A00090001087230
:1076B0000846C079F0218843CA49C8710846C07895
:1076C00000090001C87008468078F0218843C54948
:1076D000887008464078F0218843C24948700846BF
:1076E000407800090001487008460079000900014F
:1076F00008710846C078F0218843BA49C87062E230
:10770000B8484079F0218843B649487108468078E6
:107710000009000188700846C07900090001C8719D
:1077200008468079000900018871084640790009FF
:10773000000148710846007AF0218843A94908727F
:107740000846007A0009000108720846C079F02155
:107750008843A449C8710846C07800090001C87070
:1077600008468078F02188439E4988700846407812
:10777000F02188439B494870084640780009000181
:107780004870084600790009000108710846C07871
:10779000F02188439349C87015E2012F73D10A2163
:1077A0000398F0F7CDFC0546F9F794F9002802D1CB
:1077B0008D48445D01E08D48445DE007C00F00281E
:1077C00007D08848C07900090001C01D8549C871EB
:1077D00005E08448C079000900018249C87102208F
:1077E0002040002807D07F48807900090001C01D93
:1077F0007C49887105E07B4880790009000179495E
:10780000887104202040002807D07648407900097C
:107810000001C01D7349487105E0724840790009B4
:1078200000017049487108202040002807D06D48A9
:10783000007AF021884370306A49087205E069488F
:10784000007AF02188436749087210202040002800
:1078500007D06448007A00090001C01D6149087220
:1078600005E06048007A000900015E4908722020A6
:107870002040002808D05B48C079F0218843703050
:107880005849C87106E09DE05648C079F021884308
:107890005449C87140202040002807D05148407901
:1078A000F021884370304F49487105E04D484079D8
:1078B000F02188434B4948710A210398F0F740FCB6
:1078C0000D464948445DE007C00F002807D04548F1
:1078D000C07800090001C01D4249C87005E0414858
:1078E000C078000900013F49C870022020400028EC
:1078F00007D03C488078F02188437030394988703F
:1079000005E038488078F0218843364988700420A3
:107910002040002807D033484078F0218843703059
:107920003049487005E02F484078F02188432D49C0
:10793000487008202040002807D02A4840780009D5
:107940000001C01D2749487005E02648407800091D
:1079500000012449487010202040002807D0214809
:10796000007900090001C01D1E49087105E01D488D
:107970000079000900011B490871202020400028DF
:1079800007D01848C078F021884370301549C87076
:1079900005E01448C078F02188431249C87040209F
:1079A0002040002807D00F48807800090001C01D42
:1079B0000C49887007E10B488078000900010949EB
:1079C000887000E107484079F0218843703005490C
:1079D00048710846807800090001C01D887008467B
:1079E000C07905E0842600202C1002003F10020020
:1079F00000090001C87108468079000900018871FA
:107A0000084640790009000148710846007AF021D3
:107A100088436E4908720846007A0009000108721E
:107A20000846C079F02188436849C8710846C07883
:107A300000090001C87008468078F0218843634936
:107A4000887008464078F0218843604948700846AD
:107A500040780009000148700846007900090001DB
:107A600008710846C078F02188435849C870AAE0D8
:107A7000032E9FD1F9F70EF9002858D053484079CA
:107A8000F0218843703051494871084680780009D8
:107A90000001C01D88700846C07900090001C01DA2
:107AA000C8710846807900090001C01D8871084628
:107AB000407900090001C01D48710846007AF02194
:107AC00088437030414908720846007A0009000175
:107AD00008720846C079F021884370303B49C8716C
:107AE0000846C07800090001C01DC87008468078AB
:107AF000F021884370303549887008464078F0217D
:107B000088437030314948700846407800090001C8
:107B1000C01D487008460079000900010871084638
:107B2000C078F021884370302849C8704BE027485E
:107B30004079F0218843254948710846807800093A
:107B4000000188700846C07900090001C871084624
:107B50008079000900018871084640790009000118
:107B600048710846007AF02188431849087208468F
:107B7000007A0009000108720846C079F0218843A4
:107B80001249C8710846C07800090001C87008464B
:107B90008078F02188430D49887008464078F021AC
:107BA00088430A4948700846407800090001487037
:107BB000084600790009000108710846C078F021E4
:107BC00088430249C87005B0F0BD0000842600203B
:107BD00070B505460C46012D7ED1B348407D0009A5
:107BE0000001C01DB04948750846007DF02188435A
:107BF0001030AD4908750846007D00090001401CA1
:107C000008750846C07CF02188431030A649C87426
:107C10000846807CF02188431030A34988740846C8
:107C2000807C00090001401C8874F9F78BF8022859
:107C300003D0F9F787F801286ED19C480078012815
:107C40006AD0F4F791FE9A49884265D3F9F722F891
:107C500000282FD09448007DF0218843703092494D
:107C600008750846007D00090001C01D087508461A
:107C7000C07CF021884370308B49C8740846807CF2
:107C8000F02188437030884988740846807C000958
:107C90000001C01D88740846407DF0218843703083
:107CA000814948750846407CF021884370307E4900
:107CB0004874F8E07C48007DF021884310307A4910
:107CC00008750846007D00090001401C087508463B
:107CD000C07CF021884300E0B8E010307249C874DD
:107CE0000846807CF021884310306F49887408462C
:107CF000807C00090001401C88740846407DF0210A
:107D000088431030684948750846407CF021884314
:107D1000103065494874C6E0F8F78AFE002826D17D
:107D2000F4F722FE6249884221D3F8F7B3FF002816
:107D30000ED05D48407DF021884370305A49487527
:107D40000846407CF02188437030574948741CE055
:107D50005548407DF0218843103053494875084606
:107D6000407CF021884310304F4948740DE04E4864
:107D7000407DF021884370304B4948750846407C6F
:107D8000F0218843703048494874F8F751FE0128C3
:107D90002AD146480078012826D0F4F7E5FD444969
:107DA000884221D34048407DF021884370303E49CD
:107DB00048750846407CF021884370303A49487441
:107DC000F8F768FF002807D03748007DF021884386
:107DD00070303549087566E03348007DF0218843EE
:107DE0001030314908755EE0230008F085F9062C53
:107DF000241C140C042D2C48807C00090001C01D9B
:107E00002949887400BF2848807CF021884370305D
:107E10002549887400BF2448C07CF0218843703015
:107E20002149C87400BF2048007D00090001C01D21
:107E30001D49087500BF1C48007DF0218843703043
:107E40001949087500BF00E000BF2CE01648407DCE
:107E5000F0218843144948750846007DF021884385
:107E6000114908750846007D00090001087508469B
:107E7000C07CF02188430C49C8740846807CF021FE
:107E80008843094988740846807C00090001887489
:107E90000846407D0009000148750846407CF021F5
:107EA00088430149487470BD64260020FD0000200D
:107EB000B80B000030B50246002901D1002000E0D7
:107EC0000720130008F018F90F09141F2B3743502F
:107ED0005D67727C88929FA9B500574B5B7EF0244A
:107EE000A3430401F0252C402343534C6376A1E0C7
:107EF000524B9B79F024A3430401F0252C402343EB
:107F00004E4CA37196E04D4B2033DB791B091B01CE
:107F10000407240F2343494C2034E3718AE0464B85
:107F20002033DB7C1B091B010407240F2343424C35
:107F30002034E3747EE0404B40331B781B091B0167
:107F40000407240F23433C4C4034237072E03A4B27
:107F50002033DB7FF024A3430401F0252C4023438E
:107F6000354C2034E37765E0334B20335B7BF024E2
:107F7000A3430401F0252C4023432F4C203463738A
:107F800058E02E4B9B791B091B010407240F234348
:107F90002A4CA3714EE0294B9B7CF024A34304019F
:107FA000F0252C402343254CA37443E0234BDB7E78
:107FB0001B091B010407240F2343204CE37639E0FF
:107FC0001D4B2033DB7F1B091B010407240F2343B8
:107FD000194C2034E3772DE0174B9B7E1B091B01C6
:107FE0000407240F2343144CA37623E0134B2033C0
:107FF0009B79F024A3430401F0252C4023430F4C2C
:108000002034A37116E00D4BDB7D1B091B01040717
:10801000240F2343094CE3750CE0074B20335B7CB2
:108020001B091B010407240F2343034C20346374F2
:1080300000E000BF00BF30BD44260020182700200C
:10804000F7B582B00746154600260024FE480078A2
:10805000012804D0F4F788FCFC49884279D2FC4816
:10806000407CF02188437030F94948740846807C90
:1080700000090001C01D88740846007D0009000148
:10808000C01D08750846007DF02188437030F04916
:1080900008750846807CF02188437030EC4988746C
:1080A0000846C07C00090001C01DC8740846C07C99
:1080B000F02188437030E649C8740846407C0009C6
:1080C0000001C01D48740846407D00090001C01D24
:1080D00048750846407DF02188437030DC4948757A
:1080E0000846007CF02188437030D949087408465E
:1080F000007C00090001C01D08740846C07BF02107
:1081000088437030D249C873FF220A210020FBF750
:108110009DF9FF2213210020FBF798F9FF2211217E
:108120000020FBF793F9FF2212210020FBF78EF9C4
:10813000FF220E210020FBF789F9FF220F210020EA
:10814000FBF784F9FF2210210020FBF77FF9F4E30D
:10815000FFE7039836283DD019DC08287ED007DCDD
:10816000801E030007F0C8FF0635A8FCFBFAF97E65
:10817000102874D006DC092872D00D2871D00E2882
:1081800070D1FDE333286ED03428F9D170E13F2857
:108190006AD00FDC3738082864D243007B449B88C0
:1081A0005B009F448A009702FF025F005F00650347
:1081B000CB0318004E287BD006DC402879D041281C
:1081C00078D04D28DCD1BBE14F2874D05028D7D1CE
:1081D0004FE100BF00BF9E48407CF02188439C498E
:1081E00048740846807C0009000188740846007DB8
:1081F00000090001C01D08750846007DF021884374
:108200007030934908750846807CF0218843904976
:1082100088740846C07C00090001C01DC874084667
:10822000C07CF02188438A49C8740846407C000914
:10823000000148740846407D000900014875084661
:10824000407DF0218843824948750846007CF02132
:1082500088437F4908740846007C06E0A1E2FDE3FC
:1082600037E2D2E3FBE394E028E000090001087460
:108270000846C07BF02188437549C873FF220A2154
:108280000020FBF7E3F8FF2213210020FBF7DEF8C4
:1082900000220E211046FBF7D9F800220F211046CC
:1082A000FBF7D4F8002210211046FBF7CFF877E255
:1082B000ABE110E2DDE26DE000BF00BF6448407C4E
:1082C000F0218843624948740846807C0009000117
:1082D00088740846007D00090001C01D0875084625
:1082E000007DF02188437030594908750846807C2C
:1082F000F0218843564988740846C07C0009000173
:10830000C8740846C07CF02188435149C8740846A7
:10831000407C0009000148740846407D00090001C6
:10832000C01D48750846407DF0218843484948757E
:108330000846007CF0218843454908740846007CC3
:108340000009000108740846C07BF02188434049B9
:10835000C873FF220A21002003E055E1EFE086E028
:1083600016E0FBF773F8FF2213210020FBF76EF8ED
:1083700000220E211046FBF769F800220F2110465B
:10838000FBF764F8002210211046FBF75FF88EE738
:1083900000BF00BF2E48407CF02188432C49487420
:1083A0000846807C00090001C01D88740846007DD5
:1083B00000090001C01D08750846007DF0218843B2
:1083C0007030234908750846807CF021884370305E
:1083D0001F4988740846C07C00090001C87408461B
:1083E000C07CF02188431A49C8740846407C0009C3
:1083F000000148740846407D0009000148750846A0
:10840000407DF0218843124948750846007CF021E0
:1084100088430F4908740846007C0009000108746D
:108420000846C07BF02188430949C873FF220A210E
:108430000020FBF70BF8FF2213210020FBF706F8C2
:1084400000220E21104605E0FD000020B80B0000C0
:1084500084260020FAF7FAFF00220F211046FAF7CF
:10846000F5FF002210211046FAF7F0FF1FE700BFCA
:1084700000BFFE48407CF0218843FC494874084610
:10848000807C00090001C01D88740846007D000939
:108490000001C01D08750846007DF021884370303A
:1084A000F24908750846807CF0218843EF498874BA
:1084B0000846C07C00090001C8740846C07CF02151
:1084C0008843EA49C8740846407C00090001C01D81
:1084D00048740846407D0009000148750846407D03
:1084E000F0218843E14948750846007CF021884323
:1084F000DE4908740846007C00090001087408463B
:10850000C07BF0218843D949C873FF220A2100208B
:10851000FAF79CFFFF2213210020FAF797FF0022B1
:108520000E211046FAF792FF00220F211046FAF7AB
:108530008DFF002210211046FAF788FFF6E300BFF6
:10854000CA48407CF0218843C84948740846807C6A
:108550000009000188740846007D000900010875C3
:108560000846007DF02188437030C04908750846F0
:10857000807CF0218843BD4988740846C07C00098E
:108580000001C8740846C07CF02188437030B749A8
:10859000C8740846407C0009000148740846407DC4
:1085A0000009000148750846407DF0218843AF4925
:1085B00048750846007CF0218843AC490874084699
:1085C000007C0009000108740846C07BF021884344
:1085D000A649C873FF220A210020FAF737FFFF22BD
:1085E00013210020FAF732FF00220E211046FAF77D
:1085F0002DFF00220F211046FAF728FF002210213C
:108600001046FAF723FF91E300BF9848407CF02121
:108610008843964948740846807C000900018874A4
:108620000846007D0009000108750846007DF0211C
:10863000884370308D4908750846807CF021884356
:108640008A4988740846C07C00090001C87408463D
:10865000C07CF02188438549C8740846407C0009E5
:10866000000148740846407D00090001487508462D
:10867000407DF021884370307C4948750846007C75
:10868000F0218843794908740846007C00090001FC
:1086900008740846C07BF02188437449C873FF22E0
:1086A0000A210020FAF7D2FEFF2213210020FAF758
:1086B000CDFE00220E211046FAF7C8FE00220F213F
:1086C0001046FAF7C3FE002210211046FAF7BEFE4C
:1086D0002CE300BF00BF6548407CF0218843703028
:1086E000624948740846807C00090001C01D8874F6
:1086F0000846007D00090001C01D08750846007D80
:10870000F02188437030594908750846807CF02173
:108710008843564988740846C07C00090001C87423
:108720000846C07CF02188435049C8740846407C04
:108730000009000148740846407D000900014875A1
:108740000846407DF0218843484948750846007C2A
:10875000F0218843454908740846007C000900015F
:1087600008740846C07BF02188434049C873FF2243
:108770000A210020FAF76AFEFF2213210020FAF7EF
:1087800065FE00220E211046FAF760FE00220F213E
:108790001046FAF75BFE002210211046FAF756FE4B
:1087A000C4E200BF3148407CF02188432F4948741F
:1087B0000846807C0009000188740846007D000995
:1087C000000108750846007DF02188437030274974
:1087D00008750846807CF02188432449887408463F
:1087E000C07C00090001C8740846C07CF0218843A1
:1087F00070301E49C8740846407C00090001487466
:108800000846407D0009000148750846407DF0217A
:108810008843164948750846007CF021884313496F
:1088200008740846007C0009000108740846C07BF3
:10883000F02188430D49C873FF220A210020FAF76E
:1088400005FEFF2213210020FAF700FE00220E2170
:108850001046FAF7FBFD00220F211046FAF7F6FD4D
:10886000002210211046FAF7F1FD5FE28426002075
:1088700000BFFC48407CF0218843FA494874084610
:10888000807C0009000188740846007D0009000111
:1088900008750846007DF02188437030F14908755D
:1088A0000846807CF0218843EE4988740846C07CE5
:1088B00000090001C8740846C07CF0218843E949DA
:1088C000C8740846407C0009000148740846407D91
:1088D0000009000148750846407DF021884370304A
:1088E000E04948750846007CF0218843DD4908745A
:1088F0000846007C0009000108740846C07BF0218E
:108900008843D849C873FF220A210020FAF79EFD48
:10891000FF2213210020FAF799FD00220E211046B4
:10892000FAF794FD00220F211046FAF78FFD00227E
:1089300010211046FAF78AFDF8E1F8E1C948407CB9
:10894000F02188437030C74948740846807C00098C
:108950000001C01D88740846007D00090001C01D8B
:1089600008750846007DF0218843BE490875084611
:10897000807CF0218843BB4988740846C07C00E0B5
:10898000A9E000090001C8740846C07CF0218843B2
:10899000B449C8740846407C000900014874084680
:1089A000407D0009000148750846407DF02188435C
:1089B000AC4948750846007CF0218843A9490874F1
:1089C0000846007C0009000108740846C07BF021BD
:1089D0008843A449C873FF220A210020FAF736FD14
:1089E000FF2213210020FAF731FD00220E2110464C
:1089F000FAF72CFD00220F211046FAF727FD00227E
:108A000010211046FAF722FD90E19648407CF021B3
:108A10008843944948740846807C000900018874A2
:108A20000846007D0009000108750846007DF02118
:108A300088438C4908750846807CF0218843894921
:108A400088740846C07C00090001C8740846C07CD0
:108A5000F02188438349C874084601E09EE003E1A1
:108A6000407C0009000148740846407D000900016F
:108A700048750846407DF02188437A494875084684
:108A8000007CF0218843774908740846007C00097F
:108A9000000108740846C07BF0218843703071499A
:108AA000C87300220A211046FAF7D0FC00221321D5
:108AB0001046FAF7CBFCFF220E210020FAF7C6FC85
:108AC00000220F211046FAF7C1FC002210211046A7
:108AD000FAF7BCFC2AE16348407CF02188436149F5
:108AE00048740846807C0009000188740846007DAF
:108AF0000009000108750846007DF02188435949A6
:108B000008750846807CF0218843564988740846D9
:108B1000C07C00090001C8740846C07CF02188436D
:108B20005049C8740846407C000900014874084652
:108B3000407D0009000148750846407DF0218843CA
:108B4000484948750846007CF02188434549087427
:108B50000846007C00090001C01D08740846C07B5F
:108B6000F02188433F49C87300220A211046FAF7D2
:108B70006DFC002213211046FAF768FC00220E213A
:108B80001046FAF763FCFF220F210020FAF75EFC83
:108B9000002210211046FAF759FCC7E03148407C0A
:108BA000F02188432F4948740846807C0009000161
:108BB00088740846007D0009000108750846007D9C
:108BC000F0218843274908750846807CF0218843B6
:108BD000244988740846C07C00090001C87408460E
:108BE000C07CF02188431F49C8740846407C0009B6
:108BF000000148740846407D000900014875084698
:108C0000407DF0218843174948750846007CF021D3
:108C100088437030134908740846007C000900013D
:108C200008740846C07BF02188430E49C8730022AF
:108C30000A211046FAF70AFC002213211046FAF71F
:108C400005FC00220E211046FAF700FC00220F213D
:108C50001046FAF7FBFBFF2210210020FAF7F6FB83
:108C600064E0000084260020FB48407CF02188431B
:108C7000F94948740846807C000900018874084658
:108C8000007D0009000108750846007DF021884339
:108C9000F14908750846807CF0218843EE498874C4
:108CA0000846C07C00090001C8740846C07CF02159
:108CB0008843E949C8740846407C000900014874AB
:108CC0000846407D0009000148750846407DF021B6
:108CD0008843E14948750846007CF0218843DE4915
:108CE00008740846007C0009000108740846C07B2F
:108CF000F0218843D849C87300220A211046FAF7A8
:108D0000A5FB002213211046FAF7A0FB00220E213A
:108D10001046FAF79BFB00220F211046FAF796FB4C
:108D2000002210211046FAF791FB00BF00BF002F70
:108D300003D0CA48007A002804D1F3F715FEC849C9
:108D4000884272D2FF2211210020FAF77FFBFF2216
:108D500012210020FAF77AFBC2480078012804D0DB
:108D6000F3F702FEBE49884216D2BF48807BF0214D
:108D700088437030BC498873084640300078F02141
:108D800088437030B84940310870084600780009BF
:108D90000001C01D08702DE07D20C000854214D266
:108DA000B148807BF0218843AF4988730846403042
:108DB0000078F02188437030AB4940310870084694
:108DC000007800090001087014E0A748807BF021BA
:108DD00088437030A4498873084640300078F021F9
:108DE0008843A14940310870084600780009000115
:108DF000C01D08707D20C000854205D2014628466E
:108E0000EFF79EF9064604E098492846EFF798F9EF
:108E1000064694480078012804D0F3F7A5FD904950
:108E2000884203D29248845D02E0A0E29148845DCA
:108E3000E007C00F002809D08B484030C0780009F7
:108E40000001C01D88494031C87007E086484030A5
:108E5000C0780009000184494031C87002202040D8
:108E6000002807D08048C07900090001C01D7E4954
:108E7000C87105E07C48C079000900017A49C871D1
:108E800004202040002807D077488079000900019D
:108E9000C01D7549887105E073488079000900019B
:108EA0007149887108202040002807D06E48407919
:108EB000F021884370306C49487105E06A48407978
:108EC000F02188436849487110202040002807D0CD
:108ED0006548407900090001C01D6349487105E0FB
:108EE00061484079000900015F4948712020204015
:108EF000002807D05C480079F021884370305A4937
:108F0000087105E058480079F021884356490871F6
:108F100040202040002807D053488079F021884322
:108F200070305149887105E04F488079F0218843BD
:108F30004D4988717D20C000854213D264212846A6
:108F4000EFF7FEF8064647480078012804D0F3F70B
:108F50000BFD4349884202D24548845D23E04548E1
:108F6000845D20E0642128463230EFF7E9F87D2166
:108F7000C9000090EFF7E4F8019164210198EFF740
:108F8000DFF806463C48854208D23648007801287A
:108F900004D0F3F7E9FC3249884202D23448845DB8
:108FA00001E03448845DE007C00F002809D02E4856
:108FB00040308078F021884370302B4940318870F0
:108FC00007E0294840308078F02188432649403125
:108FD000887002202040002807D02348807A0009AA
:108FE0000001C01D2049887205E01F48807A0009F1
:108FF00000011D49887204202040002807D01A482B
:10900000407A00090001C01D1749487205E0164862
:10901000407A0009000114494872082020400028C5
:1090200007D01148007AF021884370300E49087249
:1090300005E00D48007AF02188430B4908721020A2
:10904000204000281AD00848007A00090001C01DFD
:109050000549087218E0000084260020540A002008
:10906000B80B0000FD000020F8260020A0860100BB
:109070002C1002003F10020010270000FE48007A6A
:1090800000090001FC49087220202040002807D078
:10909000F948C079F02188437030F749C87105E07C
:1090A000F548C079F0218843F349C8714020204039
:1090B000002807D0F048407AF02188437030EE490C
:1090C000487205E0EC48407AF0218843EA4948724A
:1090D0007D20C000854219D20A212846EFF730F8DA
:1090E0000A210190EFF72CF80E460A2D08D2E3482A
:1090F0000078012804D0F3F737FCE149884202D216
:10910000E048845D12E0E048845D0FE06421284679
:109110003230EFF715F80A210090EFF711F80A2125
:109120000190EFF70DF80E46D6498C5DE007C00FB1
:10913000002809D0D0484030807800090001C01DC7
:10914000CD494031887007E0CB4840308078000935
:109150000001C9494031887002202040002807D012
:10916000C548807B00090001C01DC349887305E024
:10917000C148807B00090001BF498873042020405A
:10918000002807D0BC48407B00090001C01DBA4937
:10919000487305E0B848407B00090001B6494873B0
:1091A00008202040002807D0B348007BF0218843E6
:1091B0007030B149087305E0AF48007BF021884367
:1091C000AD49087310202040002807D0AA48C07A73
:1091D00000090001C01DA849C87205E0A648C07A70
:1091E00000090001A449C87220202040002807D0AF
:1091F000A148807AF021884370309F49887205E049
:109200009D48807AF02188439B4988724020204005
:10921000002807D09848407BF02188437030964959
:10922000487305E09448407BF02188439249487395
:109230007D20C000854207D20A212846EEF780FF34
:109240000E469048845D0BE0642128463230EEF7EC
:1092500077FF0A210190EEF773FF0E4689498C5D76
:10926000E007C00F002809D0834840304078F02143
:109270008843703080494031487007E07E48403074
:109280004078F02188437C494031487002202040DA
:10929000002809D078484030407800090001C01DFE
:1092A00075494031487007E0734840304078000904
:1092B000000171494031487004202040002807D047
:1092C0006D48007CF021884370306B49087405E0DC
:1092D0006948007CF02188436749087408202040D1
:1092E000002807D06448007C00090001C01D6249C5
:1092F000087405E06048007C000900015E490874BC
:1093000010202040002807D05B48C07BF021884314
:1093100070305949C87305E05748C07BF021884335
:109320005549C87320202040002807D05248C07BF0
:1093300000090001C01D5049C87305E04E48C07BBC
:10934000000900014C49C87340202040002807D084
:109350004948407C00090001C01D47494874ECE0C1
:109360004548407C0009000143494874E5E000227B
:109370000A211046FAF76AF8002213211046FAF77C
:1093800065F8002211211046FAF760F80022122138
:109390001046FAF75BF800220E211046FAF756F84D
:1093A00000220F211046FAF751F800221021104632
:1093B000FAF74CF830484030C078000900012E49D7
:1093C0004031C8702C48C079000900014039C8718B
:1093D0000846807900090001887108464079F0212B
:1093E00088432549487108464079000900014871C1
:1093F00008460079F02188431F49087108468079A2
:10940000F02188431C498871084640308078F0215B
:1094100088431949403188701748807A0009000153
:10942000403988720846407A0009000148720846AF
:10943000007AF0218843104908720846007A000932
:10944000000108720846C079F02188430A49C871B2
:109450000846407AF0218843074948720846403060
:10946000807800090001403188700348807B000942
:1094700000014039887309E0F8260020FD00002033
:10948000B80B00002C1002003F1002000846407B81
:109490000009000148730846007BF02188432849F1
:1094A00008730846C07A00090001C8720846807A2D
:1094B000F0218843224988720846407BF021884386
:1094C0001F494873084640304078F02188431C49C2
:1094D000403148700846407800090001487018483B
:1094E000007CF0218843164908740846007C000976
:1094F000000108740846C07BF02188431049C873F6
:109500000846C07B00090001C8730846407C00097A
:10951000000148740846807BF0218843084988731D
:10952000084640300078F0218843054940310870F2
:109530000846007800090001087005B0F0BD000081
:10954000F8260020F7B582B007460E460121FF201D
:109550000830FBF7A7FF0121FC48FBF7A3FFFC48FD
:10956000007801287ED0F3F7FFF9FA49884279D3D1
:10957000F7F770FA032843D1F7F766FA002803D00B
:10958000F7F762FA01283BD1002F1CD1F7F782FBD5
:1095900000280CD0F048407CF0218843EE49487404
:1095A0000846807C00090001C01D8874EEE0EA488E
:1095B000407CF0218843E84948740846807C0009D3
:1095C00000018874E2E0F7F765FB00280CD0E24860
:1095D000407CF02188437030DF4948740846807C25
:1095E000000900018874D1E0DB48407CF021884309
:1095F000D94948740846807C000900018874C5E098
:10960000F7F722FA002803D0F7F71EFA012865D1F0
:10961000002F0CD1D048407CF0218843CE494874BB
:109620000846807C00090001C01D88740BE0CA4810
:10963000407CF02188437030C74948740846807CDC
:10964000000900018874F7F7FFF9002821D1C2480A
:109650002030C078F02188437030BF492031C87075
:10966000BD4800E064E0807D000900012039887574
:109670000846807DF0218843B7498875FF22232161
:109680000020F9F7E3FE002222211046F9F7DEFE62
:109690007CE0F7F7D9F9012878D1AF482030C078BD
:1096A000F0218843AC492031C870AB48807D000967
:1096B0000001C01D203988750846807DF02188434F
:1096C0007030A5498875002223211046F9F7BEFEA7
:1096D000FF2222210020F9F7B9FE57E09E48407C86
:1096E000F02188439C4948740846807C00090001A9
:1096F000887408462030C078F0218843964920318C
:10970000C8709548807D0009000120398875084699
:10971000807DF021884390498875002223211046DE
:10972000F9F794FE002222211046F9F78FFE2DE072
:109730008948407CF0218843703087494874084646
:10974000807C00090001C01D887408462030C07864
:10975000F0218843703080492031C8707E48807D78
:1097600000090001C01D203988750846807DF02160
:109770008843703078498875FF2223210020F9F74B
:1097800065FEFF2222210020F9F760FEF7F75CF961
:10979000002808D06E480078012804D0F3F7E4F8D8
:1097A0006C49884276D26D48864209D96A48203091
:1097B0004079F0218843703067492031487107E0D3
:1097C000654820304079F021884363492031487151
:1097D00063493046EEF7B4FC0A210190EEF7B0FC85
:1097E0000D465E48401C864202D35E48445D01E05F
:1097F0005D48445DE007C00F002809D0564820307E
:10980000C07800090001C01D53492031C87007E02D
:1098100051482030C078000900014F492031C870FC
:1098200002202040002809D04B4820308078F021C9
:109830008843703048492031887007E0464820301E
:109840008078F021884344492031887004202040EA
:10985000002809D0404820304078F02188437030FB
:109860003D492031487007E03B4820304078F021E6
:1098700088433949203148700820204000280AD008
:1098800035482030407900090001C01D324920319F
:10989000487108E0A1E23048203040790009000119
:1098A0002D492031487110202040002809D02A4835
:1098B00020300079F0218843703027492031087129
:1098C00007E0254820300079F021884322492031E3
:1098D000087120202040002809D01F48203000793E
:1098E00000090001C01D1C492031087107E01A4819
:1098F000203000790009000117492031087140200B
:109900002040002809D01448203080780009000148
:10991000C01D11492031887007E00F482030807841
:10992000000900010C49203188707D21C9003046B2
:10993000EEF706FC0A210190EEF702FC0D460848FE
:10994000864213D30748445D12E00000050500007D
:10995000FD000020B80B0000F82600209F860100C3
:10996000102700002C1002003F100200F948445D4F
:10997000E007C00F002807D0F748C07FF0218843D8
:109980007030F549C87705E0F348C07FF02188437F
:10999000F149C87702202040002807D0EE48C07F58
:1099A00000090001C01DEC49C87705E0EA48C07F06
:1099B00000090001E849C87704202040002807D0AA
:1099C000E548807F00090001C01DE349887705E074
:1099D000E148807F00090001DF49887708202040A6
:1099E000002809D0DC482030407800090001C01D63
:1099F000D9492031487007E0D74820304078000925
:109A00000001D5492031487010202040002809D09D
:109A1000D14820300078F02188437030CE49203181
:109A2000087007E0CC4820300078F0218843CA490C
:109A30002031087020202040002809D0C64820305E
:109A4000007800090001C01DC3492031087007E0FB
:109A5000C1482030007800090001BF49203108705A
:109A600040202040002807D0BB48807FF021884359
:109A70007030B949887705E0B748807FF021884386
:109A8000B549887764213046EEF75AFB0A210190E8
:109A9000EEF756FB0D467D20C000864202D3AF484C
:109AA000445D01E0AB48445DE007C00F002807D0EB
:109AB000A948007F00090001C01DA749087705E0FB
:109AC000A548007F00090001A34908770220204033
:109AD000002807D0A048C07EF021884370309E49FE
:109AE000C87605E09C48C07EF02188439A49C87634
:109AF00004202040002807D09748807EF02188432A
:109B000070309549887605E09348807EF02188433F
:109B10009149887608202040002807D08E48407F51
:109B2000F021884370308C49487705E08A48407FAF
:109B3000F02188438849487710202040002807D02A
:109B40008548407F00090001C01D8349487705E032
:109B50008148407F000900017F494877202020404C
:109B6000002807D07C48007FF021884370307A4974
:109B7000087705E07848007FF02188437649087728
:109B800040202040002807D07348C07E0009000113
